:020000040000FA
:1000000000EFF6F08FEF00F0E9CF0BF1EACF0CF143
:10001000D9CF0DF171EF1AF0D8CF30F0E8CF31F031
:10002000E0CF32F0E9CF33F0EACF34F0E1CF35F072
:10003000E2CF36F0D9CF37F0DACF38F0F3CF39F05E
:10004000F4CF3AF0F6CF3BF0F7CF3CF0F8CF3DF0ED
:10005000F5CF3EF09DA001D001D00AD09EA001D0E6
:1000600001D006D09FB001D001D002D0BCECABF0E3
:10007000A0A201D001D00AD0A1A201D001D006D007
:10008000A2B201D001D002D076EC0BF09DA401D039
:1000900001D00AD09EA401D001D006D09FB401D0D7
:1000A00001D002D005EC3AF09DAA01D001D00AD0CF
:1000B0009EAA01D001D006D09FBA01D001D002D0B3
:1000C00057ECECF0A3AA01D001D00AD0A4AA01D029
:1000D00001D006D0A5BA01D001D002D00DEC34F089
:1000E0003EC0F5FF3DC0F8FF3CC0F7FF3BC0F6FF48
:1000F0003AC0F4FF39C0F3FF38C0DAFF37C0D9FF88
:1001000036C0E2FF35C0E1FF34C0EAFF33C0E9FF8B
:1001100032C0E0FF31C0E8FF30C0D8FF1000ADEFC3
:1001200017F0FFFFFFFFFFFFFFFFFFFFFFFFFFFFD6
:10013000FFFFFFFFFFFFFFFFFFFFFFFFFFFFFFFFCF
:10014000FFFFFFFFFFFFFFFFFFFFFFFFFFFFFFFFBF
:10015000FFFFFFFFFFFFFFFFFFFFFFFFFFFFFFFFAF
:10016000FFFFFFFFFFFFFFFFFFFFFFFFFFFFFFFF9F
:100400001F1F1F1B1B1B1B1B13131313131319116C
:10041000130919191919191919191B1D1919190075
:100420000005310791073207920733079307340716
:1004300094073505950599073907360537053805B9
:1004400098050000960544070A0314000101020004
:100450000000EFFF009091A5FF123400000303009D
:1004600033CC123403010104000A0206010000002B
:100470000F02033C02020800000000000000000020
:10048000090909090911780585054005410588050F
:100490008907900770007105696E7465726E6574E6
:1004A0002E6C6D742E6C76000000000000000000C1
:1004B000000000000000000000000000000000003C
:1004C00000000000000000003932330000323133F8
:1004D0002E32312E3139362E363800000047736DFA
:1004E00054736300000000000000000000000000E2
:1004F00000000000000000000000000000000000FC
:1005000000000000000000000000000000000000EB
:1005100000000000000000000000000000000000DB
:1005200000000000000000000000000000000000CB
:1005300000000000000000000000000000000000BB
:1005400000000000000000000000000000000000AB
:10055000000000000000000000000000000000009B
:10056000000000000000000000000000000000008B
:10057000000000000000000000000000000000007B
:10058000000000000000000000000000000000006B
:10059000000000000000000000000000000000005B
:1005A000000000000000000000000000000000004B
:1005B000000000000000000000000000000000003B
:1005C000000000000000000000000000000000002B
:1005D000000000000000000000000000000000001B
:1005E000000000000000000000000000000000000B
:1005F00000000000000000000000000000000000FB
:1006000000000000000000000000000000000000EA
:1006100000000000000000000000000000000000DA
:1006200000000000000000000000000000000000CA
:1006300000000000000000000000000000000000BA
:1006400000000000000000000000000000000000AA
:10065000000000000000000000000000000000009A
:10066000000000000000000000000000000000008A
:10067000000000000000000000000000000000007A
:10068000000000000000000000000000000000006A
:10069000000000000000000000000000000000005A
:1006A000000000000000000000000000000000004A
:1006B00000000000460545054205430501A0A1A232
:1006C000A3A4A5A6A7A8A9AAABACADAEAF01B0B133
:1006D000B2B3B4B5B6B7B8B9BABBBCBDBEBF01C042
:1006E000C1C2C3C4C5C6C7C8C9CACBCCCDCECFD082
:1006F000D1D2D3D4D5D6D7D8D9DADBDCDDDEDFE072
:10070000E1E2E3E4E5E6E7E8E9EAEBECEDEEEF0051
:1007100000000000000000000000000000000000D9
:10072000696E7465726E6574000000000000000060
:1007300000000000000000000000000000000000B9
:1007400000000000000000000000000000000000A9
:10075000033E033E033E033E033E00000000000054
:100760000000000000000000000000000000000089
:100770000000000000000000000000000000000079
:100780000000000000000000000000000000000069
:100790000000000000000000000000000000000059
:1007A0000000000000000000000000000000000049
:1007B0000000000000000000000000000000000039
:1007C0000000000000000000000000000000000029
:1007D0000000000000000000000000000000000019
:1007E0000000000000000000000000000000000009
:1007F00000000000000000000000000000000000F9
:1008000001011B6B1C6B0601315194EC44F01D6F10
:100810000601325194EC44F01E6F000E42EC34F0AD
:100820001B510001F06F01011B6B1C6B0601345161
:1008300094EC44F01D6F0601355194EC44F01E6FAA
:10084000000E42EC34F01B510001F16F01011B6BF3
:100850001C6B0601375194EC44F01D6F06013851B2
:1008600094EC44F01E6F000E42EC34F01B5100017A
:10087000F26FF1C028F10101D8902833D8902833C5
:10088000D89028330001F039E842F80B0101281113
:100890000001F06FF2C028F10101D8902833000167
:1008A000F139E846E00B010128110001F16FF24136
:1008B000800BF26F01011B6B1C6B06012E5194EC37
:1008C00044F01D6F06012F5194EC44F01E6F000E92
:1008D00042EC34F01B51296F2945E846FC0B00011E
:1008E000F21301011B6B1C6B06012B5194EC44F0BD
:1008F0001D6F06012C5194EC44F01E6F000E42EC6B
:1009000034F01B51296F2941E8423F0B0001F213DB
:10091000F36B01012941E842C00B0001F31301010F
:100920001B6B1C6B0601285194EC44F01D6F0601F3
:10093000295194EC44F01E6F000E42EC34F01B5130
:10094000296FD89029310001F313F46B010129417B
:10095000800B0001F411F46F120000011EA466D098
:10096000000E4424D96EDA6A0B0EDA22F9C0DFFFDA
:10097000442A44500201A619A711D8A41200A66B5C
:10098000A76B11D0000E0201A625D96EDA6A0B0EF4
:10099000DA22000EA625E16EE26A0A0EE222DFCF1D
:1009A000E7FFA64BA72B44C01FF0206A1F50A65D8F
:1009B0002050A759E7E30D8C446A00011E941200F1
:1009C0000001F951490AD8A41200442A120000017A
:1009D000F951500AFAE0446A12000001F951440A40
:1009E000FAE10201FA6BC26BC36BEFD70001F95158
:1009F0003A0AF1E0F951D00F0201FA6FE6D700018F
:100A0000F9513A0A23E0F951D00F0201C26FDDD744
:100A10000001F9513A0A1AE0F951D00F0201C36FEF
:100A2000D4D70001F9513A0AD6E110D04450C8E0B9
:100A3000010ACDE0030AD1E0010AD8E0070ADFE0AD
:100A4000010AE6E0030AD8A41200EBD7446A0201C7
:100A5000A66BA76BC26706D0C36704D0FAC2A6F222
:100A6000A76B1ED0C36708D0FA510A0DC251F324F8
:100A7000A66F000EF42013D0FA51640DF3CF1FF0CF
:100A8000F4CF20F0C2510A0DF3501F24216EF45010
:100A90002020226EC3512124A66F000E2220A76FB2
:100AA000A10EA65D000EA759D8B0120000011E8449
:100AB0001200E8CF64F1000114B202D0D890120005
:100AC00005C515F10101645192EC41F0F7E3050110
:100AD000D351070AF3E11F0ED325D96EDA6A050E4A
:100AE000DA22DF6A220E01015F6F050E606F5FC1BF
:100AF0001BF160C11CF1ABEC1CF01BC161F11CC10E
:100B000062F161C11FF162C120F128EC40F0D6E32F
:100B100006BA4ED0000115A82ED0068A0788099083
:100B20000201CA6B08BE8A9C468405012051300A26
:100B300010E1020E0101166FFE0E156F32EC1BF074
:100B40000101186B540E176F3F0E196FD6EC36F07B
:100B50000FD0020E0101166FCC0E156F32EC1BF098
:100B60000101186B540E176F1F0E196FD6EC36F07B
:100B70000001469410D0B1EC0FF001016439F00B84
:100B8000636F480E4A6F63518CECF2F0050105511A
:100B900029EC46F002E2D88012006451C3EC3EF02A
:100BA0000101636F63C158F1645124ECE8F0F3D79D
:100BB0000A9C0A9A0B9409900201CA6B08BE8A9C8F
:100BC000069A468419A610D0020E0101166FDD0E9A
:100BD000156F32EC1BF00101186B540E176F2F0EBE
:100BE000196FD6EC36F00FD0020E0101166FDD0E34
:100BF000156F32EC1BF00101186B540E176F0F0EBE
:100C0000196FD6EC36F00798B3D72DC133F12EC14A
:100C100034F12E512D110AE12BC115F12CC116F121
:100C200024EC38F015C133F116C134F133C115F19C
:100C300034C116F162EC25F015C135F116C136F15B
:100C400020EE02F03551D9263651DA22DF50FDEC84
:100C500044F0306F20EE03F03551D9263651DA22B8
:100C6000DF50FDEC44F0316F20EE04F03551D92611
:100C70003651DA22DF50FDEC44F0326F09A409D07E
:100C8000FA0E0101176F170E166F010EA3EC33F069
:100C900008D0FA0E0101176F0C0E166F010EA3ECAF
:100CA00033F0010130515CEC44F0010131515CEC56
:100CB00044F0010132515CEC44F00D0E5CEC44F068
:100CC000B3EC46F00AD089EC46F007E3AFEC46F00F
:100CD00001012F6F2F513E0A0DE07BEC46F0890E8B
:100CE0000101295D130E2A59EEE31B0E5CEC44F062
:100CF000D89012002BC116F12CC117F1000EA3ECF5
:100D000033F00301B26BB36B02941CD0ABECEAF08E
:100D100002A418D002940201CE6701D013D0080EAD
:100D200001011C6FA00E1B6FFD0E1E6F6B0E1D6F61
:100D3000206B070E1F6F0AEC28F01C511B1102E1FB
:100D4000D8801200310E0301B25D750EB359DEE397
:100D50001B0E5CEC44F0CCD7E8CF1AF1C1C1FCF417
:100D6000C12965E1200E01011A25D96EDA6A050153
:100D7000050EDA22DF5094EC44F0186F1F0E0101CB
:100D80001A25D96EDA6A0501050EDA22DF5094ECD5
:100D900044F07BD8FC6F280E01011A25D96EDA6A5F
:100DA0000501050EDA22DF5094EC44F0186F270E8F
:100DB00001011A25D96EDA6A0501050EDA22DF5023
:100DC00094EC44F062D8FD6F2C0E01011A25D96E07
:100DD000DA6A0501050EDA22DF5094EC44F0186F50
:100DE000290E01011A25D96EDA6A0501050EDA22EB
:100DF000DF5094EC44F049D8FE6F2E0E01011A2505
:100E0000D96EDA6A0501050EDA22DF5094EC44F05F
:100E1000186F2D0E01011A25D96EDA6A0501050E2B
:100E2000DA22DF5094EC44F030D8FF6F28D0C105AF
:100E300006E10401FD6BFE6BC4C1FFF420D0C1517B
:100E4000020A03E0C151030A07E1C4C1FDF4C5C1B0
:100E5000FEF4C6C1FFF413D0C151060A03E0C1512C
:100E6000070A0DE1C4C1FDF4C6C118F10F0E181731
:100E7000C551F00B18110401FE6FC7C1FFF4040E39
:100E80000101176FFC0E166F1200196F193BF00E5F
:100E9000191719511811040112000101476B03AA17
:100EA00096D0039A880E0101296F130E2A6F2B6BBF
:100EB0002C6B010E2D6FFCEC9FF001014B6F4B5121
:100EC000370A03E04B510C0AEDE14B51370A70E150
:100ED00006019551220A6CE105011E6B01014B6B65
:100EE000960E01014B25D96EDA6A0601060EDA224A
:100EF000220EDF6201D016D0960E01014B25D96E6D
:100F0000DA6A060EDA220E0E4B25E16EE26A050160
:100F1000050EE222DFCFE7FF1E2B01014B2B0F0E48
:100F20004B65DED789ECE4F04A6F4A5141E0050E8B
:100F30004A613ED04A0504E1020E496F520E11D0BB
:100F40004A51020A04E1020E496F630E0AD04A5167
:100F5000030A04E1020E496F740E03D0020E496FBA
:100F6000850E486F0501D36B01014B6B1F0E01010C
:100F70004B25D96EDA6A050EDA224B514825186FD7
:100F8000000E4921196FE5EC2FF0DF6E1F0E0101F5
:100F90004B25D96EDA6A0501050EDA22DF5006E02C
:100FA000D32B01014B2B100E4B65E0D74AC147F103
:100FB000FF0E0101176FE50E166F010EA3EC33F063
:100FC000130E01012A6F880E296FD8EC38F0010149
:100FD0004751120020EE04F01E51D9261F51DA228B
:100FE00010EE06F01E51E1261F51E222DFCFE7FF8F
:100FF00020EE03F01E51D9261F51DA2210EE05F023
:101000001E51E1261F51E222DFCFE7FF20EE02F062
:101010001E51D9261F51DA2210EE04F069D810EEC5
:1010200003F066D8D051DF6E20EE02F01E51D926B3
:101030001F51DA22CFC1DFFF20EE05F01E51D92665
:101040001F51DA22DF50216F206B226B0F0E21150A
:10105000236F20EE06F01E51D9261F51DA22DF50F1
:101060002211246F2351256F24C115F125C116F1DA
:1010700062EC25F015C126F116C127F120EE06F02D
:101080001E51D9261F51DA22DF6A20EE06F01E51CA
:10109000D9261F51DA2210EE04F02651E1262751FD
:1010A000E222E750206F10EE03F02651E12627518F
:1010B000E222E750216F2139F00B2011DF6E20EE84
:1010C00005F01E51D9261F51DA22F00EDF1620EE50
:1010D00002F02651D9262751DA22DF50206F20EE68
:1010E00005F01E51D9261F51DA222051DF121200BD
:1010F0001E51E1261F51E222DFCFE7FF20EE01F073
:101100001E51D9261F51DA221200010E8DECDAF0A1
:1011100004E2010E8DECDAF014E3426B0AD03D6B71
:101120006AD80E0E0101422583D8D6EC36F00101B3
:10113000422B6CD8F4E33D6B5ED8000E196BD6ECF5
:1011400036F0020E8DECDAF004E2020E8DECDAF0ED
:1011500016E3426B0BD0110E3D6F4DD80E0E010100
:10116000422566D8D6EC36F00101422B4FD8F3E386
:10117000110E3D6F40D8000E196BD6EC36F0030E01
:101180008DECDAF004E2030E8DECDAF016E3426B3C
:101190000BD0220E3D6F2FD80E0E0101422548D8EC
:1011A000D6EC36F00101422B31D8F3E3220E3D6F2D
:1011B00022D8000E196BD6EC36F0040E8DECDAF066
:1011C00005E2040E8DECDAF0D8A01200426B0BD0D1
:1011D000330E3D6F10D80E0E0101422529D8D6ECF2
:1011E00036F00101422B12D8F3E3330E3D6F03D8E2
:1011F000196BD6EF36F0010E3E6F3D514225176F49
:10120000000E42BFFF0E3E21186F12001EC53DF1B9
:1012100001013E6B42C13FF1406B3FBF400740516F
:10122000800A416F3D513F5D3E51800A4159120095
:10123000D96EDA6A050EDA22DF50196F1200E8CF94
:1012400037F1000111A4000C11A41200130E0101CA
:10125000196F6A0E186FE5EC2FF0386F3851800A5D
:10126000500F04E33851800A460F03E3375138EC3E
:1012700033F089EC20F004E389EC20F001E3020C68
:101280000101386B280E01013825D96EDA6A060192
:10129000060EDA22DF506CE00101376733D0370EDB
:1012A0003825D96EDA6A060EDA226A0E336F130E0B
:1012B000346F33513825186F000E38BFFF0E3421BC
:1012C000196FE5EC2FF0DF6E280E01013825D96E7D
:1012D000DA6A060EDA22DF50336F346B33BF34071D
:1012E0006A0E356F130E366F35513825186F000EA4
:1012F00038BFFF0E3621196FE5EC2FF0331934118A
:10130000BEE131D0370E01013825D96EDA6A060EFA
:10131000DA22790E336F130E346F33513825186F7C
:10132000000E38BFFF0E3421196FE5EC2FF0DF6E91
:10133000280E01013825D96EDA6A060EDA22DF504E
:10134000336F346B33BF3407790E356F130E366F3E
:1013500035513825186F000E38BFFF0E3621196F32
:10136000E5EC2FF0CBD7382B3851800A710F8AE388
:10137000010C840EF66EEB0EF76E000EF86E21EE89
:101380002CF0060E0900F5CFDEFFE82EFBD7070E86
:10139000366F36C128F1F90E28272C0E2825D96E74
:1013A000DA6A010EDA22DF50296F73D8291902E0B8
:1013B000D8901200362B0B0E3665EBD7030E242582
:1013C000286F000E2521296F28C11BF129C11CF1AE
:1013D000ABEC1CF01BC134F11CC135F1326B336B2B
:1013E000070E366F0DD032C115F133C116F151D849
:1013F000176FAFEC40F015C132F116C133F1362B47
:10140000070E3425286F000E3521296F36C12AF1C9
:101410002B6B28512A5D29512B59E5E320EE02F070
:101420002451D9262551DA22DF50286F296B28BF95
:10143000290720EE01F02451D9262551DA22DF5068
:101440002B6F2A6B28512A11346F29512B11356FBC
:101450003551331902E134513219AAE10C0E242519
:10146000286F000E2521296F28C11BF129C11CF10D
:1014700049EC19F01BC134F11CC135F135510301A0
:10148000B51904E1010134510301B41991E1D88087
:10149000120036512425D96E000E2521DA6EDF5058
:1014A0001200E8CF3EF13F6B406B05010E512B0A55
:1014B00015E1010E0101406F11D00E0E0101402512
:1014C000D96EDA6A050EDA22280E3F25E16EE26A4D
:1014D000010EE222DFCFE7FF402B3F2B05011E511B
:1014E0000101405DEAE3280E3F25D96EDA6A010E5C
:1014F000DA22DF6A166F280E156F24EC38F01551CA
:101500003F6F3FC11DF11E6B206B020E1F6F79EC08
:101510003CF01DC13AF11EC13BF11FC13CF120C19D
:101520003DF13B51800A800F010ED8B43A5D0AE3C9
:10153000010E166F280E156FFB0E186FEC0E176F4D
:10154000BCEC3BF0406B2CD040C125F1252B280E84
:101550002525D96EDA6A010EDA221F0E266F050ED6
:10156000276F40512627000E27233E512625E16E86
:10157000000E2721E26EDFCFE7FF280E4025D96E4F
:10158000DA6A010EDA2218D82527000E262325292B
:10159000E16E000E2621E26EDFCFE7FF020E40274C
:1015A0003F51405DD1E308D82525D96E000E262194
:1015B000DA6E000EDF6E000C1F0E256F050E266F13
:1015C00040512527000E26233E51120064502FE182
:1015D00004010031E8320F0B0D0A0FE104BF046B68
:1015E0000401BF6B0401C06B0401C56BC46BC0EC8C
:1015F00027F0E1EC26F0AFEF25F00401C051020A1C
:1016000044E1070E0401CB6F040EC86F280EC76FAC
:10161000040ECA6FCE0EC96FDDEC3DF0010E040161
:10162000D56F040E0401036F200E026F1200645088
:10163000040AD8A412000401CD51080A0AE122C408
:101640005EFF040ECD6F0F015E5103E0100E04012A
:10165000CD6F0401C00519E1040E0401076F280EC7
:10166000066F2FEC23F00401BF51020A04E1840E3F
:101670000401046F840C040104BD03D0C80E046F80
:10168000C80C880E0401046F880C0401C16B0401AE
:10169000C051020AD8B465A81CD004010151080A3F
:1016A00018E10031E8320F0B0D0A13E100BF11D031
:1016B000040E036F200E026F040E0401C86F280E83
:1016C000C76F040ECA6F200EC96F080ECB6FF9EFFB
:1016D0003DF00401C06B080E0401016F040E036F9E
:1016E000200E026F8C0E006F046B1200A192F60E9A
:1016F0007B6E3C0E7A260101D86701D03C0C010EAE
:10170000D807D8A4010C00010FAE010C0FBA09D004
:1017100010A81088416A0F9C10960001109CF19C43
:10172000120010A86AD010AC02D0109C66D0412ADA
:1017300081A402D0D89001D0D8800301EF370301F3
:10174000F0370301F1370301F2370301F3370301E7
:10175000F4370301F5370301F6370301F7370301C7
:10176000F8374150070B03E10301EF5140260FAC5E
:1017700020D010A403D04150500A05E010B43DD051
:101780004150400A3AE1108C0301EF51405EEF51A5
:1017900040620CD009B20AD0030E216EEF0E206E0B
:1017A00066EC1DF0416A8F80138A27D01080416A51
:1017B00009D010A609D041502A0A03E041502B0A53
:1017C0001CE11082F18C19D04150080A16E1EFC3D8
:1017D00040F0108C0301EF51110A02E110861A84C7
:1017E00010A404D00301EF51EB0A06E010B405D0B9
:1017F0000301EF51A50A01E10F8C140E0101D86F0E
:1018000000010F9A140C2FC176F130C177F1510EFF
:101810007B6F7A6B31051CE1196B750E186FE5EC67
:101820002FF0786F7851080B756F755167E0510E86
:10183000196F750E186FE5EC2FF0786F7887510EE1
:10184000186F750E176F78C119F1D6EC36F056D0B7
:10185000196B750E186FE5EC2FF0E3D7C00E7625E7
:10186000326FFF0E7721336F3351800A800F010EE4
:10187000D8B4325D20E3796B47D8E5EC2FF0DF6E0A
:101880007A4B7B2B792B3F0E7965F6D72DC126F14C
:101890002EC127F1010E296F350E286F400E2A6FD9
:1018A00021EC3EF0400E2D27000E2E23C00E762791
:1018B000FF0E772323D0796B07D026D8E5EC2FF0E5
:1018C000DF6E7A4B7B2B792B79C132F1336B33513D
:1018D000800A346F7651325D7751800A3459EDE3D6
:1018E0002DC126F12EC127F1010E296F350E286F6B
:1018F00076C12AF121EC3EF0766B776B01017751CE
:101900007611D8B41200AAD7350E7925D96EDA6AC5
:10191000010EDA227AC118F17BC119F11200E8CF69
:1019200023F1C839E8461F0B156F166B62EC25F0E2
:1019300015C121F116C122F15BD862D8FDEC44F04B
:10194000DF6E232B55D864D8FDEC44F0DF6E232BDB
:101950004FD83A0EDF6E232BC939E842070BC8C1B6
:101960001FF1206BD8901F372037D8901F372037B2
:1019700057D862EC25F015C121F116C122F138D8F3
:101980003FD8FDEC44F0DF6E232B32D841D8FDEC7C
:1019900044F0DF6E232B2CD83A0EDF6E232BCA4582
:1019A000010BC9C11FF1206B3BD862EC25F015C1BA
:1019B00021F116C122F11CD823D8FDEC44F0DF6ED2
:1019C000232B16D825D8FDEC44F0DF6E232B1E51B7
:1019D00004E00ED8200EDF6E232B1F0E01012325FD
:1019E000D96EDA6A0501050EDA22000EDF6E000CF0
:1019F0001F0E01012325D96EDA6A050EDA221200C4
:101A000010EE03F02151E1262251E222E7501200AC
:101A100010EE04F02151E1262251E222E75012009B
:101A2000D8901F3720371F133F0E1F15156F166BE9
:101A3000000CE8CF5EF100010CBC02D0D89012007F
:101A400057C615F101015E5192EC41F0F7E3050133
:101A500025EED3F0020EDF64F1D725EED3F0050EAC
:101A6000DF6401D0EBD700010CACE8D7020E010116
:101A70005D6F0ED01F0E01015D255AD8500FDEE3B9
:101A80001F0E01015D2554D8460FD8E201015D2BE0
:101A90000501D35101015D5DEDE305011F0ED32565
:101AA000D96EDA6A050EDA22DF6A210E0101586F5B
:101AB000050E596F58C11BF159C11CF149EC19F0C1
:101AC0001BC15BF11CC15CF1000E5B5D010E5C593A
:101AD000B5E28A8E5BC1F2F45CC1F3F400011480BC
:101AE000B1EC0FF001015E39F00B5A6F080E4A6F2E
:101AF0005A518CECF2F04AC15BF14BC15CF106012A
:101B0000575129EC46F002E2D88012005E51C3EC36
:101B10003EF001015A6F5BC139F15CC13AF15EC11F
:101B20003BF15AC13CF1030E3D6FABEC35F0ECD705
:101B3000D96EDA6A0501050EDA22DF50800A12003A
:101B4000E8CF30F10101326BFD0E176F530E166FA7
:101B5000010EA3EC33F0880E0101296F130E2A6FDA
:101B6000000E2B6B2C6B2D6BFCEC9FF00101346F86
:101B70003451080A02E1010E326F3451360A17E07F
:101B80003451280A14E03451290A11E034510C0A66
:101B90000EE034512C0A0BE0880E296F130E2A6FC9
:101BA0002B6B2C6B010E2D6FFCEC9FF0DFD73451AB
:101BB0000C0A08E0320506E0130E2A6F880E296F22
:101BC000D8EC38F00101336BFD0E176F5B0E166F0A
:101BD000010EA3EC33F0880E0101296F130E2A6F5A
:101BE000000E2B6B2C6B2D6BFCEC9FF00101316F09
:101BF000130E2A6F880E296FD8EC38F0010131518D
:101C0000380A0EE0B3EC46F07BEC46F0D10E010151
:101C1000295D070E2A59F8E3332B020E3365D4D71A
:101C20003351030A02E10C0E346FB3EC46F07BEC47
:101C300046F0B90E0101295D0B0E2A59F8E31894FC
:101C40003051310A01E118840101345112000001C0
:101C50000D9CB3EC46F059D04DEC07F00301EB6F4F
:101C600000010DAC52D00A010051300A01E1010C13
:101C70000051310A03E00051320A47E1010E01012F
:101C80004F6F4E6B0AD060D83A0EDF6204D04F0718
:101C90004FC14EF105D001014F2B56D8DF50F3E173
:101CA00001014E6701D0020C4F6B13D0BB0E010136
:101CB0004F25D96EDA6A070EDA22DF504C6F010E1B
:101CC0004F25D96EDA6A0A0EDA22DF504C1904E188
:101CD0004F2B4E514F5DEAE34F514E19E4E14F6BEC
:101CE00006D023D81F0E01014F2518D84F2B1DD821
:101CF000DF50F7E14FC1D3F50A010051310A01E18C
:101D0000030C0051320A01E1040C7BEC46F0E90EB1
:101D10000101295DFD0E2A599FE3000CE16EE26A84
:101D2000050EE222DFCFE7FF1200020E4C6F0A0E13
:101D30004D6F4E514C27000E4D234F514C25D96EFF
:101D4000000E4D21DA6E1200000E01014F25D96EF2
:101D5000DA6A0A0EDA221200E8CF64F1000114B246
:101D600002D0D890120005C515F10101645192EC22
:101D700041F0F7E30501D351070AF3E11F0ED32524
:101D8000D96EDA6A050EDA22DF6A220E01015F6F70
:101D9000050E606F5FC11BF160C11CF1ABEC1CF064
:101DA0001BC161F11CC162F161C11FF162C120F16F
:101DB00028EC40F0D6E3000115A835D0068A199624
:101DC00005012051300A02E1198601D007880990E7
:101DD0000201CA6B08BE8A9C468405012051300A64
:101DE00010E1020E0101166FFE0E156F32EC1BF0B2
:101DF0000101186B540E176F3F0E196FD6EC36F0B9
:101E00000FD0020E0101166FCC0E156F32EC1BF0D5
:101E10000101186B540E176F1F0E196FD6EC36F0B8
:101E20000001469410D0B1EC0FF001016439F00BC1
:101E3000636F480E4A6F63518CECF2F00501055157
:101E400029EC46F002E2D88012006451C3EC3EF067
:101E50000101636F63C158F1645124ECE8F0F3D7DA
:101E6000E8CF5EF100010CBA02D0D890120054C63F
:101E700015F101015E5192EC41F0F7E300010CAA6B
:101E8000F4D7050125EED3F0020EDF64EED725EE80
:101E9000D3F0050EDF6401D0E8D7020E01015D6FBB
:101EA00010D01F0E01015D2598EC0DF0500FDDE301
:101EB0001F0E01015D2598EC0DF0460FD6E20101E1
:101EC0005D2B0501D35101015D5DEBE305011F0EA3
:101ED000D325D96EDA6A050EDA22DF6A210E0101F6
:101EE000586F050E596F58C11BF159C11CF149ECCF
:101EF00019F01BC15BF11CC15CF1000E5B5D010EB2
:101F00005C59B3E28A8C5BC1D8F45CC1D9F400019E
:101F10000686B1EC0FF001015E39F00B5A6F050E29
:101F20004A6F5A518CECF2F04AC15BF14BC15CF143
:101F30000601545129EC46F002E2D88012005E51AD
:101F4000C3EC3EF001015A6F5BC139F15CC13AF15B
:101F50005EC13BF15AC13CF1030E3D6FABEC35F075
:101F6000ECD7B80EF66EEA0EF76E000EF86E21EEA4
:101F700030F0120E0900F5CFDEFFE82EFBD7030E7E
:101F80000101436F39D0FC0E176FEB0E166F010E77
:101F9000A3EC33F0D00E0101296F070E2A6F000E5B
:101FA0002B6B2C6B2D6BFCEC9FF00101426F4251AF
:101FB000270A22E1070E436F8F0E01014325D96ED8
:101FC000DA6A060EDA22210E4325E16EE26A060E77
:101FD000E222DFCFE7FF432B4351800A680FECE397
:101FE000210E4325D96EDA6A060EDA22DF6AD00E98
:101FF00026D8FCEC9FF004D0430701014329C3E13C
:10200000010143671200426B0BD021D8280E010159
:102010004225E16EE26A060EE222DFCFE7FF422BA5
:1020200016D8DF50F2E1422B280E01014225D96E6D
:10203000DA6A0601060EDA22000EDF6E000C296F46
:10204000070E2A6F2B6B2C6B010E2D6F010C300EBF
:102050004225D96EDA6A010EDA2212000401220545
:102060000EE120511F0B0BE10401C48F0401C66B6C
:1020700004012151030A03E1010E0401C66F0401AA
:102080002267120020511F0B020AD8A4120024510B
:102090000F0BD8B412000401C48FABEC43F0C7C4DB
:1020A000F6FFC8C4F7FF000EF86E0F0EF76404D0F9
:1020B000840EF56E0C0006D0F6CFE9FFF7CFEAFFED
:1020C000840EEF6E04012151030AD8B4120024518A
:1020D0000F0B0101006F4C0E016F0F0E026F0051CC
:1020E0000127E86A00BFE868022301C1D9FF02C1E5
:1020F000DAFFFE0EDE16000EDD16C7C4F6FFC8C4FA
:10210000F7FF000EF86E0F0EF76404D0C80EF56EE0
:102110000C0006D0F6CFE9FFF7CFEAFFC80EEF6E4E
:10212000040124AF1200C7C4F6FF0401C8C4F7FFBE
:10213000000EF86E0F0EF76404D0400EF56E0C0022
:1021400006D0F6CFE9FFF7CFEAFF400EEF6E1200A0
:102150000301CE2BFC0E0101176FB30E166F010E9B
:10216000A3EC33F0880E0101296F130E2A6F000EC5
:102170002B6B2C6B2D6BFCEC9FF00101306F305101
:10218000160A03E03051170A11E118B407D017A856
:102190000BD0179812AE178A0E9206D018A004D052
:1021A000189012AC1882F8D7048027D03051180A42
:1021B00009E03051190A06E030511A0A03E03051A3
:1021C0001B0A0DE100010490B3EC46F07BEC46F0F5
:1021D000210E0101295D4E0E2A590FE2F7D7305129
:1021E0000C0A0BE0880E296F130E2A6F2B6B2C6BD9
:1021F000010E2D6FFCEC9FF0C0D7010130510C0A8D
:1022000006E0130E2A6F880E296FD8EC38F0010112
:1022100030511B0A0CE030511A0A09E03051190AFA
:1022200006E03051180A03E00301CE6B07D0020E1E
:102230000301CE6503D0CE6BD8901200D880120077
:102240002E0E0101166FE00E156F01D0040068D844
:10225000D8B41629FBE19B8CEA0E166F600E156F41
:1022600001D004005DD8D8B41629FBE1F26AF06A07
:102270009D6AA06ABB6AB66AC66AAC6AC26A060E82
:10228000C16EC088C16AF80EC26EC098896A8C6A35
:102290002F0E926E4F0E956E868E8A6A8D6A050E8F
:1022A000936E020E966EF19E8B6A8E6AD40E946EB9
:1022B000BC0E976E8B828F6A656A1C0E986ED56A0B
:1022C000810ECD6ED10ECF6E200ECE6E9E909F9061
:1022D0009D80810E796EF60E7B6E3C0E7A6EA19219
:1022E000A292A082C088020ECE6EC098D0B805D04F
:1022F000A80E0301BB6FC00E04D0020E0301BB6F1A
:10230000D00EBA6F0B9C750E0101166F300E156F53
:1023100001D0040005D8D8B41629D8B41200F9D7D2
:1023200001011507D8A0160715291200190E246EF1
:10233000280EC26EC28024062428FDE1C282320E1D
:10234000246E2406242802E0C2B2FBD7C4CF25F0B5
:10235000630E25600DD00301C76BC62B3B0EC6650F
:1023600007D0C66BC56704D00E8A010EC56F1980F1
:10237000EC0E0201D1251F6E206AFF0E202225C01F
:1023800021F0226A2250800A236E1F50215C2050C7
:10239000800A23580BE30301C66BC72B3B0EC765AE
:1023A00005D0C76B19B0FF00C56B1990C26A280E23
:1023B000256007D00301C12B020EC165020CFF008E
:1023C000020C0301C451255C11E3C26BC16BC32B2A
:1023D000770EC365770CC36B079C079AC56B199082
:1023E000000108A212000880089212002550020184
:1023F000D15DD8A012000301C36BC16BC22B3B0E91
:10240000C2653B0CC26B078C0882000107BA120040
:10241000078E078A12000001F9510A0A10E015BC64
:102420000ED0000E4424D96EDA6A0B0EDA22F9C0FF
:10243000DFFF442AA00E4464A00C446A120000018D
:10244000F9510A0A2FE115BC2DD00B01000E4424CE
:10245000D96EDA6A0B0EDA22DF6A446A0B0E206E3E
:10246000000E1F6EEE0E226EE90E216E246A110E12
:10247000236E2CEC29F020501F1014E10001158C64
:10248000110E2E6E0B0E2F6E2EC025F02FC026F0D3
:102490000FEC1AF0FF0E25240401DC6FFF0E26203E
:1024A000DD6F1200000115AC12000401DD51DC11DA
:1024B00004E0DC07D8A0DD0701D0159C0001F9512C
:1024C0000A0A0FE10201DC07000EDC25D96EDA6A88
:1024D0000A0EDA22000EDF6A0D8CDCC2E4F2DC6B3D
:1024E0001200F9510A0AD8B41200000E0201DC25CC
:1024F000D96EDA6A0A0EDA22F9C0DFFFDC2B12008D
:1025000004921EC546F105010E512B0A03E101019B
:1025100046070482050E0101376F1F0E366FFE0E4F
:10252000396F4C0E386F30EC3DF03651476F47C174
:1025300048F151D846390F0BFDEC44F0DF6E482BC3
:102540004AD846510F0BFDEC44F0DF6E482B04A235
:1025500009D01F0E39D8FF0E396FF10E386F30ECED
:102560003DF008D01F0E30D8FF0E396FF40E386FD3
:1025700030EC3DF03651476F47514827485151ECF8
:102580000AF01F0E446F050E456F44C115F145C199
:1025900016F124EC38F01551486F1F0E15D8FF0EB8
:1025A000396F980E386F30EC3DF03651476F475118
:1025B00048271F0E01014825D96EDA6A0501050E6C
:1025C000DA22000EDF6E000C01014825366F376BF2
:1025D000050E372312001F0E01014825D96EDA6A55
:1025E000050EDA2212004D0E0201006FA36B5ED8B9
:1025F000DF501BE1A3C237F10101372B5FD80D0E6D
:10260000DF6EA3C237F1020E372758D80A0EDF6EED
:10261000A3C237F1030E3727000E3725D96EDA6AC9
:102620000201020EDA22DF6A12D040D8A3C237F1CB
:102630000101372B000E3725E16EE26A0201020E1E
:10264000E222DFCFE7FFA32B9F0EA365D0D79F0E1B
:10265000A36505D00D0EA06F0A0EA16FA26B020E2E
:1026600001012C6F000E2B6F000E2E6B2D6B05ECF5
:1026700006F002E2D8901200199C00010D9CB3EC08
:1026800046F00BD000010DAC08D00A010051300A11
:1026900002E1D880120000010D9C7BEC46F0E90EAF
:1026A0000101295DFD0E2A59E5E2ECD71F0E02015A
:1026B000A325D96EDA6A050EDA221200000E37253C
:1026C000D96EDA6A020EDA221200E8CF30F1305108
:1026D000360A06E030512C0A03E030510C0A02E1C0
:1026E000D89012003051290A5EE1196B5C0E186F08
:1026F000E5EC2FF02D6F196B5B0E186FE5EC2FF0EA
:102700002F6F2D512E6FFC0E176FCB0E166F010E13
:10271000A3EC33F02EC115F12FC116F162EC25F0B8
:1027200015C131F116C132F120EE01F03151D92637
:102730003251DA22DF50FDEC44F05CEC44F0010150
:1027400020EE02F03151D9263251DA22DF50FDEC71
:1027500044F05CEC44F0010120EE03F03151D92645
:102760003251DA22DF50FDEC44F05CEC44F0010120
:1027700020EE04F03151D9263251DA22DF50FDEC3F
:1027800044F05CEC44F0F10E0101176F310E166F4E
:10279000000EA3EC33F0130E01012A6F880E296F8F
:1027A000D8EC38F09DE3D8801200040122050EE138
:1027B00020511F0B0BE10401C48F0401C66B0401FF
:1027C0002151030A03E1010E0401C66F04012267CF
:1027D000120020511F0B020AD8A4120024510F0B23
:1027E000D8B412000401C48F0FEC44F0ADEC29F012
:1027F000F76404D0840EF56E0C0006D0F6CFE9FF26
:10280000F7CFEAFF840EEF6E04012151030AD8B41A
:10281000120024510F0B0101156F4C0E166F0F0E95
:10282000176F15511627E86A15BFE868172316C1F8
:10283000D9FF17C1DAFFFE0EDE16000EDD16ADEC75
:1028400029F0F76404D0C80EF56E0C0006D0F6CF60
:10285000E9FFF7CFEAFFC80EEF6E040124AF1200C4
:10286000C7C4F6FF0401C8C4F7FF000EF86E0F0ED0
:10287000F76404D0400EF56E0C0006D0F6CFE9FFE9
:10288000F7CFEAFF400EEF6E1200E8CF19F186860F
:102890000001FA6B3A0E36EC44F03A0E6DEC46F05D
:1028A0000101176702D00F0E176F18051DE11751B0
:1028B000F00B0CE017390F0BFDEC44F01A6F1A51B6
:1028C00036EC44F001011A516DEC46F0010117514C
:1028D0000F0BFDEC44F01A6F1A5136EC44F0010175
:1028E0001A516DEC46F00DD017510F0BFDEC44F072
:1028F0000301BF6FBF5136EC44F00301BF516DECD3
:1029000046F00101195136EC44F0010119516DEC0A
:1029100046F00101165136EC44F0010116516DEC00
:1029200046F0FA390F0BFDEC44F036EC44F00001B0
:10293000FA510F0BFDEC44F036EC44F00D0E36EC82
:1029400044F00A0E36EC44F00301A86BA96B000EAC
:10295000A76F0A0EA66F00011D9CADB203D0000147
:102960001DACFBD786961200E8CF23F1DF07DF51BD
:10297000220DF90EF324296F3F0EF4202A6F29C18E
:1029800018F12AC119F1E5EC2FF0276F286BD890C8
:1029900027351F6F2835206F23511F252B6F000E01
:1029A00020212C6F2BC124F12B07D8A02C07D89005
:1029B00027351F6F2835206FDF51220D1F51F3245B
:1029C000216F2051F420226FF90E2125296F3F0E2F
:1029D00022212A6F2ED029C118F12AC119F1E5EC64
:1029E0002FF01F6FFF0E2925186FFF0E2A21196F78
:1029F000E5EC2FF0266F1F51256F1E0E01012B25D0
:102A0000D96EDA6A050EDA222651DF6E1F0E2B25EB
:102A1000D96EDA6A050EDA2225C1DFFF2707D8A0B2
:102A20002807FE0E2B27FF0E2C23020E295F000E17
:102A30002A5B2851800A800F010ED8B4275DCBE2B3
:102A4000245112000301F25194EC44F0166F03017B
:102A5000F15194EC44F0176F1739F00B1611030184
:102A6000EF6F05AE1DD0F45194EC44F0166F0301E6
:102A7000F35194EC44F0176F1739F00B1611030162
:102A8000F06FF65194EC44F0166F0301F55194EC9D
:102A900044F0176F1739F00B16110301F16F06D0D0
:102AA0000101D0510301F06FCFC1F1F3F85194EC63
:102AB00044F0166F0301F75194EC44F0176F173987
:102AC000F00B16110301F26FFA5194EC44F0166FFB
:102AD0000301F95194EC44F0176F1739F00B1611FC
:102AE0000301F36FFC5194EC44F0166F0301FB51AA
:102AF00094EC44F0176F1739F00B16110301F46FC3
:102B0000FE5194EC44F0166F0301FD5194EC44F037
:102B1000176F1739F00B16110301F56FF66B1200E2
:102B2000E8CF5EF16EC615F101015E5192EC41F005
:102B300002E2D89012000501D3510B0AFAE126C532
:102B40005AF1266B220E0101586F050E596F58C1BC
:102B50001BF159C11CF1ABEC1CF01BC15CF11CC199
:102B60005DF15CC11FF15DC120F128EC40F0E1E3B3
:102B70005AC126F505011F0ED325D96EDA6A050E56
:102B8000DA22DF6A260E0101586F050E596F58C10F
:102B90001BF159C11CF1ABEC1CF01BC15CF11CC159
:102BA0005DF15CC11EF15DC11FF123EC44F0010138
:102BB0005E39F00B5B6F300E4A6F5B518CECF2F0BC
:102BC0004AC15CF14BC15DF106016E5129EC46F042
:102BD00002E2D88012005E51C3EC3EF001015B6F4F
:102BE0005CC139F15DC13AF15EC13BF15BC13CF1C1
:102BF000030E3D6FABEC35F0ECD7E8CF5EF16EC65F
:102C000015F101015E5192EC41F002E2D890120000
:102C10000501D3510B0AFAE126C55AF1266B220EA3
:102C20000101586F050E596F58C11BF159C11CF1B4
:102C3000ABEC1CF01BC15CF11CC15DF15CC11FF170
:102C40005DC120F128EC40F0E1E35AC126F5050111
:102C50001F0ED325D96EDA6A050EDA22DF6A260E38
:102C60000101586F050E596F58C11BF159C11CF174
:102C7000ABEC1CF01BC15CF11CC15DF15CC11EF131
:102C80005DC11FF1CAEC44F001015E39F00B5B6FCE
:102C9000300E4A6F5B518CECF2F04AC15CF14BC1D3
:102CA0005DF106016E5129EC46F002E2D880120077
:102CB0005E51C3EC3EF001015B6F5CC139F15DC157
:102CC0003AF15EC13BF15BC13CF1030E3D6FABECF1
:102CD00035F0ECD70201B46BB56BB66BB76B010185
:102CE000086B2AD008510025D96E000E0121DA6E3A
:102CF000DF500201B427000EB523B45D010EB559B3
:102D000003E3B44BB52BB56BB429B51102E1B46B39
:102D1000B56BB451B627B551B723000EB65D010EA1
:102D2000B75903E3B64BB72BB76BB629B71102E11E
:102D3000B66BB76B0101082BFE0E0225036F046B07
:102D4000FF0E042308C105F1066B0651800A076FC8
:102D50000351055D0451800A0759C4E302511ED88E
:102D6000FE0E12D8B45D0101086F08670BD0025146
:102D700015D8FF0E09D8B65D0101086F086702D0AB
:102D8000D8801200D89012000325D96EFF0E0421BE
:102D9000DA6EDF50056F0551020112000025036F46
:102DA000E86A02BFE8680121046F120020EE01F01A
:102DB0001E51D9261F51DA22DF50206F20C121F188
:102DC000226B213B223BF00E221721510F0B2213C5
:102DD000F00E2117236B0F0E2215246F20EE02F048
:102DE0001E51D9261F51DA22DF502311256F24519D
:102DF000266F25C115F126C116F162EC25F015C12B
:102E000027F116C128F11EC1D9FF1FC1DAFF10EE4C
:102E100002F01E51E1261F51E222DFCFE7FF20EE34
:102E200004F02751D9262851DA22DF50206F20EEF6
:102E300003F02751D9262851DA22DF50216F21399A
:102E4000F00B20111EC1D9FF1FC1DAFFDF6E20EE8B
:102E500001F01E51D9261F51DA2210EE02F027513F
:102E6000E1262851E222E750206F10EE01F01E51BA
:102E7000E1261F51E222E750216F2139F00B20118A
:102E8000DF6E1200E8CFBEF1010E0101C06FBE512E
:102E900002E0030EC06F1B6B1C6B060E0101C02508
:102EA000D96EDA6A0501050EDA22DF5094EC44F09F
:102EB0001D6F050E0101C025D96EDA6A0501050EE8
:102EC000DA22DF5094EC44F01E6F000E42EC34F036
:102ED0001B51BF6FBE6702D0039003D0BE0501E156
:102EE00003920101BD6BBF5106ECF1F010E300014C
:102EF0001B9689ECE4F0C06FC051800A7A0F07E29C
:102F0000C05156ECC9F003E3010E0101BD6F010190
:102F1000BD671FD0FB0E176F8B0E166F010EA3EC53
:102F200033F0130E01012A6F880E296FD8EC38F0A8
:102F30000101BF5106ECF1F00CE300011B9689EC96
:102F4000E4F0C06FC051800A7A0F03E2C05156EC22
:102F5000C9F00101BF5184EF1FF004EE00F0D60E5E
:102F6000EE6AE806FDE10DEE00F0F00EEE6AE8060E
:102F7000FDE10CEE00F0960EEE6AE806FDE10BEEC8
:102F800000F0F00EEE6AE806FDE10AEE00F0F00E49
:102F9000EE6AE806FDE109EE00F0B40EEE6AE8061E
:102FA000FDE108EE00F0F20EEE6AE806FDE107EE44
:102FB00000F0F50EEE6AE806FDE106EE00F0FE0E0A
:102FC000EE6AE806FDE105EE00F0FA0EEE6AE806AC
:102FD000FDE103EEA6F05A0EEE6AE806FDE102EE10
:102FE000A6F05A0EEE6AE806FDE101EEC1F02A0EE7
:102FF000EE6AE806FDE100EEE9F0170EEE6AE8067B
:10300000FDE100EE01F01E0EEE6AE806FDE100EEC5
:103010003FF0070EEE6AE806FDE104EED6F02A0E58
:10302000EE6AE806FDE100011AEF8EF0F50E176F6B
:103030002F0E166F010EA3EC33F04DD0ABECEAF07F
:1030400002A449D002940201CE6701D044D0080EF8
:1030500001011C6FA00E1B6FFD0E1E6F630E1D6F16
:10306000206B070E1F6F0AEC28F01C511B1133E177
:10307000080E2E6F10D037D8DF620DD007D033D8AE
:10308000DF6204D02EC12DF1320E2E6F01012E51C0
:10309000800A4E0FF4E301012E51800A4E0FEBE33C
:1030A000A00E296F080E2A6F2D512927000E2A2302
:1030B00029C11BF12AC11CF149EC19F01BC12BF1EC
:1030C0001CC12CF12C51800A750FB80ED8B42B5DA1
:1030D00008E2D8901200310E0301B25D750EB359AB
:1030E000ADE3D88012002E2B2E05296FA00E010112
:1030F0002925D96EDA6A080EDA222C0CE8CF26F0E0
:1031000026500A0A57E10301DA6B0C010C0E206EFF
:10311000000E1F6EFD0E226E130E216E246A070E26
:10312000236E2CEC29F020501F1004E1020E000148
:10313000FC6F020C0C010C0E206E000E1F6EFD0EBB
:10314000226E700E216E246A020E236E2CEC29F082
:1031500020501F1004E1010E0001FC6F010C0C0156
:103160000C0E206E000E1F6EFF0E226E9D0E216E45
:10317000246A030E236E2CEC29F020501F1004E16A
:10318000030E0001FC6F030C0C010C0E206E000EF0
:103190001F6EFF0E226E250E216E246A040E236E12
:1031A0002CEC29F020501F10D8A41200040E0001AE
:1031B000FC6F040C000E0301DA25D96EDA6A0C0EDE
:1031C000DA2226C0DFFFDA2B12003251B0EC39F0E0
:1031D00015C137F116C138F137C1D9FF38C1DAFF4F
:1031E000DF50356F320502E1280E0AD03251020A53
:1031F000FBE03251030AF8E03251040AF5E0020E16
:10320000366F3651355D2AE3F00E176F260E166FB6
:10321000000EA3EC33F0880E0101296F130E2A6F04
:10322000000E2B6B2C6B2D6BFCEC9FF032C118F158
:10323000000EE5EC28F03251B0EC39F015C137F151
:1032400016C138F137C1D9FF38C1DAFFDF50356F09
:10325000500E206FE00E1F6FACEC38F037C1D9FF75
:1032600038C1DAFFDF2A0101325104EC39F015C10F
:1032700033F116C134F13551020DF3503325D96EB7
:10328000000E3421DA6E30C1DEFF31C1DDFFD8809F
:10329000120003D001011B4B1C2B1BC1D9FF1CC109
:1032A000DAFFDF50200AF6E01BC1D9FF1CC1DAFFAC
:1032B000DF50090AEFE00101226B236B216B2D0E19
:1032C0001BC1D9FF1CC1DAFFDF6202D0212B07D05E
:1032D0002B0E1BC1D9FF1CC1DAFFDF6222D01B4BB2
:1032E0001C2B1FD01BC1D9FF1CC1DAFFDF501D6F83
:1032F0001E6B1DBF1E0722C115F123C116F1186BED
:103300000A0E176F65EC42F01D5115251F6F1E51F7
:103310001621206FD00E1F25226FFF0E2021236F54
:10332000DED71BC1D9FF1CC1DAFFDF501FEC45F00F
:10333000D9E221510DE022C11DF123C11EF11D1F53
:103340001E1F1D4B1E2B1DC11BF11EC11CF11200A7
:1033500022C11BF123C11CF112001A51B0EC39F04B
:1033600015C11FF116C120F11FC1D9FF20C1DAFF1D
:10337000DF50256F256701D012001A5104EC39F097
:1033800015C121F116C122F1236B44D02351020D46
:10339000F3502125D96E000E2221DA6EDECF1BF10B
:1033A000DDCF1CF11B511D6F030E1C151E6F19196B
:1033B00002E118511D192DE11FC1D9FF20C1DAFF0B
:1033C000DF50DF06256F23C124F11ED0D8902435AD
:1033D0001B6F1B5121251C6FE86A1BBFE868222167
:1033E0001D6F020E1C25D96E000E1D21DA6E2451B0
:1033F000020DF3502125E16E000E2221E26EDECF98
:10340000E6FFDDCFE5FF242B2551245DD8B0120067
:10341000DDD7232B2551235DD8B01200B7D702D0BA
:10342000254A262A25C0D9FF26C0DAFFDF50200A08
:10343000F7E025C0D9FF26C0DAFFDF50090AF0E027
:103440002C6A2D6A2B6A2D0E25C0D9FF26C0DAFF03
:10345000DF6202D02B2A07D02B0E25C0D9FF26C051
:10346000DAFFDF6222D0254A262A1FD025C0D9FFE5
:1034700026C0DAFFDF50276E286A27BE28062CC038
:103480001FF02DC020F0226A0A0E216EE9EC42F0F6
:1034900027501F24296E285020202A6ED00E292460
:1034A0002C6EFF0E2A202D6EDED725C0D9FF26C038
:1034B000DAFFDF50ECEC44F0D9E22B500DE02CC0E9
:1034C00027F02DC028F0271E281E274A282A27C0AB
:1034D00025F028C026F012002CC025F02DC026F0C3
:1034E0001200DACF0EF1F3CF0FF1F4CF10F1F6CFD7
:1034F00011F1F7CF12F1F8CF13F1F5CF14F13BEC46
:1035000046F0F2A801D001D006D0F2A201D001D03D
:1035100002D06DEC43F0F0A801D001D00AD0F0A2A7
:1035200001D001D006D0F0AE01D001D002D017EC0E
:1035300046F0A3A601D001D00AD0A4A601D001D0A4
:1035400006D0A5A601D001D002D0DAECDDF0F2AAB7
:1035500001D001D012D0F2A401D001D00ED0F1A43C
:1035600001D001D00AD0000110AE01D001D003D0AB
:10357000C3EC3CF002D052EC38F014C1F5FF13C19B
:10358000F8FF12C1F7FF11C1F6FF10C1F4FF0FC120
:10359000F3FF0EC1DAFF0DC1D9FF0CC1EAFF0BC169
:1035A000E9FF1100E8CF24F1276B24072451330DE4
:1035B0008D0EF324286F130EF420296F28C118F103
:1035C00029C119F1E5EC2FF0256F266B284B292B2B
:1035D0002651800A800F020ED8B4255D07E32651DC
:1035E000800A800F180ED8B4255D20E31F6920697A
:1035F00012002829186F000E2921196FE5EC2FF011
:10360000216F28C118F129C119F1E5EC2FF0236FC2
:103610002151226F22513F0A2311D8B4272B2507AD
:10362000D8A02607020E2827000E29232651800A3B
:10363000800F010ED8B4255DDCE2020E276505D0AF
:10364000F00E206F000E1F6F000C2751020A04E1DC
:103650002069000E1F6F000C2705C8E12069F00EDD
:103660001F6FF00C000119B0120014BE128814A2D2
:103670001AD001011551220A161110E01551260A1F
:1036800016110CE015512A0A161108E015512E0AE0
:10369000161104E01551360A161105E1098008BE1D
:1036A0008A8CD2C2CAF2130E0101DA652BD0DA0776
:1036B0001C6B17D0D8901C35176F020E010117250F
:1036C000D96EDA6A060EDA221C51020D000EF324BE
:1036D000E16EE26A060EE222DECFE6FFDDCFE5FF15
:1036E0001C2BDAC117F1186B1CC119F11A6B19BF29
:1036F0001A071A51800A1B6F1751195D1851800A59
:103700001B59D8E3DA51020D000EF324D96EDA6AA0
:10371000060EDA22010115C1DEFF16C1DDFFDA2B2C
:103720001200000119B0120014BE128814A219D0A0
:103730001F50220A201010E01F50260A20100CE013
:103740001F502A0A201008E01F502E0A201004E003
:103750001F50360A201005E1098008BE8A8CD2C2AB
:10376000CAF2130E0101DA652BD0DA07266A16D0E9
:10377000D8902634216E020E2124D96EDA6A060E04
:10378000DA222650020D000EF324E16EE26A060EE4
:10379000E222DECFE6FFDDCFE5FF262A0101DAC116
:1037A00021F0226A26C023F0246A23BE2406245076
:1037B000800A256E2150235C2250800A2558D8E3C8
:1037C000DA51020D000EF324D96EDA6A060EDA22FF
:1037D0001FC0DEFF20C0DDFF0101DA2B12001E6BCF
:1037E0001CAF0AD01C1F1B1F1A1F196D000E1A23B5
:1037F0001B231C23010E1E6F18AF0AD0181F171FA2
:10380000161F156D000E162317231823010E1E1BFD
:103810001F6B206B216B226B1C5119111A111B118C
:1038200029E0010E1D6F06D0D89019371A371B37C3
:103830001C371D2B1CAFF8D7D8901F3720372137E6
:1038400022371951155D1A5116591B5117591C5120
:10385000185909E31951155F1A51165B1B51175B73
:103860001C51185B1F81D8901C331B331A3319333A
:103870001D2FE2D71E5108E0221F211F201F1F6DA0
:10388000000E2023212322231FC115F120C116F190
:1038900021C117F122C118F11200E8CF27F1000170
:1038A00014B202D0D890120005C515F101012751BC
:1038B00092EC41F0F7E30501D351070AF3E11F0E43
:1038C000D325D96EDA6A050EDA22DF6A220E0101EB
:1038D000256F050E266F25C11BF126C11CF1ABEC2F
:1038E0001CF01BC128F11CC129F128C11FF129C1FD
:1038F00020F128EC40F0D6E30A9C0A9A0B94099038
:103900000201CA6B08BE8A9C069A468419A610D08A
:10391000020E0101166FDD0E156F32EC1BF0010176
:10392000186B540E176F2F0E196FD6EC36F00FD0A0
:10393000020E0101166FDD0E156F32EC1BF0010156
:10394000186B540E176F0F0E196FD6EC36F000017E
:103950004694D88012001F6B206B216B02D01B4B4A
:103960001C2B1BC1D9FF1CC1DAFFDF50D3EC43F085
:10397000F6E22D0E1BC1D9FF1CC1DAFFDF6202D0B7
:103980001F2B07D02B0E1BC1D9FF1CC1DAFFDF6232
:103990001FD01B4B1C2B1CD0225130EC45F004E3F4
:1039A0002251A4EC45F0226F22511FEC45F0D00EBD
:1039B000D8A0A90E2227203B213BF00E2117205131
:1039C0000F0B2113F00E201722512027000E212368
:1039D0001BC1D9FF1CC1DAFF1B4B1C2BDF50226F10
:1039E00001012251B6EC3FF0D7E21F510DE020C19A
:1039F0001DF121C11EF11D1F1E1F1D4B1E2B1DC1C0
:103A00001BF11EC11CF1120020C11BF121C11CF1D0
:103A10001200F80E0101176FCC0E166F010EA3EC09
:103A200033F02C0E5CEC44F0070170510FE0220ED5
:103A30005CEC44F0070E0101176F700E166F000E5C
:103A4000A3EC33F0220E5CEC44F006D0220E5CECCA
:103A500044F0220E5CEC44F02C0E5CEC44F0220EA0
:103A60005CEC44F00601DF5108E0060E0101176F1F
:103A7000DF0E166F000EA3EC33F0220E5CEC44F068
:103A80002C0E5CEC44F0220E5CEC44F00601E85194
:103A900008E0060E0101176FE80E166F000EA3EC8A
:103AA00033F0220E5CEC44F0EE0E0101176F060EAF
:103AB000166F000EA3EC33F00D0E5CEC44F0130E09
:103AC00001012A6F880E296FD8EF38F0000110B479
:103AD00008D020EE03F02050D9262150DA22030E20
:103AE000DF1649D803E13FD8D8B41200020EDAEC51
:103AF00041F0000110A40AD020EE08F02050D92691
:103B00002150DA22DF50DAEC41F024D020EE05F02B
:103B10002050D9262150DA22DF3A20EE05F020503D
:103B2000D9262150DA2210EE05F02050E12621504E
:103B3000E222E750226ED8902232D8902230030B36
:103B4000DF6E20EE05F02050D9262150DA22DF501A
:103B5000DAEC41F010D8DAEC41F005D8DAEC41F0BB
:103B600000010E84120020EE02F02050D9262150D0
:103B7000DA22DF50120020EE03F02050D926215027
:103B8000DA22DF5012000301BF5194EC44F01F6FA2
:103B90007F0E01014CD81E6F1EAF12007F0E1F2535
:103BA000D96EDA6A060EDA22DF2A7F0E40D81E6F3F
:103BB0003F0E1E17030E1E5D02E38F8013887F0EDB
:103BC000010135D83F0B050A09E1530E0301F26FDD
:103BD000300EF36F01011F5157EC3AF07F0E0101D7
:103BE0001F25D96EDA6A0601060EDA22DF503F0B76
:103BF0003F0AD8A41200530E0301F26F200EF36F98
:103C000001011F5157EC3AF07F0E01011F25D96EBB
:103C1000DA6A060EDA22DF6A960E1F25176F186B16
:103C2000020E18237F0E03D8196FD6EF36F01F252A
:103C3000D96EDA6A060EDA22DF501200EF0E0101A9
:103C4000176F9D0E166F010EA3EC33F0070E0101E6
:103C5000176F700E166F000EA3EC33F0220E5CECA3
:103C600044F00D0E5CEC44F0130E01012A6F880E37
:103C7000296FD8EC38F0ED0E0101176F3B0E166F6F
:103C8000010EA3EC33F0130E01012A6F880E296F89
:103C9000D8EC38F0ED0E0101176F530E166F010EC0
:103CA000A3EC33F0130E01012A6F880E296FD8ECB4
:103CB00038F0EE0E0101176F480E166F010EA3ECDF
:103CC00033F0130E01012A6F880E296FD8EC38F0FB
:103CD000EE0E0101176F330E166F010EA3EC33F0D9
:103CE000130E01012A6F880E296FD8EC38F009EF06
:103CF0001DF020EE01F01E51D9261F51DA22DF50AF
:103D0000156F166B62EC25F015C124F116C125F173
:103D100020EE04F02451D9262551DA22DF50206FFD
:103D200020EE03F02451D9262551DA22DF50216FED
:103D30002139F00B2011226F20EE02F01E51D926FE
:103D40001F51DA22DF5099EC3DF0236F20EE02F094
:103D50001E51D9261F51DA2223C120F1203B0F0E1C
:103D600020171EC1E1FF1FC1E2FFE750F00B201139
:103D7000DF6E20EE01F01E51D9261F51DA2210EE1F
:103D800002F02451E1262551E222E750206F233929
:103D9000F00B2011DF6E1EC1D9FF1FC1DAFF22C157
:103DA000DFFF12003D6B50D83D512225186F000EE9
:103DB0002321196FE5EC2FF0DF6E46D8DF5004E0C9
:103DC0003D2B100E3D65EFD72A5107E02351020A23
:103DD000410ED8B4221901E01B8601013B6B2A5128
:103DE0002B0A03E1010E3B6F3D07DC5109E0DC517A
:103DF0003D5D3C6F3C51800A7F0F02E33C513B2705
:103E00002A0E266F010E276F3B512627000E27230F
:103E100026C11BF127C11CF10E0E286F050E296F5C
:103E200024512827000E292328C11DF129C11EF184
:103E300025C11FF1206B0AEC28F01C511B1102E177
:103E4000D8801200D89012002A0E3D25D96EDA6A69
:103E5000010EDA221200E8CF5DF102C515F1010171
:103E60005D5192EC41F002E2D89012000501D3516D
:103E7000070AFAE11F0ED325D96EDA6A050EDA2297
:103E8000DF6A220E0101586F050E596F58C11BF1F0
:103E900059C11CF1ABEC1CF01BC15AF11CC15BF108
:103EA0005AC11FF15BC120F128EC40F0DDE30001B5
:103EB0001EB602D000010E8CB1EC0FF001015D398D
:103EC000F00B5C6F800E4A6F5C518CECF2F04AC1D3
:103ED0005AF14BC15BF10501025129EC46F002E2B7
:103EE000D88012005D51C3EC3EF001015C6F5AC1F5
:103EF00039F15BC13AF15DC13BF15CC13CF1030EAC
:103F00003D6FABEC35F0ECD7E8CF2BF1FE0E176F21
:103F1000710E166F010EA3EC33F03D0E5CEC44F015
:103F200001012BC115F1166B62EC25F015C12DF1C5
:103F300016C12EF120EE03F02D51D9262E51DA2292
:103F4000DF50FDEC44F05CEC44F0010120EE04F0A5
:103F50002D51D9262E51DA22DF50FDEC44F05CECD5
:103F600044F00D0E5CEC44F0B3EC46F001012C6B18
:103F700019D089EC46F016E3AFEC46F001012F6F43
:103F80000DD02F517BEC42F00DE301012C2B0AD018
:103F90002F51BDEC42F0D8B0120004D02C51F1E00A
:103FA000010AF6E07BEC46F0D10E0101295D070E17
:103FB0002A59D8B01200DDD720EE01F01E51D926C3
:103FC0001F51DA22DF50156F166B62EC25F015C118
:103FD00024F116C125F120EE04F02451D9262551F3
:103FE000DA22DF50206F20EE03F02451D92625512C
:103FF000DA22DF50216F2139F00B2011226F20EEE1
:1040000002F01E51D9261F51DA22DF50236F20EE15
:1040100002F01E51D9261F51DA2223C120F1203B84
:104020000F0E20171EC1E1FF1FC1E2FFE750F00B8A
:104030002011DF6E20EE01F01E51D9261F51DA2229
:1040400010EE02F02451E1262551E222E750206FC4
:104050002339F00B2011DF6E1EC1D9FF1FC1DAFF1B
:1040600022C1DFFF1200E8CF5DF103C515F10101A8
:104070005D5192EC41F002E2D89012000501D3515B
:10408000070AFAE11F0ED325D96EDA6A050EDA2285
:10409000DF6A220E0101586F050E596F58C11BF1DE
:1040A00059C11CF1ABEC1CF01BC15AF11CC15BF1F6
:1040B0005AC11FF15BC120F128EC40F0DDE30001A3
:1040C0000E8AB1EC0FF001015D39F00B5C6F840ECC
:1040D0004A6F5C518CECF2F04AC15AF14BC15BF172
:1040E0000501035129EC46F002E2D88012005D512F
:1040F000C3EC3EF001015C6F5AC139F15BC13AF18A
:104100005DC13BF15CC13CF1030E3D6FABEC35F0A2
:10411000ECD7FD0E0101176F810E166F010EA3EC97
:1041200033F0880E0101296F130E2A6F000E2B6BDE
:104130002C6B2D6BFCEC9FF00101306F06018F5151
:10414000800A500F04E38F51800A460F12E30101E9
:1041500030510C0A0EE03051090A0BE0880E296F2D
:10416000130E2A6F2B6B2C6B010E2D6FFCEC9FF046
:10417000E3D7010130510C0A03E13051090A1DE077
:10418000306B8F0E01013025D96EDA6A060EDA2205
:10419000280E3025E16EE26A060EE222DFCFE7FF4D
:1041A000302B3051800A710FECE3130E2A6F880E0A
:1041B000296FD8EC38F0D8901200D8801200E8CFE0
:1041C0005DF15EC615F101015D5192EC41F002E234
:1041D000D89012000501D351070AFAE11F0ED3252A
:1041E000D96EDA6A050EDA22DF6A220E0101586FF3
:1041F000050E596F58C11BF159C11CF1ABEC1CF0F5
:104200001BC15AF11CC15BF15AC11FF15BC120F106
:1042100028EC40F0DDE398EC37F0B1EC0FF0010151
:104220005D39F00B5C6F150E4A6F5C518CECF2F04F
:104230004AC15AF14BC15BF106015E5129EC46F0CF
:1042400002E2D88012005D51C3EC3EF001015C6FC8
:104250005AC139F15BC13AF15DC13BF15CC13CF13E
:10426000030E3D6FABEC35F0ECD717C1D9FF18C189
:10427000DAFFDF50D95FD951D8B4120020EE01F037
:104280001751D9261851DA22000EDF6E32D017C12D
:10429000D9FF18C1DAFFDF5034D81AC1D9FF1BC1CA
:1042A000DAFF10EE02F01751E1261851E222DFCFBB
:1042B000E7FF20EE02F01751D9261851DA2210EE4E
:1042C00001F01751E1261851E222E7501AD81AC11D
:1042D000E1FF1BC1E2FFDFCFE7FF20EE01F0175146
:1042E000D9261851DA22DF2A17C1D9FF18C1DAFFFF
:1042F000DF2A17C1D9FF18C1DAFF3F0EDF64C7D725
:104300003F0C196F195115251A6FE86A19BFE86833
:1043100016211B6F1200E8CF5BF11BB609D001011B
:104320005B5103E05B51050A03E1010E5B6F128AEA
:1043300051C615F101015B5192EC41F002E2D890B7
:104340001200000112AA0CD0129A01012B6B010E6F
:104350002C6F050E6CECD5F0F2E3050E01015B6FDE
:10436000B1EC0FF0FB0E0101376F790E366F5BC1B8
:1043700038F1396B4AEC41F05B39F00B5A6F8D0E16
:104380004A6F5A518CECF2F04AC158F14BC159F1C5
:104390000601515129EC46F002E2D88012005B512F
:1043A000C3EC3EF001015A6F58C139F159C13AF1DD
:1043B0005BC13BF15AC13CF1030E3D6FABEC35F0F4
:1043C000ECD72FC174F130C175F139D0C00E74250E
:1043D000316FFF0E7521326F3251800A800F010E4E
:1043E000D8B4315D14E3766B2FD87651800A400F34
:1043F000FBE333D8400E2A6F21EC3EF0400E2D2710
:10440000000E2E23C00E7427FF0E752318D0766B76
:1044100001D01AD876C131F1326B31BF3207325137
:10442000800A336F7451315D7551800A3359F1E35D
:1044300014D874C12AF121EC3EF0746B756B755180
:104440007411D8B41200C2D7340E7625D96EDA6A48
:10445000010EDA22DF68762B12002DC126F12EC163
:1044600027F1010E296F340E286F12000101186B1D
:10447000196B0BD047D8240EDF6203D00101192B32
:1044800004D040D8DF50181BF9D73CD8DF50F2E1F8
:104490001F0E1925D96EDA6A050EDA222A0EDF6E92
:1044A00019C116F1176B16BF1707200E1625D96E06
:1044B000050E1721DA6E18390F0B18BFF009FDEC45
:1044C00044F0DF6E19C116F1176B16BF1707210EE6
:1044D00001011625D96E050E1721DA6E18510F0B42
:1044E000FDEC44F0DF6E19C116F1176B16BF17070C
:1044F000220E01011625D96E050E1721DA6E000E67
:10450000DF6E000C1F0E01011925D96EDA6A050E47
:10451000DA2212000A0E236FA00E226F256B48D0FC
:104520002307D36B41EC43F001012251E2EC3EF052
:104530000101D3672FD01851E2EC3EF00101175171
:10454000E2EC3EF00101246B1DD024511925D96EF7
:10455000000E1A21DA6EDF50E2EC3EF00101252B4D
:10456000C00E1715206F1851216F174B182BC00E56
:1045700017151C6F18511D6F211902E120511C19CC
:1045800004E1242B1B51245DE0E395EC40F0010194
:1045900025511200070E1F6FD00E1E6F01D000F0C4
:1045A00001011E07D8A01F071E29D8B41F29F7E153
:1045B0002351800A7F0FEBE3B3D70101706BD03931
:1045C0000F0B506F516B50510F0BFDEC44F06B6FA4
:1045D0003ED8D0510F0BFDEC44F0DF6E38D8CF3908
:1045E0000F0BFDEC44F0DF6E32D8CF510F0BFDEC1A
:1045F00044F0DF6E2CD8DF6A010E376F520E366F33
:10460000FC0E396F900E386F070E01013B6FBB0E29
:104610003A6F010E3D6F6B0E3C6F30EC3DF0365142
:10462000706F520E7025D96EDA6A010EDA22DF6AD7
:104630002C6F520E2B6F000E2E6B2D6B05EC06F0BF
:1046400001E2000C000109B4010C27EF0EF0702B01
:104650006B0E7025D96EDA6A010EDA221200080E8E
:104660000401CB6F0401C5610CD0C5C4CBF40401B7
:10467000BF0502E1020EBF6F0401BF6702D0010E49
:10468000BF6F040104930491CBC405F40401CB5122
:104690000401C55DC56F040E0401CA6F280EC96F01
:1046A0000401C4A11DD022D0C2C4F6FFC3C4F7FFC9
:1046B000000EF86EC9C4D9FFCAC4DAFF0F0EF76442
:1046C00003D00800F55005D0F6CFE9FFF7CFEAFF99
:1046D000EF50DF6E0401C24BC32B0401C94BCA2B40
:1046E0000401CB07CB29D8B41200DED7C2C4C7F46B
:1046F000C3C4C8F4DDEC3DF0C7C4C2F4C8C4C3F4FD
:104700001200080E0401CB6F0401C5610CD0C5C4B2
:10471000CBF40401BF0502E1020EBF6F0401BF67C5
:1047200002D0010EBF6F040104930491CBC405F4C1
:104730000401CB510401C55DC56F040E0401CA6FAD
:10474000280EC96F0401C4A11DD022D0C2C4F6FF37
:10475000C3C4F7FF000EF86EC9C4D9FFCAC4DAFF9C
:104760000F0EF76403D00800F55005D0F6CFE9FF2F
:10477000F7CFEAFFEF50DF6E0401C24BC32B0401F9
:10478000C94BCA2B0401CB07CB29D8B41200DED702
:10479000C2C4C7F4C3C4C8F477EC3DF0C7C4C2F4C4
:1047A000C8C4C3F412000101E6511F0B02E01598C2
:1047B00001D015880201C92BC9513E0A06E1C96B17
:1047C00000014684B6ECEEF046940101D70507E1FE
:1047D0000201EF6702D00EEF45F0EF071200D7514C
:1047E000020A0EE10201EF67F8D7EE2BEE51080A3C
:1047F000F2E1EE6B199A8B9C960E0201EF6F960C0C
:1048000000010BB4120006AA0BD00201EF67E5D736
:10481000EE2BEE51060ADFE1EE6B199A8B8CECD78A
:1048200015A804D000010C968B8C12000CA608D0A1
:104830000201DF5105E0EF67D0D7DF070EEF45F04B
:1048400000010C968B9C1200E8CF63F1000105BAC1
:1048500002D0D890120061C615F10101635192ECAB
:1048600041F0F7E3040E0501D36101D0F2D725EE44
:10487000D3F0050EDF6401D0ECD7B1EC0FF00101ED
:104880006339F00B5A6F180E4A6F5A518CECF2F0E4
:10489000080E01015B6F0501D351040A09E12051A3
:1048A00094EC44F05C6F21C55DF122C55EF111D03E
:1048B000215194EC44F0586F0501205194EC44F0E0
:1048C000596F5939F00B58115C6F22C55DF123C542
:1048D0005EF15F6B606B616B626B010E176F5B0E5D
:1048E000166F91EC42F0D8801200050E356F03016F
:1048F000B151B01105E1E8EC3CF03FE3D880120083
:10490000B0C333F1B1C334F1010131513327325116
:1049100034233451800A7D0FE90ED8B4335D2DE382
:104920000301B06BB16BB6EC2EF023E3E7D716ECC6
:1049300018F014E2E8EC3CF0E1E22FC116F130C1CE
:1049400017F1000EA3EC33F0010131510301B02740
:10495000010132510301B123D8901200B3EC46F0AB
:104960007BEC46F0890E0101295D130E2A59F8E30C
:10497000350701013567DBD7C1D72FC116F130C12B
:1049800017F1000EA3EC33F0DFD71B6B000E44ECE5
:1049900040F01C6F19C115F11AC116F11CC117F1B5
:1049A000F6EC29F002E301011B81040E44EC40F017
:1049B0001C6F19C115F11AC116F11CC117F1B5EC24
:1049C00029F002E301011B83080E44EC40F01C6F48
:1049D00019C115F11AC116F11CC117F137EC2AF0F3
:1049E00002E301011B850C0E44EC40F01C6F19C161
:1049F00015F11AC116F11CC117F1B9EC2AF002E346
:104A000001011B87100E44EC40F01C6F19C115F119
:104A10001AC116F11CC117F178EC2AF002E301016A
:104A20001B8901011B511200000109B21200010E85
:104A300020C0D9FF21C0DAFFDF6204D0060EDAEC15
:104A400041F003D0070EDAEC41F020EE02F033D84B
:104A500020EE01F0205024D8DAEC41F020EE05F0F1
:104A60002AD8223A0F0E2216221620EE03F02050EA
:104A700017D8DAEC41F020EE05F01DD82238F00B03
:104A8000246E2450DAEC41F020EE04F02050D926B8
:104A90002150DA22DF50DAEC41F000010E841200DE
:104AA000D9262150DA22DF50236E2338F00B221052
:104AB000246E245012002050D9262150DA22DF50D3
:104AC000226E12000101010E186F190E176F196B7B
:104AD0001A6B1B6B1C6B1D6B100E155D270E165988
:104AE0000AE3192B100E155F270E165B100E155DCD
:104AF000270E1659F6E2E80E155D030E16590AE365
:104B00001A2BE80E155F030E165BE80E155D030EFB
:104B10001659F6E2640E155D000E16590AE31B2BBA
:104B2000640E155F000E165B640E155D000E1659BF
:104B3000F6E20A0E155D000E16590AE31C2B0A0E4A
:104B4000155F000E165B0A0E155D000E1659F6E293
:104B500015C11DF117C115F118C116F112006598A4
:104B6000080E0401016F0401C4BF1BD00401C15130
:104B70000EE0020E0401C06F0401056BC80E046F45
:104B8000040E036F280E026FC80E006FC80C040ECF
:104B90000401036F200E026F8C0E006F840E046FF1
:104BA000840C0401C151D8A41200040120AFE1D744
:104BB0000401C5510401265D000E2759D8A026C462
:104BC000C5F42FEC23F0010E0401C06F040E0401A4
:104BD000036F200E026F800E006F080E016F040E2F
:104BE000036F200E026F800E006F040E076F280EF9
:104BF000066FC80E046FC80CE8CF27F01C9827B2C8
:104C00001C8800010BA408D027A21200000119A8DB
:104C10001200000107881200000106AA120000011C
:104C20000ABC120000010AAA13D000F027A208D083
:104C3000206A260E1F6E91EC1BF000011C861200EC
:104C4000206A280E1F6E91EC1BF000011C961200CA
:104C500027A212000A8C19A604D00401D6C2DEF4E1
:104C600003D00401D5C2DEF4DF6BDE3BDF3BF00E88
:104C7000DF17DE510F0BDF13F00EDE17DF51DE11F1
:104C8000D8A412000A9C0A8A206A260E1F6E91EF91
:104C90001BF06598080E0401016F0401C4BF1BD00E
:104CA0000401C1510EE0020E0401C06F0401056B46
:104CB000C80E046F040E036F280E026FC80E006F3B
:104CC000C80C040E0401036F200E026F8C0E006FDF
:104CD000840E046F840C0401C151D8A41200040195
:104CE00020AFE1D70401C5510401265D000E27590C
:104CF000D8A026C4C5F481EC23F0010E0401C06FD6
:104D0000040E0401036F200E026F800E006F080E68
:104D1000016F040E036F200E026F800E006F040EF1
:104D2000076F280E066FC80E046FC80C04012051CF
:104D30001F0B0101156F1505D8A4120004012039BD
:104D4000E832030B0101156F1505D8A41200040108
:104D500024512AE02405D8A4120026D0040E040110
:104D6000C36FB50EC26F080EC56FC4810401C48F36
:104D70001200040E0401C36FB50EC26FF7D7010E07
:104D80000401C16F010C040E0401C36FCE0EC26F8B
:104D9000070EC56F810EC46F810C22C4CCF40401D0
:104DA000CC8F0401C48F120004012151D7E0010A05
:104DB000E0E0210AE4E0010AE6E0030AD8A41200D8
:104DC000ECD7040120511F0B0101006F0005D8A48E
:104DD000120004012039E832030B0101006F0005C5
:104DE000D8A41200040124512AE02405D8A41200FA
:104DF00026D0040E0401C36FB50EC26F080EC56F36
:104E0000C4810401C48F1200040E0401C36FB50EE7
:104E1000C26FF7D7010E0401C16F010C040E04012B
:104E2000C36FCE0EC26F070EC56F810EC46F810CAB
:104E300022C4CCF40401CC8F0401C48F12000401FD
:104E40002151D7E0010AE0E0210AE4E0010AE6E0AE
:104E5000030AD8A41200ECD704012039E832030B6E
:104E6000D8A412002ED00401C48F080E0401CD6F07
:104E7000080C08EF3CF0CCEF32F0040E0401C36FD5
:104E8000BD0EC26F0401C481010EC56FC48F010C39
:104E900072EF29F0D5EF13F0BE0E0101186F040E6A
:104EA000196F0401245101011827000E192318C19C
:104EB000C2F419C1C3F4E6D70401C48F22C4BEF4FE
:104EC000120004012151E4E0010AE4E0020AE2E0F8
:104ED000060AC9E0030ACDE00E0ACFE0010ACBE0E2
:104EE000030ADAE0010AD8A41200E6D73DD022C1B5
:104EF0001BF123C11CF124C11DF125C11EF124C1E8
:104F000015F125C116F124EC38F015C11FF116C1B9
:104F100020F10AEC28F01C511B1105E122C122F1FD
:104F200023C123F112002229156F000E2321166FD1
:104F300024C1F6FF25C1F7FF000EF86E0F0EF764CF
:104F400003D00800F55005D0F6CFE9FFF7CFEAFF10
:104F5000EF500101176F186B17BF180738EC42F0BC
:104F600015C122F116C123F12351221106E022C1FD
:104F7000D9FF23C1DAFFDF50BAE1226B236B1200A5
:104F800004012039E832030BD8A412002ED004010A
:104F9000C48F080E0401CD6F080C96EF3BF002EFB2
:104FA00033F0040E0401C36FBD0EC26F0401C4814F
:104FB000010EC56FC48F010CBDEF2BF02EEF10F06A
:104FC000BE0E0101036F040E046F040124510101A0
:104FD0000327000E042303C1C2F404C1C3F4E6D7BF
:104FE0000401C48F22C4BEF4120004012151E4E084
:104FF000010AE4E0020AE2E0060AC9E0030ACDE0A1
:105000000E0ACFE0010ACBE0030ADAE0010AD8A4D5
:105010001200E6D735D01BC1D9FF1CC1DAFFDF5023
:1050200013E039D8F76403D00800F55005D0F6CF67
:10503000E9FFF7CFEAFFEF500101216F1BC1D9FF54
:105040001CC1DAFFDF1818E01BC1D9FF1CC1DAFF51
:10505000DF50216F20D8F76403D00800F55005D049
:10506000F6CFE9FFF7CFEAFFEF500101215D1B6F9B
:105070001C6BD8A01C0712001B4B1C2B1D4B1E2B9E
:105080001F07D8A0200701011F29D8B42029C3E198
:105090001B6B1C6B12001DC1F6FF1EC1F7FF000E3B
:1050A000F86E0F0E1200256A000EC2EC41F0266E5B
:1050B00023C01FF024C020F026C021F0BFEC2CF04C
:1050C000D8B02580040EC2EC41F0266E23C01FF03C
:1050D00024C020F026C021F0BBEC2DF0D8B02582F2
:1050E000080EC2EC41F0266E23C01FF024C020F051
:1050F00026C021F0FAEC2DF0D8B025840C0EC2ECBD
:1051000041F0266E23C01FF024C020F026C021F0FD
:105110007CEC2DF0D8B02586100EC2EC41F0266E46
:1051200023C01FF024C020F026C021F039EC2EF05F
:10513000D8B02588255012000401E86BE96BFC0EFD
:105140000101176FB30E166F010EA3EC33F0880E3A
:105150000101296F130E2A6F000E2B6B2C6B2D6B28
:10516000FCEC9FF00101306F880E296F130E2A6F3F
:105170002B6B2C6B010E2D6FFCEC9FF0010130515D
:10518000180AD8B412003051160AD8B4120030519F
:105190001A0AD8B4120030511B0AD8B41200305188
:1051A000170AD8B41200B3EC46F07BEC46F0D10EEF
:1051B0000101295D070E2A59F8E3780E0401E85D24
:1051C000000EE959D8B01200BAD7E8CF1CF101019E
:1051D0001851B0EC39F015C11DF116C11EF11DC1F9
:1051E000D9FF1EC1DAFFDF50216F216701D0120005
:1051F000185104EC39F015C11FF116C120F11DC181
:10520000D9FF1EC1DAFFDF50DF06216F1CC122F17A
:105210001ED0D8902235196F19511F251A6FE86AD0
:1052200019BFE86820211B6F020E1A25D96E000EE7
:105230001B21DA6E2251020DF3501F25E16E000E84
:105240002021E26EDECFE6FFDDCFE5FF222B2151EC
:10525000225DD8B01200DDD733D01FC0D9FF20C0E7
:10526000DAFFDF5012E036D8F76403D00800F550BB
:1052700005D0F6CFE9FFF7CFEAFFEF50256E1FC04C
:10528000D9FF20C0DAFFDF1817E01FC0D9FF20C008
:10529000DAFFDF50256E1ED8F76403D00800F55002
:1052A00005D0F6CFE9FFF7CFEAFFEF50255C1F6E80
:1052B000206AD8A0200612001F4A202A214A222A4A
:1052C0002306D8A024062328D8B42428C6E11F6AC0
:1052D000206A120021C0F6FF22C0F7FF000EF86E10
:1052E0000F0E12000401286B296B24D00401C48F17
:1052F000040128810401C65125E00401288322D03D
:105300000401C48F1FD00401C48F0FEC44F025D8D2
:10531000F76403D00800F55005D0F6CFE9FFF7CFCA
:10532000EAFFEF500101156F15A50CD0010E040125
:10533000286F08D0040120511F0BD8E0010AE0E0DB
:10534000030AE1E00401C4AF1200040EC36F280E8B
:10535000C26FC481020EC56F020CC7C4F6FFC8C479
:10536000F7FF000EF86E0F0E120014B20AAE24D032
:10537000180E0101176503D03C0E176502D0018499
:1053800001D0019429D824E00201AA4BAB2B0101E2
:1053900015510201AA5D010116510201AB590AE340
:1053A0000001019601B4018601B602D0D890120026
:1053B000D88012000001F8D73E0E0101176102D01B
:1053C000019404D04C0E176501D0018405D8DCE1AE
:1053D0000201AA6BAB6BEED7010E01A4000E010116
:1053E000186F010E01A6000E181B120014B20AAEAF
:1053F00024D0180E0101176503D03C0E176502D0AA
:10540000018001D0019029D824E00201A84BA92BEA
:10541000010115510201A85D010116510201A959AE
:105420000AE30001019201B0018201B202D0D890DA
:105430001200D88012000001F8D73E0E010117615A
:1054400002D0019004D04C0E176501D0018005D820
:10545000DCE10201A86BA96BEED7010E01A0000EE2
:105460000101186F010E01A2000E181B120014B2E8
:105470000AAE24D0180E0101176503D03C0E176543
:1054800002D0018801D0019829D824E00201AC4B58
:10549000AD2B010115510201AC5D01011651020154
:1054A000AD590AE30001019A01B8018A01BA02D09C
:1054B000D8901200D88012000001F8D73E0E0101EA
:1054C000176102D0019804D04C0E176501D00188F5
:1054D00005D8DCE10201AC6BAD6BEED7010E01A883
:1054E000000E0101186F010E01AA000E181B120018
:1054F00014B20AAE24D0180E0101176503D03C0E79
:10550000176502D0028001D0029029D824E0020160
:10551000B04BB12B010115510201B05D01011651D3
:105520000201B1590AE30001029202B0028202B202
:1055300002D0D8901200D88012000001F8D73E0E99
:105540000101176102D0029004D04C0E176501D002
:10555000028005D8DCE10201B06BB16BEED7010E21
:1055600002A0000E0101186F010E02A2000E181B0E
:10557000120014B20AAE24D0180E0101176503D030
:105580003C0E176502D0018C01D0019C29D824E083
:105590000201AE4BAF2B010115510201AE5D0101BD
:1055A00016510201AF590AE30001019E01BC018EB0
:1055B00001BE02D0D8901200D88012000001F8D7A6
:1055C0003E0E0101176102D0019C04D04C0E1765FC
:1055D00001D0018C05D8DCE10201AE6BAF6BEED7D8
:1055E000010E01AC000E0101186F010E01AE000E9C
:1055F000181B1200E8CF27F0E2670AD027A403D0D7
:10560000206A2A0E02D0206A2C0E1F6E91EF1BF02A
:10561000E20522E10AAC03D01C9C27B41C8C0001DB
:105620000ABC120019A603D000011CBE1200000122
:1056300006AA120027A408D0206A2A0E1F6E91EC39
:105640001BF000011C8A1200206A2C0E1F6E91ECC8
:105650001BF000011C9A1200E251020AD8A41200A9
:1056600019A603D000011CBE1200000106AA1200F8
:1056700027B4E2D7E9D7E8CF27F0E1670AD027A01F
:1056800003D0206A220E02D0206A240E1F6E91EFF2
:105690001BF0E10522E10AAC03D01C9227B01C826A
:1056A00000010ABC120019A603D000011CB41200AC
:1056B000000106AA120027A008D0206A220E1F6E41
:1056C00091EC1BF000011C801200206A240E1F6E5A
:1056D00091EC1BF000011C901200E151020AD8A4C9
:1056E000120019A603D000011CB41200000106AA82
:1056F000120027B0E2D7E9D7E8CF27F0E3670AD056
:1057000027A603D0206A2E0E02D0206A300E1F6E0C
:1057100091EF1BF0E30522E10AAC03D01D9227B6FE
:105720001D8200010ABC120019A603D000011DB49D
:105730001200000106AA120027A608D0206A2E0E29
:105740001F6E91EC1BF000011D801200206A300ECC
:105750001F6E91EC1BF000011D901200E351020A34
:10576000D8A4120019A603D000011DB41200000134
:1057700006AA120027B6E2D7E9D70401286B296BE5
:105780002AD00401C48F040128810401C6512BE0F2
:105790000401288328D00401C48F25D00401C48FBC
:1057A000ABEC43F0C7C4F6FFC8C4F7FF000EF86EB9
:1057B0000F0EF76403D00800F55005D0F6CFE9FFCF
:1057C000F7CFEAFFEF500101006F00A50CD0010EEA
:1057D0000401286F08D0040120511F0BD2E0010AF8
:1057E000DAE0030ADBE00401C4AF1200040EC36F69
:1057F000280EC26FC481020EC56F020CE8CF27F0DD
:10580000E4670AD027A803D0206A360E02D0206AA7
:10581000380E1F6E91EF1BF0E40522E10AAC03D0B5
:105820001D9827B81D8800010ABC120019A603D0D4
:1058300000011DBA1200000106AA120027A808D014
:10584000206A360E1F6E91EC1BF000011D861200BF
:10585000206A380E1F6E91EC1BF000011D9612009D
:10586000E451020AD8A4120019A603D000011DBAFF
:105870001200000106AA120027B8E2D7E9D733D0F8
:1058800024C11BF125C11CF126C11DF127C11EF148
:1058900026C115F127C116F124EC38F015C11FF10E
:1058A00016C120F16EEC33F01C511B1105E124C12F
:1058B00024F125C125F112002429166F000E25219F
:1058C000176F26C1F6FF27C1F7FF000EF86E08001C
:1058D000F550186F196B18BF190764EC3EF016C12C
:1058E00024F117C125F12551241106E024C1D9FF67
:1058F00025C1DAFFDF50C4E1246B256B1200F80EDE
:105900000101176FB40E166F010EA3EC33F0020104
:10591000E32BB3EC46F07BEC46F0E90E0101295D88
:10592000030E2A59F8E3020E0201E365020CE36B51
:10593000FB0E0101176F120E166F010EA3EC33F070
:10594000010E01012A6FF40E296FD8EC38F0B3EC88
:1059500046F07BEC46F0E90E0101295D030E2A5961
:10596000F8E38E9C8D98B3EC46F07BEC46F0E90EA4
:105970000101295D030E2A59F8E3D9EFC1F014B2F1
:105980000AAE26D0180E216403D03C0E216402D04A
:10599000018001D00190010E01A0000E226E010EC7
:1059A00001A2000E221A26E00201A84BA92B1F50CB
:1059B000A85D2050A9590AE30001019201B00182BB
:1059C00001B202D0D8901200D88012000001F8D79E
:1059D0003E0E216002D0019004D04C0E216401D013
:1059E0000180010E01A0000E226E010E01A2000E28
:1059F000221ADAE10201A86BA96BE8D7E8CF17F108
:105A000001011751FE0F166F0001FA6B0101186BAF
:105A10000DD0EF0E01011825D96EDA6A0301030ECD
:105A2000DA22DF506DEC46F00101182B1651185D9B
:105A3000F0E30001FA390F0BFDEC44F0186FED0EA6
:105A400001011725D96EDA6A030EDA22DF50181920
:105A500002E0D89012000001FA510F0BFDEC44F067
:105A6000186FEE0E01011725D96EDA6A030EDA22DD
:105A7000DF501819EEE1D8801200FC0E176FA20E4D
:105A8000166F010EA3EC33F0300E0101296F750E75
:105A90002A6F000E2B6B2C6B2D6BFCEC9FF0010121
:105AA000306F30510C0A03E03051090A01E1000C5B
:105AB00030C131F1300E296F750E2A6F2B6B2C6BB4
:105AC000010E2D6FFCEC9FF0080AF1E1010131514C
:105AD0000B0A0AE1B3EC46F07BEC46F0890E0101BB
:105AE000295D130E2A59F8E331510A0A03E03151B6
:105AF0000B0ADDE13151120014B20AAE26D0180EA5
:105B0000216403D03C0E216402D0018C01D0019CA1
:105B1000010E01AC000E226E010E01AE000E221A23
:105B200026E00201AE4BAF2B1F50AE5D2050AF59A7
:105B30000AE30001019E01BC018E01BE02D0D89093
:105B40001200D88012000001F8D73E0E216002D06A
:105B5000019C04D04C0E216401D0018C010E01ACDB
:105B6000000E226E010E01AE000E221ADAE10201D1
:105B7000AE6BAF6BE8D714B20AAE26D0180E216414
:105B800003D03C0E216402D0018401D00194010EA7
:105B900001A4000E226E010E01A6000E221A26E0BC
:105BA0000201AA4BAB2B1F50AA5D2050AB590AE350
:105BB0000001019601B4018601B602D0D89012000E
:105BC000D88012000001F8D73E0E216002D0019467
:105BD00004D04C0E216401D00184010E01A4000EFA
:105BE000226E010E01A6000E221ADAE10201AA6B52
:105BF000AB6BE8D714B20AAE26D0180E216403D0DE
:105C00003C0E216402D0018801D00198010E01A848
:105C1000000E226E010E01AA000E221A26E00201D9
:105C2000AC4BAD2B1F50AC5D2050AD590AE30001C9
:105C3000019A01B8018A01BA02D0D8901200D88026
:105C400012000001F8D73E0E216002D0019804D066
:105C50004C0E216401D00188010E01A8000E226EB5
:105C6000010E01AA000E221ADAE10201AC6BAD6B43
:105C7000E8D714B20AAE26D0180E216403D03C0E29
:105C8000216402D0028001D00290010E02A0000E19
:105C9000226E010E02A2000E221A26E00201B04B73
:105CA000B12B1F50B05D2050B1590AE300010292A0
:105CB00002B0028202B202D0D8901200D880120044
:105CC0000001F8D73E0E216002D0029004D04C0EA5
:105CD000216401D00280010E02A0000E226E010E8E
:105CE00002A2000E221ADAE10201B06BB16BE8D712
:105CF000010EB0EC39F015C118F116C119F118C137
:105D0000D9FF19C1DAFFDF6A020EB0EC39F015C114
:105D100018F116C119F118C1D9FF19C1DAFFDF6AEC
:105D2000030EB0EC39F015C118F116C119F118C104
:105D3000D9FF19C1DAFFDF6A040EB0EC39F015C1E2
:105D400018F116C119F118C1D9FF19C1DAFFDF6ABC
:105D5000050EB0EC39F015C118F116C119F118C1D2
:105D6000D9FF19C1DAFF000EDF6E000C1A0E5CECD1
:105D700044F00301B26BB36B02942FD0ABECEAF0AA
:105D800002A42BD002940201CE6701D026D0080EC7
:105D900001011C6FA00E1B6FFD0E1E6F6B0E1D6FA1
:105DA000206B070E1F6F0AEC28F01C511B1102E13B
:105DB000D8901200080E01011C6FA00E1B6FFB0E85
:105DC0001E6F300E1D6F206B090E1F6F0AEC28F03E
:105DD0001C511B1102E1D8801200310E0301B25D8B
:105DE000750EB359F8E2CAD7E8CF21F1196B580EF6
:105DF000186FE5EC2FF0226F1F0507E1186B580EA6
:105E0000176F2251FE0B21110CD01F51020A0CE119
:105E1000186B580E176FD8902135206F2251FD0B4B
:105E200015D0196FD6EF36F01F51030A05E1186B34
:105E30000FD82251FB0B0AD01F51040AD8A412001C
:105E4000186B06D8D89020372251F70B2011E9D7CC
:105E5000580E176F21C120F1D8902037D8902037E5
:105E6000580C1A6B18AF06D0176D181FD8B0182B26
:105E7000010E1A6F16AF06D0156D161FD8B0162B6F
:105E8000010E1A1B1B6B1C6B185117111BE0010E26
:105E9000196F04D0D89017371837192B18AFFAD7C5
:105EA000D8901B371C371751155D1851165905E34B
:105EB0001751155F1851165B1B81D8901833173393
:105EC000192FEED71A5104E01B6D1C1FD8B01C2BE4
:105ED0001BC115F11CC116F11200E8CF5BF152C6CF
:105EE00015F101015B5192EC41F002E2D8901200F1
:105EF00000010CAAFBD78A8C0401DA6BDB6B000172
:105F00001A8EB1EC0FF001015B39F00B5A6F030EE2
:105F10004A6F5A518CECF2F04AC158F14BC159F119
:105F20000601525129EC46F002E2D88012005B5182
:105F3000C3EC3EF001015A6F58C139F159C13AF131
:105F40005BC13BF15AC13CF1030E3D6FABEC35F048
:105F5000ECD715C1D9FF16C1DAFF10EE06F028D82C
:105F600010EE05F01551E1261651E222DFCFE7FFD2
:105F700020EE04F01551D9261651DA2215C1E1FFA1
:105F800016C1E2FFDFCFE7FF20EE02F01551D92660
:105F90001651DA2210EE04F00BD8D051DF6E20EE4D
:105FA00002F01551D9261651DA22CFC1DFFF1200B7
:105FB0001551E1261651E222DFCFE7FF20EE01F076
:105FC0001551D9261651DA2212000A0E01011D6F51
:105FD000A00E1E6F30D01D07D36B41EC43F00101C2
:105FE0001E51E2EC3EF00101D36717D01951E2ECEB
:105FF0003EF001011851E2EC3EF041EC43F00101AA
:106000001E811E51E2EC3EF0000E7BEC3FF01C6F57
:1060100095EC40F001011C511200070E1B6FD00ED1
:106020001A6F01D000F001011A07D8A01B071A2926
:10603000D8B41B29F7E11D51800A7F0FCCE2000C78
:10604000E8CF5BF168C615F101015B5192EC41F0BC
:1060500002E2D8901200B1EC0FF001015B39F00BB5
:106060005A6F010E2B6F2C6B040E6CECD5F0F1E324
:10607000250E01014A6F5A518CECF2F04AC158F1D9
:106080004BC159F10601685129EC46F002E2D88073
:1060900012005B51C3EC3EF001015A6F58C139F157
:1060A00059C13AF15BC13BF15AC13CF1030E3D6F5E
:1060B000ABEC35F0ECD7E8CF5BF166C615F101012A
:1060C0005B5192EC41F002E2D8901200B1EC0FF07B
:1060D00001015B39F00B5A6F010E2B6F2C6B020E16
:1060E0006CECD5F0F1E3230E01014A6F5A518CECB0
:1060F000F2F04AC158F14BC159F10601665129EC41
:1061000046F002E2D88012005B51C3EC3EF0010180
:106110005A6F58C139F159C13AF15BC13BF15AC1CB
:106120003CF1030E3D6FABEC35F0ECD7E8CF22F03D
:10613000216A22C020F0010E20161F50010B2018EA
:10614000D8A4218022C020F0020E20161F50020B7E
:106150002018D8A4218222C020F0040E20161F503F
:10616000040B2018D8A4218422C020F0080E201689
:106170001F50080B2018D8A4218622C020F0100E32
:1061800020161F50100B2018D8A4218822C020F000
:10619000200E20161F50200B2018D8A4218A215031
:1061A0001200E8CF5BF167C615F101015B5192EC7B
:1061B00041F002E2D8901200B1EC0FF001015B391E
:1061C000F00B5A6F010E2B6F2C6B030E6CECD5F09D
:1061D000F1E3240E01014A6F5A518CECF2F04AC1EE
:1061E00058F14BC159F10601675129EC46F002E222
:1061F000D88012005B51C3EC3EF001015A6F58C1C8
:1062000039F159C13AF15BC13BF15AC13CF1030E7E
:106210003D6FABEC35F0ECD7080E236F33D00E0E8C
:10622000256F1F25216F000E2021226F12D0250718
:10623000C10E01012525D96EDA6A010EDA22210785
:10624000D8A0220721C118F122C119F1E5EC2FF0E5
:10625000DF6E2567ECD7246B256BC10E2525D96E23
:10626000DA6A010EDA22DF50241B252B2551800A21
:10627000730FF3E3245121EECEF0DF6202D0D88019
:10628000120023072367CBD7D89012000401E86BD4
:10629000E96BF80E0101176FF90E166F010EA3ECF2
:1062A00033F0880E0101296F130E2A6F000E2B6B3D
:1062B0002C6B2D6BFCEC9FF00101306F30512D0ADF
:1062C00006E1130E2A6F880E296FD8EF38F0130EEF
:1062D0002A6F880E296FD8EC38F0B3EC46F07BECCF
:1062E00046F0D10E0101295D070E2A59F8E3B40EDC
:1062F0000401E85D000EE959CCE3FF00CAD7E8CFFE
:106300005BF153C615F101015B5192EC41F002E2E1
:10631000D89012008A9C0401DA6BDB6B00011A9E94
:10632000B1EC0FF001015B39F00B5A6F040E4A6FAC
:106330005A518CECF2F04AC158F14BC159F10601A7
:10634000535129EC46F002E2D88012005B51C3ECB5
:106350003EF001015A6F58C139F159C13AF15BC1A0
:106360003BF15AC13CF1030E3D6FABEC35F0ECD77D
:1063700020EE02F01551D9261651DA22DF50196F9E
:1063800020EE02F024D8E750176F10EE02F01551FE
:10639000E1261651E222E750186F18390F0B17113A
:1063A000DF6E20EE01F013D8DFCFE7FF20EE01F023
:1063B0001551D9261651DA22DF6A20EE01F0155167
:1063C000D9261651DA221939F00BDF6E1200155159
:1063D000D9261651DA2215C1E1FF16C1E2FF1200DB
:1063E000E8CFBEF1000108BA050C000115B2050C9A
:1063F0009EC2BFF11DD0BE6704D080EC38F0010111
:10640000C06FC05119E0BF6701D016D0C051040A57
:1064100003E0C051020AD8B47FEC2CF0B3EC46F094
:106420007BEC46F0990E0101295D3A0E2A59F8E3FA
:106430000101BF07BF29DFE1C051040A03E0C051D9
:10644000020AD8B47FEC2CF00101C0511200FC0EFE
:10645000176FC30E166F010EA3EC33F0880E010107
:10646000296F130E2A6F000E2B6B2C6B2D6BFCEC1F
:106470009FF00101306F30513A0AD8A41200070E84
:10648000306F8F0E01013025D96EDA6A060EDA22DE
:10649000350E3025E16EE26A070EE222DFCFE7FF1C
:1064A000302B3051800A660FECE307014F6B130E5F
:1064B00001012A6F880E296FD8EF38F0E8CF5BF121
:1064C00055C615F101015B5192EC41F002E2D89002
:1064D000120000010CACFBD78A8EB1EC0FF0010169
:1064E0005B39F00B5A6F060E4A6F5A518CECF2F082
:1064F0004AC158F14BC159F10601555129EC46F0FA
:1065000002E2D88012005B51C3EC3EF001015A6FE9
:1065100058C139F159C13AF15BC13BF15AC13CF163
:10652000030E3D6FABEC35F0ECD7E8CF25F1250736
:10653000DF5194EC44F01F6FDE5194EC44F0206F77
:106540002039F00B1F11236F2551220DF80EF32473
:10655000186F3F0EF420196FE5EC2FF0246F2451D3
:10656000231902E0D89012002551220DF90EF324D0
:10657000216F3F0EF420226F21C118F122C119F1C1
:10658000E5EC2FF0266F010E2665ECD7100E266580
:1065900001D0E8D7D88012000401C48F0F014D6BE1
:1065A0004E6B0401BE6B22C4BDF40401226704D00B
:1065B000100E0401CD6F100C200E0401CD6F0401EC
:1065C000CE6B4B0ECF6FD06BD16BD26BD36B080EF3
:1065D000D46F010ED56F0401CC6BCC8F0401B16B6D
:1065E0000401B06B1A0E0F014E6F0401148D149F3D
:1065F0001E0E0F014F6F04011C8D1C9F188D189FDC
:106600008AEF45F00401C48F0F014D6B4E6B0401FE
:10661000BE6B22C4BDF40401226704D0100E040135
:10662000CD6F100C200E0401CD6F0401CE6B4B0E0C
:10663000CF6FD06BD16BD26BD36B080ED46F010EC2
:10664000D56F0401CC6BCC8F0401B16B0401B06B2E
:106650001A0E0F014E6F0401148D149F1E0E0F01B0
:106660004F6F04011C8D1C9F188D189F97EF45F0EC
:10667000E8CF31F189EC20F0D8B089EC20F0D8B027
:1066800012000101326B316712D06A0E3225176F8A
:10669000186B130E1823280E01013225D96EDA6A01
:1066A000060EDA22DF50196FD6EC36F011D0790ED3
:1066B0003225176F186B130E1823280E010132258F
:1066C000D96EDA6A060EDA22DF50196FD6EC36F090
:1066D0000101322B0E0E3265D6D70E0C29D01DC10A
:1066E000F6FF1EC1F7FF000EF86E0800F550B1EC82
:1066F00045F0216F1BC1D9FF1CC1DAFFDF50B1EC9F
:1067000045F0226F2151225D236F0101236706D0DE
:106710001BC1D9FF1CC1DAFFDF5006E123511B6FFB
:106720001C6B1BBF1C0712001B4B1C2B1D4B1E2B75
:106730001F07D8A0200701011F29D8B42029CFE1C5
:106740001B6B1C6B1200E8CF18F10101185118E007
:10675000410E5CEC44F0540E5CEC44F011D00101AD
:106760001FD8F76403D00800F55005D0F6CFE9FF35
:10677000F7CFEAFFEF505CEC44F00101164B172B0A
:1067800001010ED8F76403D00800F55005D0F6CF0C
:10679000E9FFF7CFEAFFEF500009D8B41200DFD7C6
:1067A00016C1F6FF17C1F7FF000EF86E0F0E1200AC
:1067B000E8CF27F16DC615F10101275192EC41F0A8
:1067C00002E2D89012000501D351080AFAE11F0E27
:1067D000D325D96EDA6A050EDA22DF6A230E0101AB
:1067E000256F050E266F25C11BF126C11CF1ABECF0
:1067F0001CF01BC128F11CC129F128C11FF129C1BE
:1068000020F128EC40F0DDE3500E206FD20E1F6F18
:10681000ACEC38F0FF00D8801200049C9CA29CB421
:10682000048CAACFF9F004AC05D09C989C88000198
:106830000592120005820CAE0AD0000E0201DD2581
:10684000D96EDA6A090EDA22F9C0DFFFDD2B0BAA56
:1068500004D00001F9517EEF18F000011EB6ADEC36
:1068600004F0000113BC02D0000117B20BEC12F0CF
:1068700005A404D00001F9516FEC3BF00001F9517F
:10688000ADEFCDF0E8CF27F127C115F1166B270E3C
:10689000186F100E176F65EC42F01C51640DF3CFAA
:1068A0001FF1F4CF20F11D510A0DF3501F25216F68
:1068B000F4502021226F15512125236F16512221DA
:1068C000246F1BC115F1166B030E186FE80E176FBE
:1068D00065EC42F015512325256F16512421266FB2
:1068E0001E5125251B6F000E26211C6F1200E8CFBC
:1068F0005BF156C615F101015B5192EC41F002E2E9
:10690000D89012008A9EB1EC0FF001015B39F00BB8
:106910005A6F070E4A6F5A518CECF2F04AC158F187
:106920004BC159F10601565129EC46F002E2D880DC
:1069300012005B51C3EC3EF001015A6F58C139F1AE
:1069400059C13AF15BC13BF15AC13CF1030E3D6FB5
:10695000ABEC35F0ECD71A6B16AF06D0156D161FE1
:10696000D8B0162B010E1A6F18AF04D0176D181F70
:10697000D8B0182B1851171117E0010E196F04D059
:10698000D89017371837192B18AFFAD71751155D4C
:106990001851165904E31751155F1851165BD8901A
:1069A00018331733192FF2D71A5104E0156D161F3B
:1069B000D8B0162B15C115F116C116F11200E8CF8B
:1069C0005BF163C615F101015B5192EC41F002E20B
:1069D000D8901200B1EC0FF001015B39F00B5A6F47
:1069E000200E4A6F5A518CECF2F04AC158F14BC15B
:1069F00059F10601635129EC46F002E2D8801200F9
:106A00005B51C3EC3EF001015A6F58C139F159C1D5
:106A10003AF15BC13BF15AC13CF1030E3D6FABEC67
:106A200035F0ECD7E8CF5BF164C615F101015B519D
:106A300092EC41F002E2D8901200B1EC0FF00101AB
:106A40005B39F00B5A6F210E4A6F5A518CECF2F001
:106A50004AC158F14BC159F10601645129EC46F085
:106A600002E2D88012005B51C3EC3EF001015A6F84
:106A700058C139F159C13AF15BC13BF15AC13CF1FE
:106A8000030E3D6FABEC35F0ECD7E8CF60F150C6AC
:106A900015F10101605192EC41F002E2D890120030
:106AA0006051C3EC3EF001015F6F60C11FF15F51A7
:106AB000010AF4EC2EF0B1EC0FF001016039F00B9B
:106AC0005F6F010E4A6F5F518CECF2F0060150517E
:106AD00029EC46F002E2D88012006051C3EC3EF08F
:106AE00001015F6F5FC158F1605124ECE8F0F3D70A
:106AF000E8CF5BF162C615F101015B5192EC41F008
:106B000002E2D8901200B1EC0FF001015B39F00BFA
:106B10005A6F190E4A6F5A518CECF2F04AC158F173
:106B20004BC159F10601625129EC46F002E2D880CE
:106B300012005B51C3EC3EF001015A6F58C139F1AC
:106B400059C13AF15BC13BF15AC13CF1030E3D6FB3
:106B5000ABEC35F0ECD739513E6F030E3A153F6F71
:106B60003DC140F1416B0D0ED89040374137E82EC2
:106B7000FBD73BC142F1436B0A0ED89042374337F3
:106B8000E82EFBD740514211446F41514311456FEC
:106B90003E514411466F3F514511476F3C51D8A4B7
:106BA000478F46C130F147C131F13BC132F1E5ECCD
:106BB00018F002E3D8801200D8901200E8CF5BF101
:106BC00065C615F101015B5192EC41F002E2D890EB
:106BD0001200B1EC0FF001015B39F00B5A6F220E7D
:106BE0004A6F5A518CECF2F04AC158F14BC159F13D
:106BF0000601655129EC46F002E2D88012005B5193
:106C0000C3EC3EF001015A6F58C139F159C13AF154
:106C10005BC13BF15AC13CF1030E3D6FABEC35F06B
:106C2000ECD7416A0301EF0502E0D89012000101A0
:106C3000016BEF0E01010125D96EDA6A0301030E23
:106C4000DA22DF50F76F0101006B0301F7514118A1
:106C5000F86F0301F83302E3180E411A00F0000147
:106C600041330301F733D8900101002B070E006573
:106C7000ECD7012B060E0165DCD70301F651411854
:106C8000D4E1D880120000010DAC000C01011C6B96
:106C900015D0000E01011C25D96EDA6A0A0EDA221F
:106CA0001CC117F1186B17BF180717511525E16E96
:106CB00018511621E26EDFCFE7FF1C2BE4C217F15B
:106CC0000101186B1CC119F11A6B19BF1A071A516F
:106CD000800A1B6F1751195D1851800A1B59D9E39F
:106CE0000D9C0201E4511200E8CF5BF101015B054C
:106CF00002E0D8901200B1EC0FF001015B39F00B0B
:106D00005A6F010E2B6F2C6B6CECD5F0F2E3230E57
:106D100001014A6F5A518CECF2F001014AC158F15D
:106D20004BC159F15B51C3EC3EF001015A6F58C1A0
:106D300039F159C13AF15BC13BF15AC13CF1030E43
:106D40003D6FABEC35F0D88012002DC127F12EC17C
:106D500028F12FC129F130C12AF185EC3EF0020162
:106D6000D05122E00301AA4BAB2BD890AA350101E8
:106D7000316F280E3125D96EDA6A080EDA22FAC48C
:106D8000DEFFFBC4DDFF0301D890AA350101316F9E
:106D9000000E3125D96EDA6A0801080EDA22000EDB
:106DA000DE6EDD6ED880000CD89012000A0E1D6FCA
:106DB000A00E1C6F26D01D07D36B41EC43F00101E0
:106DC0001C51E2EC3EF00101D3670DD01851E2EC0A
:106DD0003EF001011751E2EC3EF001011951E2ECE5
:106DE0003EF095EF40F0070E1B6FD00E1A6F01D0EA
:106DF00000F001011A07D8A01B071A29D8B41B29D3
:106E0000F7E11D51800A7F0FD8A01200D4D70101ED
:106E1000326B3DEC2DF00101336F33510B0A03E16E
:106E2000C7EC37F020D8335102E032511AE0B3EC0E
:106E300046F07BEC46F0990E0101295D3A0E2A5985
:106E4000F8E3326B3DEC2DF00101336F33510B0A47
:106E500003E1C7EC37F007D8335102E0325101E0CB
:106E6000010CBFEFF4F0010ED8A0000E326F12003B
:106E70001FC1F8F21B9A13D00101200507E11DC1C3
:106E800015F11EC116F1FDEC40F006D01DC115F143
:106E90001EC116F143EC36F00201D46FF76B02010C
:106EA000D46702D0F867E8D7F86703D000011B8ADF
:106EB000000CD407F75101011D25D96E000E1E21CB
:106EC000DA6EDF50216F0201F72B01012151120010
:106ED000E8CF58F1B1EC0FF00201F039F00B0101ED
:106EE0005B6F10D0820E4A6F5B518CECF2F005D0D4
:106EF000810E4A6F5B518CECF2F04AC159F14BC1E3
:106F00005AF104D05851EEE0010AF2E00201F051CA
:106F1000C3EC3EF001015B6F59C139F15AC13AF13E
:106F2000F0C23BF15BC13CF1030E3D6FABEF35F0BE
:106F300046840101186B520E176FE7C119F1D6ECA8
:106F400036F00101196B520E186FE5EC2FF00201BB
:106F5000F96F0101E56BB8C319F1B9C31AF1C5ECBA
:106F600024F0E76F14B20AAE06D00201F951E00B2B
:106F70000101E71905D00101E7510201F9190101E9
:106F8000E56FE5C1EDF3148E000146941200FB0E8F
:106F9000176F260E166F010EA3EC33F0E80E0101F9
:106FA000296FFD0E2A6F000E2B6B2C6B2D6BFCECEA
:106FB0009FF00101306F30510C0A11E03051090A85
:106FC0000EE03051080A0BE0E80E296FFD0E2A6F23
:106FD0002B6B2C6B010E2D6FFCEC9FF0EAD7305120
:106FE000080A02E1D8901200D880120037C12BF1B4
:106FF00038C12CF139C12DF13AC12EF105EC06F062
:1070000002E2D890120000010D9CB3EC46F013D0C0
:1070100000010DAC10D00A0E0101256F000E246F87
:1070200037C126F138C127F1B9EC09F002E3D88065
:10703000120000010D9C7BEC46F0E90E0101295D78
:10704000FD0E2A59DEE2E4D715C119F116C11AF175
:1070500001011951176F1A51186F194B1A2B17C1CB
:10706000F6FF18C1F7FF000EF86E0F0EF76403D09D
:107070000800F55005D0F6CFE9FFF7CFEAFFEF5053
:107080000009E6E1010119C117F11AC118F1155102
:10709000175F1651185BFF0E1725156FFF0E18218D
:1070A000166F1200F2943F6602D003EF46F03F04E1
:1070B00002E1E2EF45F03F50020A02E10DEF46F037
:1070C0003F50030A02E199EF3FF03F50040A02E10A
:1070D0005AEF39F03F50050A02E182EF44F03F5089
:1070E000060A02E1B8EF44F03F50070A02E17AEFE6
:1070F00040F03F50080A02E1D1EF3AF03F6A120037
:1071000007EC37F0BD6FBD5102E0BD5112001EA665
:1071100008D00301CB6B138C198416800001039EE9
:10712000000C00011782DDEC22F00101BD6F179207
:10713000BD0503E0BD51030A0EE10301CB6B138CC7
:1071400019841680039E0101BD51030AE9E1010E75
:1071500056ECC9F0000C020C1F29186F000E2021FC
:10716000196FE5EC2FF0216F1FC118F120C119F143
:10717000E5EC2FF0236F2151226F224B232B222984
:10718000D8B4232902E1226B236B1FC117F120C160
:1071900018F12351196FD6EC36F0010E01011F25AD
:1071A000176F000E2021186F22C119F1D6EF36F0AB
:1071B0000301B66BB76B01012B6B1BD0ABECEAF094
:1071C00089EC46F016E3AFEC46F001012C6F0DD0D0
:1071D0002C517BEC42F00DE301012B2B0AD02C51FA
:1071E000BDEC42F006E3D88012002B51F1E0010A19
:1071F000F6E00301B6510101295D0301B751010118
:107200002A59DCE2D8901200E8CF17F1170506E101
:10721000080E0101166F500E156F12001751020A69
:1072200006E1090E0101166F640E156F1200175169
:10723000030A06E10A0E0101166FA00E156F120077
:107240001751040A06E10B0E0101166FA00E156F0F
:107250001200060E0101166FF60E156F1200F2EC09
:1072600041F0186F20EE03F01651D9261751DA229B
:1072700018C1DFFFF2EC41F0186F20EE02F016515A
:10728000D9261751DA2218C1DFFFF2EC41F016C1FE
:10729000D9FF17C1DAFFDF6EF2EC41F0186F20EE74
:1072A00001F01651D9261751DA2218C1DFFF00016B
:1072B00009921200416609D02F0E0101016F100ED4
:1072C000006F54EC3DF03F6A12004106010E0101CF
:1072D000016F690E006F54EC3DF086A6120000F0BD
:1072E00086A6120000F086A6120011A206D0010E9A
:1072F0000401D76FF40ED66FE6D7330E0301EF6F9C
:10730000080E406E3F2A82EF44F0040E0101196F0F
:10731000030E186FE5EC2FF0216F040E196F020EAB
:10732000186FE5EC2FF0236F2151226FFF0E225DC5
:10733000000E235904E2040E206F1F6F040C040E8C
:10734000196F010E186FE5EC2FF0216F040E196F05
:10735000000E186BE5EC2FF0206F21511F6F12000B
:10736000E8CF17F10101170505E1020E166FFB0EBC
:10737000156F12001751020A06E1020E0101166F85
:10738000FC0E156F12001751030A06E1020E0101EF
:10739000166FFD0E156F12001751040A06E1020E5A
:1073A0000101166FFE0E156F1200020E0101166F1D
:1073B000FF0E156F1200E8CF1BF11A6B1C6B0AD081
:1073C000E90E01011C25D96EDA6A000EDA22DF50BF
:1073D0001A1B1C2B1BC115F1166B1CC117F1186B66
:1073E00017BF18071851800A196F1551175D1651EC
:1073F000800A1959E5E3E90E01011B25D96EDA6A05
:10740000000EDA221AC1DFFF12009E940201EB6B1C
:10741000000116BE12000301E49182ACE481080E63
:10742000E52BE56103D0D890E437080CE56BF90E45
:107430000201EA25D96EDA6A030EDA22E4C3DFFF1D
:10744000EA2B060EEA65060CEA6B829C949C829CF1
:10745000168E168C8F800001138812007F0E01019A
:1074600020D8DB8E18AE03D07F0E1BD8DB8C960E97
:107470000101D625176F186B020E18237F0ED62533
:10748000D96EDA6A060EDA22DF50196FD6EC36F0C2
:10749000530E0301F26F100EF36F0101D65157EF37
:1074A0003AF0D625D96EDA6A060EDA22000CE8CF59
:1074B0001AF1060E0301EF6F0101D0510301F06FC5
:1074C000CFC1F1F3F46B7F0E01011A25D96EDA6A90
:1074D000060EDA22DF50196F19AD05D01A510F0BC5
:1074E0000301F31304D01A39F00B0301F413F56B05
:1074F000F66B030E0101176FEF0E166F91EF42F05E
:107500000251040A02E0D890120000C1D9FF01C163
:10751000DAFFDF504E0AF7E120EE01F00051D926E4
:107520000151DA22DF50100AEEE120EE02F00051A4
:10753000D9260151DA22DF505E0AE5E120EE03F0A0
:107540000051D9260151DA22DF50AC0ADCE1D880A3
:107550001200E8CF60F151C615F10101605192ECC3
:1075600041F002E2D8901200B1EC0FF00101603955
:10757000F00B5F6F020E4A6F5F518CECF2F0060168
:10758000515129EC46F002E2D88012006051C3EC60
:107590003EF001015F6F5FC158F1605124ECE8F0EB
:1075A000F3D7402E13D011EC36F00DE31182010E0B
:1075B0000401D76FF40ED66F11961B943C0E020196
:1075C000CD6F010E456E3F6A03EF46F00301F633BF
:1075D0000301F5330301F4330301F3330301F23301
:1075E0000301F1330301F0330301EF333F067AEF78
:1075F00040F0010E01012A6FF40E296FD8EC38F02B
:10760000F60E0101176F5C0E166F010EA3EC33F03E
:10761000030E01012A6FE80E296FD8EC38F0F60E40
:107620000101176F500E166F010EA3EC33F0030E1D
:1076300001012A6FE80E296FD8EC38F00001199E7D
:107640001200E8CF21F121072151330D890EF324D7
:10765000226F130EF420236F246BFA0E01012425F0
:10766000D96EDA6A0601060EDA2222C118F123C1A8
:1076700019F1E5EC2FF0DF6E224B232B242B030EA8
:107680002465EBD7060E0101206FFA0E1F6F120062
:10769000DE6BDF6BC12903E1390EDE6FDF6FC15195
:1076A000030A0BE1C6390F0BFDEC44F0DE6FC65147
:1076B0000F0BFDEC44F0DF6F1200C151060A04E02D
:1076C000C151070AD8A41200C5510F0BFDEC44F0BC
:1076D000DE6FC6390F0BFDEC44F0DF6F1200E8CF10
:1076E0001FF01F502B0A03E10201C66B12001E0E91
:1076F0000201C625D96EDA6A070EDA221FC0DFFF43
:10770000C62BC651160AD8A4120007011E51430AFF
:107710000AE11F51470A07E12051530A04E12151B0
:107720004E0AD8B412000001059412000401205141
:10773000800AD8A41200800E0401C46F13D0EB0E8F
:107740000401C36FCD0EC26F120EC56F120CEB0E8B
:107750000401C36F8A0EC26F430EC56F430C040150
:10776000C46B120004012351010AE9E0030AEFE0AF
:10777000010AD8A41200F3D715C11BF116C11CF1E0
:1077800002D01B4B1C2B1BC1D9FF1CC1DAFFDF50E1
:10779000F8E11751196F18511A6F174B182B19C1AF
:1077A000F6FF1AC1F7FF000EF86E1BC1D9FF1CC10E
:1077B000DAFF1B4B1C2B0800F5CFDFFFDF50D8B4DE
:1077C0001200E7D7C76A300EC66E0101166B176B41
:1077D000186B196B550E1A6FE7EC43F0166B010E20
:1077E000176F186B196BAA0E1A6FE7EC43F0000EB7
:1077F000166B176B186B196BA7EC42F0550AD8A4DF
:107800001200166B010E176F186B196BA7EF42F081
:1078100004012051800AD8A41200800E0401C46F14
:1078200013D0EB0E0401C36FCD0EC26F120EC56FE5
:10783000120CEB0E0401C36F8A0EC26F430EC56FAC
:10784000430C0401C46B120004012351010AE9E056
:10785000030AEFE0010AD8A41200F3D7E8CF69F1D8
:1078600004C515F10101695192EC41F002E2D89092
:107870001200B1EC0FF001016939F00B686F790E5D
:107880004A6F68518CECF2F00001118C90EC46F0DC
:107890007FEC2CF01B9216820101DD5103E0DD0527
:1078A0000201E66FD88012007F0E0101D625D96E45
:1078B000DA6A060EDA22C00EDF167F0ED62512D83F
:1078C0001EAF2EEF3AF07F0ED6250CD81EAD05D098
:1078D000000118BE12002EEF3AF0000118AE12009F
:1078E0002EEF3AF0D96EDA6A060EDA22DF501E6FFA
:1078F00012001DC115F11EC116F11FC117F120C1E3
:1079000018F131EC2FF015C123F116C124F11DC17E
:1079100015F11EC116F11FC117F120C118F1ABEC12
:1079200034F015C121F116C122F121C11DF122C18E
:107930001EF123C11FF124C120F112001A6B1B6B31
:10794000185117111BE0010E196F04D0D89017378A
:107950001837192B18AFFAD7D8901A371B37175189
:10796000155D1851165905E31751155F1851165B2F
:107970001A81D89018331733192FEED71AC115F181
:107980001BC116F11200F294EB0E0101016F500EB3
:10799000006F54EC3DF0000111B00ED086B602D05D
:1079A000416A1200412A4150330AD8A41200416AA8
:1079B000118000011182120086B6F2D7412A41508F
:1079C000330AD8A41200416A1190000111821200FA
:1079D000F90E0101176FF60E166F010EA3EC33F0CE
:1079E000B3EC46F00CD089EC46F009E3AFEC46F07E
:1079F00001012B6F2B513E0A02E1D89012007BEC63
:107A000046F0890E0101295D130E2A59ECE31B0E85
:107A10005CEC44F0D88012000501FE51D8A412009D
:107A2000000112B012001F6A0101E6A102D0068413
:107A30001F2A0101E6A302D006841F2A0101E6A540
:107A400002D006841F2A1F6601D0069407BC02D00C
:107A500014AC03D00001088812000001089812003D
:107A600036C140F137C141F1426B436B010E3F6FAC
:107A70003A0E3E6F010E226F400E216F38C123F186
:107A800039C124F1010E266F3E0E256F1FECBFF0A9
:107A900040C1D9FF41C1DAFFDF6A3651405D366F20
:107AA00037514159376F1200D59E0051026F015175
:107AB000036F046B056B02510008066F000E03553F
:107AC000076F010E0455086F000E0555096F07C1B9
:107AD00006F108C107F109C108F1096B08BF09697E
:107AE0000651D76E00510008D66ED58E12001BD0FD
:107AF000C7C4F6FFC8C4F7FF000EF86EC9C4D9FFAB
:107B0000CAC4DAFF0F0EF76403D00800F55005D0A1
:107B1000F6CFE9FFF7CFEAFFEF50DF6E0401C74B66
:107B2000C82BC94BCA2B0401CB07CB29D8B41200F0
:107B3000DFD7E8CF15F1150501E1010C1551020A57
:107B400001E1020C1551040A01E1030C1551080A68
:107B500001E1040C1551100A01E1050C1551200A30
:107B600001E1060C1551400A01E1070C1551800A8C
:107B700001E1080C000C32EC46F00001128085ECAB
:107B800039F00201E56B149A0101010E376F440EC2
:107B9000366FF90E396FA90E386F130E3B6FFC0E5E
:107BA0003A6F30EC3DF03651556F010E166F440EB2
:107BB000156F55C117F160EF45F01BD0C7C4F6FF34
:107BC000C8C4F7FF000EF86EC9C4D9FFCAC4DAFFF3
:107BD0000F0EF76403D00800F55005D0F6CFE9FF8B
:107BE000F7CFEAFFEF50DF6E0401C74BC82BC94B3C
:107BF000CA2B0401CB07CB29D8B41200DFD74566C6
:107C000002D041EF45F0450402E1BEEF45F045509A
:107C1000020A02E144EF46F04550030AF6E04550FF
:107C2000040AF8E04550050AF0E04550060A02E172
:107C3000F8EF45F04550070A02E1D6EF45F0456AF6
:107C400012002AC12BF11CD026C117F127C118F14F
:107C500028C119F129C11AF12BC11BF18AEC22F0BC
:107C60002C6FD351D8A412002C512627000E2723A5
:107C70002C51010DF3502827000E29232C512B5F86
:107C80002B67E2D71200040E0101186F176B196FF2
:107C9000D6EC36F0040E0101186F010E176F040EBA
:107CA000196FD6EC36F0040E0101186F020E176F33
:107CB000000E196BD6EC36F0040E0101186F030E9E
:107CC000176F196BD6EF36F01851B1EC45F0186FFD
:107CD000196B18BF190710D016C1D9FF17C1DAFFE9
:107CE000DF50B1EC45F0181905E116C116F117C1C6
:107CF00017F11200164B172B16C1D9FF17C1DAFF67
:107D0000DF50EAE1166B176B120027C122F128C180
:107D100023F129C124F12AC125F120EC3FF02B6F7A
:107D20002B39F00B2C6F27C122F128C123F129C177
:107D300024F12AC125F120EC3FF02C272C5102011F
:107D4000D02701012C511200000109B2120020C0FD
:107D5000D9FF21C0DAFFDF50DAEC41F020EE01F06C
:107D60002050D9262150DA22DF50DAEC41F020EE03
:107D700002F02050D9262150DA22DF50DAEC41F00F
:107D800000010E841200E8CF22F10101196B580E98
:107D9000186FE5EC2FF0216F2251030A03E1000177
:107DA0001EBA010C22C11FF1FF0E01011F2721C1C4
:107DB00020F11F2B02D0D89020331F2FFCD7205149
:107DC000010B1200E8CF15F1166B15AF03D00001BF
:107DD000038802D000010398F0EC3FF00101D89035
:107DE0001537162B1651800A780FEFE3FBEC43F0A2
:107DF000000103A612000101D3671200030ED36F26
:107E0000030C1F511E1117E0010E206F04D0D890F3
:107E10001E371F37202B1FAFFAD71E511C5D1F5175
:107E20001D5904E31E511C5F1F511D5BD8901F3369
:107E30001E33202FF2D71CC11CF11DC11DF11200F1
:107E400022C11DF123C11EF124C11FF125C120F162
:107E500038EC37F00101266F0BAA04D026C1A9FF28
:107E6000A8A2FED70101266701D0000C400E2665AE
:107E700003D02651C90F12002651D00F1200636A99
:107E8000626A9F0E0F015D6F5E6B4D6B4E6BFB0E5A
:107E90005C6F658C0401C46B0401C16B0401BD6B94
:107EA0000401CD6B659C160E0F014C6F02D06296DB
:107EB000040062B6FCD7659812001F4B202B226B82
:107EC000F00E01012225D96EDA6A030EDA22DF50A4
:107ED000216F1F51186F2051196F1F4B202BE5EC9C
:107EE0002FF0211902E0D8901200222B050E2265F6
:107EF000E7D7D880050CE8CF15F10101176B166B99
:107F0000FBEC43F00101D8901737179103B61781A6
:107F1000162B1651800A780FF3E3155107E0000184
:107F20000398F0EC3FF001011751120000010388A3
:107F3000F8D786B611D000F086B60ED000F086B61F
:107F40000BD0010E0101016F690E006F54EC3DF082
:107F50003F2A050E416E050C2F0E0101016F100E18
:107F6000006F54EC3DF0010E3F6E010CE8CF1AF1AA
:107F7000010E196F1A51800A190F04E21A51800A72
:107F80001F0F0DE21A51800A390F04E21A51800ABC
:107F90003F0F05E21A511FEC45F0D8A0196B19C12B
:107FA00018F118311200636A626A9F0E5D6F5E6B92
:107FB0004D6B4E6BFB0E5C6F658C0401C46B040152
:107FC000C16B0401BD6B0401CD6B659C160E0F01E6
:107FD0004C6F02D06296040062B6FCD7659812001E
:107FE00096929690000103A809D0848284B209D0A9
:107FF0000101D36706D0020ED36F03D0000103A89E
:1080000084928D8000F08DB005D00101D36702D03D
:10801000010ED36F8D9012001B6BF2EC41F0186FC4
:108020001B511625196FE86A1BBFE86817211A6FE4
:1080300019C1D9FF1AC1DAFF18C1DFFF1B2B1B5171
:10804000800A790FEAE3F2EC41F000010992120094
:108050004F0E196FD40E186FE5EC2FF0216F4F0EF5
:10806000196FD50E186FE5EC2FF0226F2151246F98
:108070002251236F2051241902E11F51231902E1DB
:10808000D8801200D8901200E8CF15F115C1C2FFB8
:10809000C280190E0101166F160701011629FCE1B5
:1080A000C282320E166FC2A204D016070101162931
:1080B000FAE1C450FC0B166FC26A1651120000C1DF
:1080C000D9FF01C1DAFFDF50060A02E0D8901200A2
:1080D00020EE01F00051D9260151DA22180EDF629C
:1080E00005D002510C0A02E1D880120002510A0A9E
:1080F000FBE0ECD786969896080E416E412EFED78F
:108100009886280E416E412EFED786A603D0030125
:10811000F68F02D00301F69F010E0101016FA50E3B
:10812000006F54EC3DF03F2A1200849296928D80AD
:10813000969000F000F08DB005D00101D36702D019
:10814000010ED36F848200F000F084B205D00101EB
:10815000D36702D0040ED36F8D9000F0120017C1C8
:1081600018F1196B1551010B181BD89016331533E4
:1081700018A104D0010E151BA00E161BD8901833A1
:10818000192B070E1965EED715C115F116C116F199
:10819000070C1B6BF2EC41F0186F1B511625196F81
:1081A000E86A1BBFE86817211A6F19C1D9FF1AC105
:1081B000DAFF18C1DFFF1B2B1B51800A7B0FEAE39C
:1081C0000001099212001B6BF2EC41F0186F1B5179
:1081D0001625196FE86A1BBFE86817211A6F19C1C5
:1081E000D9FF1AC1DAFF18C1DFFF1B2B1B51800A10
:1081F0007E0FEAE30001099212006FEC44F00101E6
:10820000176F175111E0A098040E0401C86F300ECB
:10821000C76F15C1C9F416C1CAF417C1CBF477EC06
:108220003DF0A0888AEC45F00101175112001B6B4C
:10823000F2EC41F0186F1B511625196FE86A1BBF4D
:10824000E86817211A6F19C1D9FF1AC1DAFF18C1DE
:10825000DFFF1B2B1B51800A7D0FEAE3000109920F
:1082600012000101206B1EC117F11FC118F1EF0EA2
:1082700001012025D96EDA6A030EDA22DF50196F68
:10828000D6EC36F001011E4B1F2B202B060E20656D
:10829000EAD7060C3C6B3D6B8C0E3F6FE80E3E6FD1
:1082A000010E3B6F380E3A6F010E226F3C0E216FAC
:1082B00036C123F137C124F1010E266F3A0E256F26
:1082C0001FEFBFF0E8CF15F1000E4224D96EDA6A35
:1082D0000D0EDA2215C1DFFF422A4250F00AD8B44F
:1082E000426A0001FB2BFB51F00AD8A412000001E6
:1082F00009821200010E01011F6F7F0E01011F256F
:10830000D96EDA6A060EDA22960E1F25186F196BDF
:10831000020E1923E5EC2FF0DF6E1F2B0F0E1F65E9
:10832000ECD70F0CE8CF18F10101185103E01851F8
:10833000050A02E1D890120018C116F1FF0E1627A7
:1083400015C117F1162B02D0D8901733162FFCD772
:108350001731120002510E0A02E0D890120000C13B
:10836000D9FF01C1DAFF070EDF6401D0F6D720EE96
:1083700001F00051D9260151DA22010EDF62EDD75A
:10838000D880010CE8CF1FF01FC0C2FFC280190EB9
:10839000206E20062028FDE1C282320E206EC2A28D
:1083A00003D020062028FBE1C450FC0B206EC26ADB
:1083B00020501200E8CF1FF0000E4224D96EDA6A76
:1083C0000D0EDA221FC0DFFF422A4250F00AD8B455
:1083D000426A0001FB2BFB51F00AD8A412000001F5
:1083E00009821200000E0201D325D96EDA6A0D0E41
:1083F000DA22DF500101156F0201D32BD351F00AAD
:10840000D8B4D36B0001FB07FB6701D00E940101C8
:108410001551120002510B0A02E0D890120000C15F
:10842000D9FF01C1DAFFDF504E0AF7E120EE01F07B
:108430000051D9260151DA22DF50610AEEE1D880DD
:10844000120002510D0A02E0D890120000C1D9FFBB
:1084500001C1DAFFDF504E0AF7E120EE01F00051D2
:10846000D9260151DA22DF50620AEEE1D8801200EB
:10847000175115C1D9FF16C1DAFFDF6205D015C14A
:1084800015F116C116F1120015C1D9FF16C1DAFF98
:10849000154B162BDF50ECE1156B166B1200E8CF75
:1084A0001AF1185104EC39F015C11BF116C11CF179
:1084B0001A51020DF3501B25D96E000E1C21DA6EE5
:1084C000DECF18F1DDCF19F11200196B1A6B15A16F
:1084D00004D01751192718511A23D8901737183775
:1084E000D8901633153316511511F1E119C115F154
:1084F0001AC116F11200E8CF15F115514F0A04E127
:1085000015C1C5F2D890120015514B0A07E10201BE
:10851000C5514F0A03E1C56BD88012000201C56B3B
:10852000F1D7000109B212000101186B185116258C
:10853000D96E000E1721DA6EDF5062EC41F00101B6
:10854000182B070E1865F2D700010E84070C8B92CA
:10855000030E5DEC46F0010118515DEC46F001019F
:1085600017515DEC46F016515DEC46F0000E5DECE7
:1085700046F01A6F8B821A511200E8CF15F115518F
:108580000D0A04E115C1C4F2D890120015510A0A6F
:1085900007E10201C4510D0A03E1C46BD880120047
:1085A0000201C46BF1D7E8CF37F10101370508E1CB
:1085B000F90E166F930E156F0A0E176F60EF45F0E8
:1085C000F90E2C6F930E2B6F2E6B0A0E2D6F05EF8D
:1085D00006F0236A246A1FA004D0215023262250CB
:1085E0002422D89021362236D89020321F322050B3
:1085F0001F10F1E123C01FF024C020F01200E8CFCB
:1086000037F10101370508E1FA0E166FAE0E156F4E
:10861000090E176F60EF45F0FA0E2C6FAE0E2B6F40
:108620002E6B090E2D6F05EF06F0000109B2120046
:1086300020C0D9FF21C0DAFFDF50DAEC41F020EE94
:1086400001F02050D9262150DA22DF50DAEC41F037
:1086500000010E841200E8CF37F10101370508E16F
:10866000FB0E166FC10E156F080E176F60EF45F009
:10867000FB0E2C6FC10E2B6F2E6B080E2D6F05EFAE
:1086800006F08D9096908482969200F08D8000F096
:1086900000F08DB005D00101D36702D0010ED36F79
:1086A000849200F000F000F08D9000F01200E8CF0E
:1086B00037F10101370508E1F90E166F9E0E156FAF
:1086C0000A0E176F60EF45F0F90E2C6F9E0E2B6FA0
:1086D0002E6B0A0E2D6F05EF06F0F29210A003D05C
:1086E0001090F19C8A8210A206D01092F19C000199
:1086F00010BA8A8212008A92010E0101D86F00011D
:108700000F8A010C0101D76706D0010ED76F0A88C6
:108710000201EF6B1200D70506E1020ED76F0201CE
:10872000EF6BEE6B1200D76B00010B86120000019D
:108730000BA40CD00201DA51D8A4DA07DA671200D0
:1087400020EC46F0320EDA6FD82B320CFDECF5F04F
:108750000201D86B1200040124510F0B080D000E0A
:10876000F3240401C76FC86B040EC823040124AFAF
:108770001200040E0401C727000EC823000C0001DC
:1087800008BA050C000115B2050CFF0E01012C6F93
:10879000E10E2B6F000E2E6B2D6B05EC06F001E247
:1087A000000C27EF0EF0E8CF17F1010E166F1751EE
:1087B000200A09E01751800A720F04E21751800A5B
:1087C000770FD8A0166B16C115F1153112008B92D8
:1087D000020E5DEC46F0010118515DEC46F001011E
:1087E00017515DEC46F016515DEC46F01A515DEC08
:1087F00046F08B82120096829690000103968D803F
:1088000000F08DB005D00101D36702D0010ED36F07
:1088100000F084A202D0000103868D9012000401B2
:1088200024510F0B080D000EF3240401C76FC86B11
:10883000040EC823040124AF1200040E0401C7274C
:10884000000EC823000C1EC1CFF11FC1D0F1186B60
:10885000590E176F1F51196FD6EC36F00101186BC6
:108860005A0E176F1EC119F1D6EF36F0E8CF15F189
:108870000301A86BA96B000EA76F0A0EA66F00017B
:108880001D9C9EB803D000011DACFBD715C1AEFFE7
:108890001200E8CF21F0206A090E216405D0202AB9
:1088A0000A0E215E2160FBD721C01FF00F0E1F169C
:1088B0002038F00B1F101200E8CF15F10301A86B50
:1088C000A96B000EA76F0A0EA66F00011D9CA4B82D
:1088D00003D000011DACFBD715C1A9FF1200040194
:1088E00018BF000C200E0401CD6101D0000CA0A81F
:1088F000000C0401196703D08AEC45F0000C040158
:108900001951120086969896080E416E412EFED798
:108910000301EFB19886010E0101016F870E006F10
:1089200054EC3DF03F2A1200E8CF15F1600E010132
:10893000156503D01551A90F1200400E156503D01F
:108940001551C90F12001551D00F1200040118BFA4
:108950001200200E0401CD6101D0200CA0A812004D
:108960000401196702D097EF45F004011951120074
:108970009886080E416E412EFED7402E05D0400E3F
:10898000406E3F2A7AEF40F00301D890EF333F0664
:1089900082EF44F04F0E186FD40E176F1F51196FEE
:1089A000D6EC36F04F0E0101186FD50E176F1EC1B1
:1089B00019F1D6EF36F0DA2F1200FDECF5F0230EA8
:1089C0000301AC5D000EAD59320ED8B0FA0E0201B3
:1089D000DA6F010ED86F010CE8CF21F0206A215028
:1089E000800A460F06E22150800A500F02E3010E72
:1089F000206E20C01FF01F301200E8CF15F10F0EBF
:108A0000010115170A0E156104D0300E15271551F6
:108A10001200370E152701011551120019AA0CD0AA
:108A2000199A8B9C0CA604D0320E0201EF6F320C07
:108A30000F0E0201EF6F0F0C198A8B8CF3D7E8CF62
:108A400017F1166B1751800A460F06E21751800A7C
:108A5000500F02E3010E166F16C115F11531120009
:108A6000E8CF17F1166B1751800A250F06E2175150
:108A7000800A3F0F02E3010E166F16C115F1153182
:108A800012000201D86702D065EF46F0D80502E176
:108A900097EF43F0D851020A02E1DBEF44F0D86BC4
:108AA0001200FB0E0101176F8B0E166F010EA3EC67
:108AB00033F0130E01012A6F880E296FD8EF38F0BA
:108AC000AAEC46F00009FCE115C1B3F416C1B4F4F8
:108AD00017C1B2F4010E0401B16F010C90EC46F025
:108AE0007FEC2CF046ECB0F009EC1DF083ECE0F0EC
:108AF000168200011B821200E8CF68F1000113AC5E
:108B000007D00101680504E16EEC45F0D880120041
:108B1000D8901200400E0401181B040E1B6F300E7B
:108B20001A6F400E196F1817880E1813880C400E14
:108B30000401181B040E1B6F300E1A6F400E196FC4
:108B40001817880E1813880CE8CF15F11551800AF4
:108B5000250F05E21551800A3F0FD8B0158B15512E
:108B60001200E8CF15F11551800A050F05E21551E5
:108B7000800A1F0FD8B0159B155112000001FF513C
:108B8000D8A4FF07FF67120020EC46F0452A120E1A
:108B9000FF6F120CE8CF27F027AA03D0206A900EAF
:108BA00002D0206A920E1F6E91EF1BF00001FF5160
:108BB000D8A4FF07FF67120020EC46F04506640EBC
:108BC000FF6F640C869698960B0E0101016FC40E20
:108BD000006F54EC3DF03F2A12000201D76702D02B
:108BE0004DEF46F0D70502E155EF46F0D76B120086
:108BF0000001FF2F41EF45F0FDECF5F0456A020161
:108C0000D76B41EF45F098862F0E0101016F100ED2
:108C1000006F54EC3DF03F2A12009886010E0101CE
:108C2000016F870E006F54EC3DF03F2A1200F09266
:108C30005E0E776E786AA496A386000116841200F1
:108C4000AA0ECB6E550EBC6ECC6ACA843F0EBB6EAC
:108C50003F0CE8CF15F1010115A902D0D880120010
:108C6000D89012000401D56B0401CC9FA2883FEC80
:108C70003FF07CEFEFF0A0B8A1A8120026ECEDF0D9
:108C8000A6EC44F0A19812000001FF2F1200FDECA9
:108C9000F5F0452A090EFF6F090C00010AAC12001D
:108CA00020EC46F00201D72B120000010ABC120092
:108CB000FDECF5F00201D76B1200E8CF15F115C1FC
:108CC000C9FFC7A0FED7C95012000BA4EDEF45F0B5
:108CD000320E0201DA6FD82B320CE8CF15F1010108
:108CE00015510001FA1B1200E8CF15F115C1AEFFB6
:108CF000ADB21200FDD7ABECEAF0AEC329F1AFC3C1
:108D00002AF11200400E04011C1B1C17880E1C13B4
:108D1000880C000105B202D0D8901200D880120051
:108D2000139C1B920301CD6B00011A9C1200400E94
:108D300004011C1B1C17880E1C13880C17C1F8FF9C
:108D400016C1F7FF15C1F6FF1200E8CF15F115C1E6
:108D5000F5F01200A0A8010C0401B1511200059217
:108D60000001F95112000301AE6BAF6B1200FFFF5F
:108D7000FFFFFFFFFFFFFFFFFFFFFFFFFFFFFFFF03
:108D8000FFFFFFFFFFFFFFFFFFFFFFFFFFFFFFFFF3
:108D9000FFFFFFFFFFFFFFFFFFFFFFFFFFFFFFFFE3
:108DA000FFFFFFFFFFFFFFFFFFFFFFFFFFFFFFFFD3
:10EAB000FFFFFFFFFFFFFFFF30352F30312F3031D9
:10EAC0002C30303A30303A30300051495552433AC8
:10EAD0002022636C6F7365642200434D53204552BE
:10EAE000524F523A2031393300434D532045525250
:10EAF0004F523A2035313500434D45204552524F53
:10EB0000523A20313300434D45204552524F523A3C
:10EB10002031310051495552433A202272656376C3
:10EB20002200434F4E4E454354204641494C00512C
:10EB3000534D54505055543A202D0001000A0064A2
:10EB400000E80310274353513A20302C3000435241
:10EB5000494E473A2000434D54493A20004352451C
:10EB6000473A2000434C4F53454400735F6C6F633A
:10EB70006B002B43504252002B43504257002B4313
:10EB80004D4752002241434B22000902430002013B
:10EB900000C0640904000001020200000524001006
:10EBA00001042402020524060001052401000107D6
:10EBB00005820308000209040100020A00000007A0
:10EBC0000503024000010705830240000112011005
:10EBD0000102000008D8040A000100000000012B17
:10EBE000514654504346473D226163636F756E74CE
:10EBF000222C22636F72746578757064617465226B
:10EC00002C2242647467246664764B220D00432FE5
:10EC100025642E466C617368696E672120446F6EAF
:10EC2000277420706F776572206F6666210D0A0069
:10EC30002B514654504F50454E3D227570646174BF
:10EC4000652E636F727465782E6C76222C32310DCE
:10EC5000002B514655504C3D227570646174652EF1
:10EC6000686578222C3336353030302C350D002B4A
:10EC7000515552434346473D22757263706F72741B
:10EC8000222C227561727431220D00446F776E6CF4
:10EC90006F61646564207375636365737366756C17
:10ECA0006C792E0D0A002E686578222C2255465369
:10ECB0003A7570646174652E686578222C300D0099
:10ECC000436F6D6D616E64206E6F74206176616953
:10ECD0006C61626C652E0D0A005570677261646923
:10ECE0006E672E2E2E506C65617365207761697496
:10ECF0002E002B51534D54504346473D22736D74A3
:10ED000070736572766572222C22002B5143464740
:10ED10003D226E777363616E6D6F6465222C302CBB
:10ED2000310D002B514654504346473D22636F6ED0
:10ED3000746578746964222C320D002B5149434666
:10ED4000473D227064702F7265747279222C302CCA
:10ED5000310D002B51494346473D227064702F729C
:10ED600065747279222C312C310D002B51534D5486
:10ED7000504346473D22636F6E7465787469642220
:10ED80002C3100465450206469726563746F727947
:10ED9000206572726F722E0D0A00556E706C756769
:10EDA0002074686520555342206361626C650D0ACA
:10EDB000002B43504D533D22534D222C22534D22C4
:10EDC0002C22534D220D00555047524144453A489C
:10EDD00045582053495A45204552523B002B515328
:10EDE0004D54504346473D226163636F756E7422F4
:10EDF0002C22002B51534D54504346473D227373F0
:10EE00006C74797065222C3000446F776E6C6F6182
:10EE100064696E67206572726F722E0D0A002B5145
:10EE20004644454C3D227570646174652E68657872
:10EE3000220D002B4347514D494E3D312C302C3093
:10EE40002C302C302C300D002B4347515245513D76
:10EE5000312C302C302C302C302C300D002B5153D9
:10EE60004D54504346473D2273656E646572222CB3
:10EE700022002B51494F50454E3D312C312C22540C
:10EE80004350222C220046545020736572766572DE
:10EE9000206572726F722E0D0A0023343A303230C0
:10EEA00030303030323030303046430D0A00495374
:10EEB00020414C5245414459204C4F434B45440D51
:10EEC0000A002B51494F50454E3D312C302C2254D5
:10EED0004350222C22004469726563746F7279205A
:10EEE0006572726F722E0D0A002B51495552433ACA
:10EEF000202272656376222C302C005149555243F2
:10EF00003A202272656376222C312C330023343A66
:10EF1000303030303030303146460D0A0D0A004D69
:10EF20006F64656D206572726F7220302E2E0D0A2F
:10EF3000004D6F64656D206572726F7220312E2EE8
:10EF40000D0A004D6F64656D206572726F7220321C
:10EF50002E2E0D0A004D6F64656D206572726F7202
:10EF600020332E2E0D0A00555047524144453A4851
:10EF7000455820455252313B005550475241444577
:10EF80003A48455820455252333B0055504752416C
:10EF900044453A54494D452D4F55543B002B43476A
:10EFA00044434F4E543D312C224950222C22002BF9
:10EFB000434E4D493D322C312C302C302C300D003D
:10EFC0002B43434C4B3D2230302F30312F30312CEE
:10EFD0000053544154453A20434F4E4E4543544507
:10EFE00044005761697420666F72206865782E2E20
:10EFF0000D0A0046696E616C2076657273696F6EEA
:10F000002E0D0A002B514654504357443D22475081
:10F010003531220D002B514654504745543D22476F
:10F02000505F46353100554E53454E545F4255466C
:10F030005F46554C4C0D0051495552433A202272BF
:10F04000656376222C300051495552433A20227292
:10F05000656376222C31004350494E3A204E4F547E
:10F0600020494E534552004350494E3A204E4F548A
:10F070002052454144590053494D5320554E4C4F61
:10F08000434B45440D0A002B514654504745543DCF
:10F090002247505F353100555047524144453A436D
:10F0A00053204552523B0030362C25732C383430D7
:10F0B0003939303025640030372C25732C38343002
:10F0C0003939303025640030362C25732C383431F2
:10F0D0003939303025640030372C25732C383431E1
:10F0E0003939303025640030362C25732C383538CA
:10F0F000393930302564002B51534D54504453540A
:10F100003D312C312C2200434D45204552524F5267
:10F110003A20313030004845582053495A4520455F
:10F1200052520D0A002B514654504E4C53543D221E
:10F130002E220D005465737454696D653A20256460
:10F140002C200030362C25732C38353039393030AE
:10F15000300030372C25732C383530393930303089
:10F160000030362C25732C383031393930303000AE
:10F1700030362C25732C383231393930303000306C
:10F18000362C25732C383232393930303000303754
:10F190002C25732C38323239393030300030362C4F
:10F1A00025732C38323339393030300030362C2545
:10F1B000732C38303439393030300030362C2573E8
:10F1C0002C38323439393030300030372C25732C1C
:10F1D00038303839393030300030362C25732C38FF
:10F1E000323939393030300030372C25732C3832F1
:10F1F0003939393030300030362C25732C383333E0
:10F2000039393032300030372C25732C38333339CC
:10F21000393032300030362C25732C3833303939C0
:10F220003030310030372C25732C383330393930B9
:10F2300030310030362C25732C38303239393030AB
:10F24000310030372C25732C383032393930303199
:10F250000030362C25732C383534393930303100B4
:10F2600030362C25732C3835353939303031003073
:10F27000372C25732C38353539393030310030365C
:10F280002C25732C38333039393030320030372C5C
:10F2900025732C38333039393030320030362C2554
:10F2A000732C38303239393030320030372C2573F6
:10F2B0002C38303239393030320030362C25732C2E
:10F2C00038353439393030320030362C25732C380B
:10F2D000353539393030320030372C25732C3835FC
:10F2E0003539393030320030362C25732C383330F4
:10F2F00039393030330030372C25732C38333039DE
:10F30000393030330030362C25732C3835343939C8
:10F310003030330030362C25732C383330393930C7
:10F3200030340030372C25732C38333039393030B5
:10F33000340030362C25732C38353439393030349C
:10F340000030362C25732C383330393930303500C5
:10F3500030372C25732C3833303939303035003084
:10F36000362C25732C38333039393030360030376D
:10F370002C25732C38333039393030360030362C68
:10F3800025732C38343039393025640030372C253A
:10F39000732C38343039393025640030362C2573DD
:10F3A0002C38343139393025640030372C25732C12
:10F3B00038343139393025640030362C25732C38F7
:10F3C00035383939302564002B51464C44533D22A1
:10F3D000554653220D00514654504F50454E3A2049
:10F3E000302C300051534D54505055543A20302C4D
:10F3F0003000434D45204552524F523A20313000A3
:10F400004350494E3A2053494D2050494E004970CF
:10F410005254696D653A25646D2C20004155544F56
:10F4200020555047524144453A002B5149444E53D0
:10F430004346473D312C22002B435343533D224941
:10F440005241220D0051534D5450424F44593A20DD
:10F450002D0051465450434C4F53453A20300051F3
:10F46000534D5450424F44593A203100434F4E4E71
:10F47000454354204641494C00762E25645F6D6F0C
:10F480006465300D0A00762E25645F6D6F6465310A
:10F490000D0A00484558205752204552520D0A0087
:10F4A0005349412049503A4F46462C20004770723C
:10F4B000734174743A25642C20004F4E2C28256427
:10F4C0002064617973290030362C25303364393952
:10F4D0003030300030372C2530336439393030301B
:10F4E0000030362C3834303939303025640030372C
:10F4F0002C3834303939303025640030362C3834EB
:10F50000313939303025640030372C3834313939CD
:10F51000303025640030362C3835383939303025D4
:10F520006400222C22382E382E382E38220D002B43
:10F53000514953454E443D302C300D002B4950521B
:10F540003D31393230300D002B434F50533D342C78
:10F55000302C22002B5149434C4F53453D310D0077
:10F5600031363030203939203030300031333031CD
:10F5700020393920303030003333303120393920D0
:10F5800030303000313330322039392030303000E3
:10F590003333303220393920303030003136303298
:10F5A0002039392030303000313339332039392097
:10F5B00030303000313134302039392030303100B2
:10F5C000333134302039392030303100313134306A
:10F5D000203939203030320033313430203939206D
:10F5E000303032003131343020393920303033007E
:10F5F00033313430203939203030330051494F50C5
:10F60000454E3A20302C300051494F50454E3A205B
:10F61000312C300051494E49535441543A20320064
:10F6200051494F50454E3A20302C350051494E49F2
:10F63000535441543A2037004350494E3A205245E2
:10F64000414459004953204C4F434B45440D0A0057
:10F650002B514944454143543D320D002B514654F2
:10F6600050434C4F53450D00537461794128256434
:10F67000292C20005349412049503A4F4E2C20005C
:10F680005154696D653A2564732C20004E6F2055E6
:10F690007067726164652E0030362C383530393928
:10F6A0003030300030372C38353039393030300098
:10F6B00030362C38303139393030300030362C3853
:10F6C000323139393030300030362C383232393935
:10F6D0003030300030372C38323239393030300069
:10F6E00030362C38323339393030300030362C381F
:10F6F000303439393030300030362C383234393902
:10F700003030300030372C38303839393030300034
:10F7100030362C38323939393030300030372C38E7
:10F72000323939393030300030362C3833333939CA
:10F730003032300030372C38333339393032300002
:10F7400030362C38333039393030310030372C38BE
:10F75000333039393030310030362C3830323939A5
:10F760003030310030372C383032393930303100D8
:10F7700030362C38353439393030310030362C3889
:10F78000353539393030310030372C383535393965
:10F790003030310030362C383330393930303200A7
:10F7A00030372C38333039393030320030362C385D
:10F7B000303239393030320030372C383032393944
:10F7C0003030320030362C38353439393030320070
:10F7D00030362C38353539393030320030372C3826
:10F7E000353539393030320030362C38333039390C
:10F7F0003030330030372C38333039393030330043
:10F8000030362C38353439393030330030362C38F6
:10F81000333039393030340030372C3833303939DF
:10F820003030340030362C3835343939303034000B
:10F8300030362C38333039393030350030372C38C9
:10F84000333039393030350030362C3833303939AF
:10F850003030360030372C383330393930303600DC
:10F86000555047524144453A4F4B3B0030362C38B7
:10F87000343039393025640030372C383430393958
:10F880003025640030362C38343139393025640065
:10F8900030372C38343139393025640030362C3843
:10F8A0003538393930256400466F7263654F6666B6
:10F8B0003A2564002B514944454143543D310D00E4
:10F8C0002B5149444E534346473D22002B51494357
:10F8D0005347503D312C33002B4346554E203D209D
:10F8E000310D002B5149435347503D310D002B43FF
:10F8F00056455253494F4E0D002B51494E495354D2
:10F9000041540D0051534D54505055543A2000511C
:10F910004654504357443A203000514654504745CE
:10F92000543A20300043475245473A20312C3000AA
:10F9300043475245473A20312C310043475245470F
:10F940003A20312C320043475245473A20312C337C
:10F950000043475245473A20312C34004347524533
:10F96000473A20312C3500434F4E4E454354204FEB
:10F970004B0048455820455252310D0A0048455821
:10F9800020455252330D0A0049532057524F4E47DB
:10F990000D0A00434F4445204552520D0A0053546E
:10F9A0004154204552520D0A000D0A474320762546
:10F9B000640D0A002B514654504745543D220050D7
:10F9C0004F5254313A25732C2000504F5254323A42
:10F9D00025732C2000504F5254333A25732C2000AD
:10F9E0007374616E646172742C200064696769705D
:10F9F0006C65782C20002B514953454E443D300D09
:10FA0000002B51534D5450434C520D002B51495330
:10FA1000454E443D302C002B514953454E443D3119
:10FA20002C002B43475245473D310D002B514E577B
:10FA3000494E464F0D002241444D2D43494422007A
:10FA4000514453494D3A20302C00514453494D3ACA
:10FA500020312C00435245473A20312C300043528C
:10FA600045473A20312C3100435245473A20312C4A
:10FA70003200435245473A20312C33004352454728
:10FA80003A20312C3400435245473A20312C35007E
:10FA9000514654504E4C53543A00434D4520455224
:10FAA000524F5200434D53204552524F5200434F44
:10FAB0004445204F4B0D0A00484558204552520DF1
:10FAC0000A00526573746172740D0A002B5149412A
:10FAD00043543D320D0047454E4552414C2C2000C9
:10FAE000554E4B4E4F574E2C2000424154204C4F08
:10FAF000572C20006D6167656C616E2C2000756E5F
:10FB00006B6E6F776E2C2000536563757269747924
:10FB10003A002B51504F57443D310D002B51494174
:10FB200043543D310D002B43474154543D310D00AA
:10FB300053454E44204641494C002B435344483DD5
:10FB4000300D002B434F50533D300D002B434D459E
:10FB5000453D310D002B435245473D310D002B43B0
:10FB60004C49503D310D002B43545A553D330D0047
:10FB70002B43475245473F0D0049443A2564200D29
:10FB80000A002B434D47463D300D002B434D474661
:10FB90003D310D002B5149535441540D0043474111
:10FBA00054543A20300043475245473A20310043ED
:10FBB000474154543A2031004445414354204F4B6F
:10FBC000004545204552520D0A00435320455252EC
:10FBD0000D0A002B4346554E3D300D002A23736914
:10FBE0006D5F6730004546463646303846006674DD
:10FBF000705F6C6F6164004C4E723A25642C20007B
:10FC000053413A2025732C2000534D3A2025732C64
:10FC10002000534E3A2025732C200053503A2025C3
:10FC2000732C20004950313A25732C200049503262
:10FC30003A25732C20004950333A25732C2000417B
:10FC4000504E3A25732C2000444E533A25732C20F5
:10FC5000005757573A25732C2000657370726974EA
:10FC60002C20002843524547256420004347524535
:10FC700047256420004E6F5F436172642900536919
:10FC80006D4C6F636B3A0050616E537461743A004F
:10FC90006125732C25730D0A002B514453494D3FA8
:10FCA0000D002B43474154543F0D002B4352433D1D
:10FCB000310D002B435245473F0D002B434F50530E
:10FCC0003F0D002B51434349440D002B4350494EF7
:10FCD0003D22002B43434C4B3D2200302E302E3032
:10FCE0002E30003A757064617465002B43434C4BB1
:10FCF0003F0D002B434D47533D22000A303030303A
:10FD0000303000435041533A2030004346554E3A7C
:10FD1000203100434F4E4E45435400455252256416
:10FD200029200044282564292C200070616E656C10
:10FD30002C20004C3A2025732C20004F6E6C696EED
:10FD4000653A0047454E4552414C00554E4B4E4F8B
:10FD5000574E002B4350494E3F0D002B4346554E06
:10FD60003F0D00514953454E443A0053454E4420FF
:10FD70004F4B00286E756C6C29002B435355420D78
:10FD8000002B43494D490D002B4347534E0D002B8B
:10FD90005147534E0D002B43474D520D002B5147F9
:10FDA0004D520D002B435042523D002B434D4753C3
:10FDB0003D00434C49503A2000435042523A200003
:10FDC000434F50533A2000432F25640D0A00442826
:10FDD00031292C200053494D312C200064736331AC
:10FDE0002C2000647363322C200042454C4C2C20A4
:10FDF00000475052532C2000414F66662C20004D86
:10FE00004F66662C20004C3A25732C2000503A2572
:10FE1000732C2000616275732C2000563A25643BD8
:10FE20002000434D4525642000434D5325642000A8
:10FE300053494D313A280028636F64652900557392
:10FE40006572733A004143544956450030303031B1
:10FE50003030002B4353510D002B3038220D0075EC
:10FE6000706F6666002C3134352C002C3132392C01
:10FE7000002B434D474400224E414B220043535137
:10FE80003A200043434C4B3A00434D47533A00510C
:10FE9000434349440053494D31200053494D3220DA
:10FEA0000023343A3130006D6F646530006D6F644B
:10FEB0006531006D6F64653F006E636F646500724D
:10FEC000656465660073696D5F6C00736669726D69
:10FED000002825642920002F256429200047534D40
:10FEE0002C2000414F6E2C20004D4F6E2C200028FE
:10FEF000747874290053494D313A004F5554313AC2
:10FF0000004F5554323A004D6F64653A00524543F4
:10FF10004F4E0053494D455200534D534552004DED
:10FF20003A202573002B434D450075706F6E0051CC
:10FF300047534E0033334343006C74616200737463
:10FF4000616200252E3264006C636667007363662D
:10FF500067006C6C6F67006C746D70006C74787403
:10FF60000073747874006E782C200025733B200099
:10FF70002F256429004F55543A002573293B004E24
:10FF80004F4E450047505253004441595300475289
:10FF90005354004D525354003030303800524459BD
:10FFA0000045310D004F4E2F004950310020553192
:10FFB000004950320020553200205533002055347E
:10FFC00000494E3A004F4646004255460047534DC1
:10FFD0000045525200444E5300282564002F2564EA
:10FFE00000510D0A00480D005530004C3000222C05
:10FFF0000039310041310023005B007C003E0000ED
:020000040001F9
:100000000101976B5F51156F030E6015166F186B2A
:100010000E0E176F65EC42F0040E15259A6F040E54
:1000200016219B6F6051996F9941E8423F0B070B76
:10003000996F9AC11FF19BC120F10CEC31F001E2E4
:10004000000C13AC03D00101990523E01EAA04D0D3
:1000500001019951030A1DE0370EAE6E010199515D
:100060008DECDAF0EDE3380EAE6E1EC597F19E6BA7
:100070000BD000EC8EF0650E9E25E16EE26A010E5B
:10008000E222DFCFE7FF9E2B05011E5101019E5D9D
:10009000F0E3C1054EE160AF34D00501ACEC8DF06A
:1000A00098EC8DF0310EDF6E9E2B1F0E73EC8DF0F1
:1000B0005AEC8DF0616F61390F0BFDEC44F0DF6E8F
:1000C0009E2B5AEC8DF00F0BFDEC44F0E2EC8DF022
:1000D0009D65EED71F0E69EC8DF01F0E9E257EEC00
:1000E0008DF0FDEC44F08CEC8DF0FDEC44F0DF6E17
:1000F0009E2B9E51CAECF1F0D8EC8DF036EC22F03C
:1001000015D00501D48117A409D0010E01011E6F7D
:10011000000E8FEC0CF016EC8EF002D001019E6BFD
:100120009E5190ECE3F002E20101996B01019951BB
:100130001200C151020A4FE160AF3AD00501ACECA8
:100140008DF098EC8DF0320EDF6E9E2B1F0E73EC4F
:100150008DF05AEC8DF0616F61390F0BFDEC44F0BE
:10016000DF6E9E2B5AEC8DF00F0BFDEC44F0E2ECB1
:100170008DF09D65EED71F0E69EC8DF0030E9D6F1F
:100180005AEC8DF0616F61390F0BFDEC44F0DF6EBE
:100190009E2B5AEC8DF00F0BFDEC44F0DF6E9E2B86
:1001A0009D2B040E9D65ECD79E51CAECF1F0A4D7AF
:1001B0000501D48117A409D0010E01011E6F000EA4
:1001C0008FEC0CF016EC8EF002D001019E6B9E516C
:1001D00090ECE3F0A8D7C151030A4FE160AF3AD0E9
:1001E0000501ACEC8DF098EC8DF0330EDF6E9E2B9C
:1001F0001F0E73EC8DF05AEC8DF0616F61390F0BAF
:10020000FDEC44F0DF6E9E2B5AEC8DF00F0BFDECF5
:1002100044F0E2EC8DF09D65EED71F0E69EC8DF099
:10022000030E9D6F5AEC8DF0616F61390F0BFDEC81
:1002300044F0DF6E9E2B5AEC8DF00F0BFDEC44F07A
:10024000DF6E9E2B9D2B050E9D65ECD79E51CAEC53
:10025000F1F052D70501D48117A409D0010E010194
:100260001E6F000E8FEC0CF016EC8EF002D0010128
:100270009E6B9E5190ECE3F056D7C151060A03E005
:10028000C151070A5CE160AF47D00501D46B0101A1
:100290009E6BC1390F0BFDEC44F005011F6F01018E
:1002A00098EC8DF0C1510F0BFDEC44F0DF6E9E2BEE
:1002B0001F0E69EC8DF0010E9D6F5AEC8DF0616F91
:1002C00061390F0BFDEC44F0DF6E9E2B5AEC8DF084
:1002D0000F0BFDEC44F0E2EC8DF09D65EED71F0EA8
:1002E00069EC8DF0030E9D6F5AEC8DF0616F6139F2
:1002F0000F0BFDEC44F0DF6E9E2B5AEC8DF00F0BD4
:10030000FDEC44F0DF6E9E2B9D2B060E9D65ECD719
:100310009E51CAECF1F0F0D60501D48117A409D0A2
:10032000010E01011E6F000E8FEC0CF016EC8EF02A
:1003300002D001019E6B9E5190ECE3F0F4D6C129EE
:1003400001E07ED6C4C1DBF1C451190A09E0C451F1
:10035000200A06E0C451210A03E0C451220A30E118
:100360000501D46B010E01019D6FC451200A02E109
:10037000020E9D6FC451210A02E1030E9D6FC4510C
:10038000220A02E1040E9D6F9D518DECDAF001E22C
:1003900057D69E6B07D000EC8EF01F0E9E258EEC7C
:1003A0000EF09E2B05011E5101019E5DF4E31F0E10
:1003B0009E25D96EDA6A050EDA22DF6A32EF8DF0F9
:1003C000C451810A0AE10501B4EC8DF0EC0E396FDD
:1003D000D90E386F30EC3DF00CD0C451820A0DE1DB
:1003E0000501B4EC8DF0F60E396F8C0E386F30ECE1
:1003F0003DF036519D6F32EF8DF0C4518A0A01E015
:100400000DD10501D46B050E0101A0EC8DF030EC8F
:100410003DF036519D6F9DC19EF11DBE23D001015F
:100420009C6B85EC8DF0CD0E9C25186F196B000E22
:100430001923E5EC2FF0DF6E85EC8DF0DF5004E042
:100440009C2B0F0E9C65EDD71F0E4DEC8DF0FC0E16
:10045000396F240E386F010E3B6F770E3A6F30EC18
:100460003DF01ED01F0E4DEC8DF0FC0E396F510E7D
:10047000386F070E3B6F500E3A6F30EC3DF036513F
:100480009D6F9D519E271F0E4DEC8DF0FC0E396F18
:10049000480E386F070E3B6FAB0E3A6F30EC3DF0F5
:1004A00054EC8DF085EC8DF0C80E9C25186F196BFF
:1004B000000E1923E5EC2FF0DF6E85EC8DF0DF5098
:1004C00004E09C2B040E9C65EDD71F0E4DEC8DF0C7
:1004D000F90E396FBF0E386F010E3B6F770E3A6F12
:1004E00030EC3DF054EC8DF085EC8DF08A0E9C25BF
:1004F000186F196B010E1923E5EC2FF0DF6E85ECF8
:100500008DF0DF5004E09C2B0F0E9C65EDD71F0E85
:100510004DEC8DF0FC0E396F2D0E386F010E3B6FD8
:10052000770E3A6F30EC3DF054EC8DF085EC8DF0A9
:10053000850E9C25186F196B010E1923E5EC2FF021
:10054000DF6E85EC8DF0DF5004E09C2B040E9C6583
:10055000EDD71F0E4DEC8DF0F90E396FCA0E386FC6
:10056000010E3B6F770E3A6F30EC3DF054EC8DF09E
:1005700085EC8DF00FEC8EF0E5EC2FF0DF6E85EC66
:100580008DF0DF5004E09C2B0F0E9C65F1D71F0E01
:100590004DEC8DF0FC0E396F360E386F010E3B6F4F
:1005A000770E3A6F30EC3DF054EC8DF085EC8DF029
:1005B00008EC8EF0E5EC2FF0DF6E85EC8DF0DF506F
:1005C00004E09C2B040E9C65F1D71F0E4DEC8DF0C2
:1005D000F90E396FD50E386F010E3B6F770E3A6FFB
:1005E00030EC3DF036519D6F9D519E27196B750E75
:1005F000186FE5EC2FF09D6FD8909D33030E9D177B
:100600001F0E4DEC8DF0F80E396FA80E386F9DC19E
:100610003AF13B6B30EC3DF032EF8DF0C4518B0A78
:1006200001E011D10501D46B01019E6B050EA0EC18
:100630008DF030EC3DF036519D6F9D519E271F0E81
:100640004DEC8DF0F10E396F340E386FF2C23AF185
:100650003B6B30EC3DF036519D6F9D519E271F0E38
:100660004DEC8DF0F60E396F800E386FE1C23AF125
:100670003B6B30EC3DF036519D6F9D519E271F0E18
:100680004DEC8DF0F40E396F100E386FDDC13AF17C
:100690003B6B30EC3DF036519D6F9D519E271F0EF8
:1006A0004DEC8DF0F40E396F0E0E386FDEC23AF15C
:1006B0003B6B30EC3DF036519D6F9D519E271F0ED8
:1006C0004DEC8DF0F40E396FAD0E386FD5C33AF1A5
:1006D0003B6B30EC3DF036519D6F9D519E271EA621
:1006E0000AD01F0E4DEC8DF0F60E396F740E386F78
:1006F00030EC3DF009D01F0E4DEC8DF0F40E396F4B
:10070000A00E386F30EC3DF036519D6F9D519E2705
:100710001F0E4DEC8DF0FB0E396FF70E386FDCC1FC
:100720003AF13B6B30EC3DF036519D6F9D519E2769
:100730001F0E4DEC8DF0FE0E396FFB0E386F30EC56
:100740003DF036519D6F9D519E270CAA0ED01F0E75
:100750004DEC8DF0FA0E396FD60E386F30EC3DF05F
:1007600036519D6F9D519E272ED00DAE0AD01F0E83
:100770004DEC8DF0FE0E396FDD0E386F30EC3DF034
:10078000EFD70DA40AD01F0E4DEC8DF0FD0E396F82
:10079000F10E386F30EC3DF0E3D708AE0AD01F0EF3
:1007A0004DEC8DF0FD0E396FEA0E386F30EC3DF0F8
:1007B000D7D71F0E4DEC8DF0FA0E396FE00E386F63
:1007C00030EC3DF0CDD71F0E4DEC8DF0FF0E396FA4
:1007D000010E386F30EC3DF036519D6F9D519E27D4
:1007E0000CAC0FD01F0E4DEC8DF0FD0E396F430E8B
:1007F000386F30EC3DF036519D6F9D519E2732EFA2
:100800008DF00EA00AD01F0E4DEC8DF0FF0E396F4B
:10081000CD0E386F30EC3DF0EED70DA60AD01F0E8E
:100820004DEC8DF0FF0E396F840E386F30EC3DF0DB
:10083000E2D71F0E4DEC8DF0FD0E396F4B0E386F69
:1008400030EC3DF0D8D7C4518C0A01E06AD10501E3
:10085000D46B050E0101A0EC8DF030EC3DF036516B
:100860009D6F9DC19EF1500E196FEA0E186FE5EC59
:100870002FF0550A17E11F0E4DEC8DF0F80E396F71
:10088000600E386F30EC3DF036519D6F500E186F92
:10089000EA0E176F000E196BD6EC36F001019D5170
:1008A0009E275AD0500E196FEA0E186FE5EC2FF004
:1008B000430A0AE11F0E4DEC8DF0F00E396F970ED2
:1008C000386F30EC3DF0E0D7500E196FEA0E186F1C
:1008D000E5EC2FF0470A0AE11F0E4DEC8DF0EF0E0C
:1008E000396F670E386F30EC3DF0CED7500E196F70
:1008F000EA0E186FE5EC2FF0410A0AE11F0E4DECED
:100900008DF0EF0E396F790E386F30EC3DF0BCD7BB
:10091000500E196FEA0E186FE5EC2FF0530A0AE13A
:100920001F0E4DEC8DF0ED0E396FC70E386F30ECA9
:100930003DF0AAD7500E196FEA0E186FE5EC2FF0B4
:10094000540A0AE11F0E4DEC8DF0EF0E396F8B0E3D
:10095000386F30EC3DF098D71F0E4DEC8DF0FF0E48
:10096000396F6B0E386F070E3B6F9B0E3A6F30EC92
:100970003DF036519D6F9D519E271F0E4DEC8DF021
:10098000FF0E396F6B0E386F080E3B6FD20E3A6F49
:1009900030EC3DF036519D6F9D519E271F0E4DEC62
:1009A0008DF0FF0E396F6B0E386F070E3B6F8B0E9D
:1009B0003A6F30EC3DF036519D6F9D519E271F0ED2
:1009C0004DEC8DF0FE0E396F300E386F30EC3DF08F
:1009D00054EC8DF085EC8DF0ED0E9C25186F196BA5
:1009E000000E1923E5EC2FF0DF6E85EC8DF0DF5063
:1009F00004E09C2B080E9C65EDD71F0E4DEC8DF08E
:100A0000FE0E396F060E386F010E3B6F770E3A6F90
:100A100030EC3DF054EC8DF085EC8DF0F60E9C251D
:100A2000186F196B000E1923E5EC2FF0DF6E85ECC3
:100A30008DF0DF5004E09C2B080E9C65EDD71F0E57
:100A40004DEC8DF0FE0E396F0D0E386F010E3B6FC1
:100A5000770E3A6F30EC3DF054EC8DF085EC8DF074
:100A6000980E9C25186F196B000E1923E5EC2FF0DA
:100A7000DF6E85EC8DF0DF5004E09C2B1A0E9C6538
:100A8000EDD71F0E4DEC8DF0FC0E396F3F0E386F19
:100A9000010E3B6F770E3A6F30EC3DF054EC8DF069
:100AA0003C0E01019C25D96EDA6A070EDA22770E18
:100AB0009C25E16EE26A010EE222DFCFE7FF85ECC2
:100AC0008DF0DF5004E09C2B130E9C65E9D71F0EC0
:100AD0004DEC8DF0FF0E396F7A0E386F010E3B6FC3
:100AE000770E3A6F30EC3DF036519D6F010E1C6F62
:100AF000770E1B6FFA0E1E6F9E0E1D6F206B050E7C
:100B00001F6F0AEC28F01C511B1101E076D61F0E56
:100B10004DEC8DF0FC0E396F750E386F30EC3DF0FA
:100B20006AD6C4518D0A01E0C1D30501D46B050E0C
:100B30000101A0EC8DF030EC3DF036519D6F9DC170
:100B40009EF11F0E4DEC8DF0FF0E396F070E386FC2
:100B500030EC3DF036519D6F9D519E27E0670AD0E5
:100B60001F0E4DEC8DF0F90E396FE00E386F30EC42
:100B70003DF070D0E051080A0AE11F0E4DEC8DF0F7
:100B8000FE0E396F140E386F30EC3DF063D0E0513B
:100B9000040A0AE11F0E4DEC8DF0FC0E396F5A0E5F
:100BA000386F30EC3DF056D0E051060A0AE11F0ED6
:100BB0004DEC8DF0FA0E396FF40E386F30EC3DF0DD
:100BC00049D0E0510C0A0AE11F0E4DEC8DF0FD0EEC
:100BD000396FDC0E386F30EC3DF03CD0E051020A4A
:100BE0000AE11F0E4DEC8DF0FD0E396F2B0E386FA4
:100BF00030EC3DF02FD0E0510A0A0AE11F0E4DEC17
:100C00008DF0FD0E396FE30E386F30EC3DF022D0E1
:100C1000E0510E0A0AE11F0E4DEC8DF0F90E396F0E
:100C2000EB0E386F30EC3DF015D0E0050AE11F0EF9
:100C30004DEC8DF0FF0E396F660E386F30EC3DF0E5
:100C400009D01F0E4DEC8DF0FA0E396FFE0E386F85
:100C500030EC3DF036519D6F9D519E271F0E4DEC9F
:100C60008DF0FE0E396FF50E386F30EC3DF03651D9
:100C70009D6F9D519E2712AC0ED01F0E4DEC8DF036
:100C8000FF0E396F7F0E386F30EC3DF036519D6F9F
:100C90009D519E2716D018A40AD01F0E4DEC8DF042
:100CA000FF0E396FD10E386F30EC3DF0EFD71F0ECD
:100CB0004DEC8DF0FE0E396F450E386F30EC3DF087
:100CC000E5D71F0E4DEC8DF0FD0E396FD20E386F4B
:100CD00030EC3DF036519D6F9D519E271F0E4DEC1F
:100CE0008DF0F40E396F1C0E386F30EC3DF036513C
:100CF0009D6F9D519E2707A435D00301BA51010174
:100D0000616F0301BB510101626F636B646B6151E1
:100D1000C008156FA80E6255166F000E6355176F49
:100D2000000E6455186FA00E196F050E1A6F000E95
:100D30001B6B1C6BEFEC1BF015C175F116C176F146
:100D40001F0E4DEC8DF0F40E396FBA0E386F75C171
:100D50003AF176C13BF130EC3DF036519D6F9D513B
:100D60009E270AD01F0E4DEC8DF0FF0E396FC50E79
:100D7000386F30EC3DF0F1D71F0E4DEC8DF0FD0ECD
:100D8000396FD20E386F30EC3DF036519D6F9D516A
:100D90009E271F0E4DEC8DF0FF0E396FC10E386F80
:100DA00030EC3DF036519D6F9D519E27E6A10DD050
:100DB0001F0E4DEC8DF0FB0E396FAD0E386F30EC21
:100DC0003DF036519D6F9D519E27E6A30DD01F0E1D
:100DD0004DEC8DF0F60E396F1E0E386F30EC3DF095
:100DE00036519D6F9D519E27E6A50DD01F0E4DECEF
:100DF0008DF0FA0E396F7A0E386F30EC3DF03651C7
:100E00009D6F9D519E27E6A70DD01F0E4DEC8DF0D6
:100E1000FA0E396F840E386F30EC3DF036519D6F0D
:100E20009D519E27E6A90DD01F0E4DEC8DF0F60EBC
:100E3000396F2A0E386F30EC3DF036519D6F9D5161
:100E40009E271F0E4DEC8DF0FD0E396FD20E386FC0
:100E500030EC3DF036519D6F9D519E2707AC0DD073
:100E60001F0E4DEC8DF0FA0E396FEA0E386F30EC34
:100E70003DF036519D6F9D519E271F0E4DEC8DF01C
:100E8000FF0E396F750E386F30EC3DF036519D6FA7
:100E90009D519E278AAE0DD01F0E4DEC8DF0F60EA3
:100EA000396F1E0E386F30EC3DF036519D6F9D51FD
:100EB0009E278AAC0DD01F0E4DEC8DF0FB0E396FC6
:100EC000AD0E386F30EC3DF036519D6F9D519E2731
:100ED0001F0E4DEC8DF0FD0E396FD20E386F30ECD9
:100EE0003DF036519D6F9D519E2714A26BD01F0E71
:100EF0004DEC8DF0FC0E396F870E386F30EC3DF005
:100F000036519D6F9D519E2709A00DD01F0E4DECAF
:100F10008DF0FD0E396FEA0E386F30EC3DF0365132
:100F20009D6F9D519E270101196B540E186FE5ECC2
:100F30002FF0986F9851F00B0BE11F0E4DEC8DF0D8
:100F4000FD0E396F230EBBEC8DF030EC3DF036D04A
:100F50009851F00B100A0BE11F0E4DEC8DF0F60EC0
:100F6000396F6C0EBBEC8DF030EC3DF027D0985112
:100F7000F00B200A0BE11F0E4DEC8DF0FD0E396FCA
:100F8000230EBBEC8DF030EC3DF018D09851F00BF7
:100F9000300A0BE11F0E4DEC8DF0F60E396F680E26
:100FA000BBEC8DF030EC3DF009D01F0E4DEC8DF018
:100FB000FD0E396FCE0E386F30EC3DF036519D6F1F
:100FC0009D519E271F0E4DEC8DF0FE0E396F3E0E8B
:100FD000386F30EC3DF036519D6F9D519E27010ECC
:100FE0008DECDAF029E31F0E4DEC8DF0FF0E396F1A
:100FF000AD0E386F30EC3DF036519D6F9D519E2700
:10100000010EC3EC3EF000090AE11F0E4DEC8DF01D
:10101000FE0E396FEF0E386F30EC3DF009D01F0E29
:101020004DEC8DF0FE0E396F370E386F30EC3DF021
:1010300036519D6F9D519E27020E8DECDAF029E30B
:101040001F0E4DEC8DF0FF0E396FB50E386F30EC82
:101050003DF036519D6F9D519E27020EC3EC3EF030
:1010600000090AE11F0E4DEC8DF0FE0E396FEF0EF8
:10107000386F30EC3DF009D01F0E4DEC8DF0FE0EB8
:10108000396F370E386F30EC3DF036519D6F9D5102
:101090009E27030E8DECDAF029E31F0E4DEC8DF048
:1010A000FF0E396FB90E386F30EC3DF036519D6F41
:1010B0009D519E27030EC3EC3EF000090AE11F0E6E
:1010C0004DEC8DF0FE0E396FEF0E386F30EC3DF0C9
:1010D00009D01F0E4DEC8DF0FE0E396F370E386FB4
:1010E00030EC3DF036519D6F9D519E27040E8DECE6
:1010F000DAF029E31F0E4DEC8DF0FF0E396FBD0EB7
:10110000386F30EC3DF036519D6F9D519E27040E97
:10111000C3EC3EF000090AE11F0E4DEC8DF0FE0E0F
:10112000396FEF0E386F30EC3DF009D01F0E4DECEB
:101130008DF0FE0E396F370E386F30EC3DF03651C2
:101140009D6F9D519E271F0E4DEC8DF0FD0E396F4A
:10115000D20E386F30EC3DF036519D6F9D519E2779
:101160001F0E4DEC8DF0FB0E396F080E386F30EC12
:101170003DF036519D6F9D519E274F0E196FD30E36
:10118000186FE5EC2FF0616F61AD0AD01F0E4DECCA
:101190008DF0F60E396F7B0E386F30EC3DF009D0D4
:1011A0001F0E4DEC8DF0F40E396FA70E386F30EC3A
:1011B0003DF054EC8DF01F0E4DEC8DF0FC0E396FB0
:1011C0007E0E386F30EC3DF036519D6F9D519E275D
:1011D000000E1FEC09F000090FE01F0E4DEC8DF022
:1011E000FD0E396FD50E386F30EC3DF036519D6FE6
:1011F000010E9C6F9D519E2701019C6710D01F0E10
:101200009E25366F376B050E3723F40E396FA70E08
:10121000386F30EC3DF036519D6F9D519E271F0E6B
:101220004DEC8DF0FD0E396F3B0E386F30EC3DF01C
:1012300036519D6F9D519E2713AC23D01F0E4DEC50
:101240008DF0FF0E396FA50E386F30EC3DF0365142
:101250009D6F9D519E2709A60AD01F0E4DEC8DF063
:10126000FF0E396FB10E386F30EC3DF0FBD31F0E1F
:101270004DEC8DF0FF0E396FA90E386F30EC3DF05C
:10128000F1D316A00AD01F0E4DEC8DF0FF0E396F72
:101290000D0E386F30EC3DF0E5D31F0EFEDBFF0E78
:1012A000396FC50E386F30EC3DF0DCD3C4518E0A77
:1012B00001E0E4D00501D46B1EAA0CD0050E01019B
:1012C000376F1F0E366FFE0E396FE90E386F30EC38
:1012D0003DF00BD0050E0101376F1F0E366FFD0E6E
:1012E000396FFF0E386F30EC3DF036519D6F9DC168
:1012F0009EF19C6B85EC8DF00FEC8EF0E5EC2FF001
:10130000DF6E85EC8DF0DF5004E09C2B1F0E9C659A
:10131000F1D71F0EC2DBFC0E396F000E386F010EC5
:101320003B6F770E3A6F30EC3DF0BEDBEEDB08EC46
:101330008EF0E5EC2FF0DF6EE8DBDF5004E09C2B55
:10134000050E9C65F3D71F0EA8DBFC0E396F1B0E34
:10135000386F010E3B6F770E3A6F30EC3DF0A4DB37
:10136000D4DBC00E9C25186F196B010E1923E5EC18
:101370002FF0DF6ECADBDF5004E09C2B1F0E9C6554
:10138000EFD71F0E8ADBFD0E396F330E386F010E5B
:101390003B6F770E3A6F30EC3DF036519D6F9D51AB
:1013A0009E271EA809D01F0E78DBFE0E396FE30EB4
:1013B000386F30EC3DF008D01F0E6FDBFD0E396F3B
:1013C000F80E386F30EC3DF06FDB9FDBF10E9C25A3
:1013D000186F196B010E1923E5EC2FF0DF6E95DB0A
:1013E000DF5004E09C2B0F0E9C65EFD71F0E55DBE2
:1013F000FC0E396F120E386F010E3B6F770E3A6F8D
:1014000030EC3DF051DB81DB9C29186F196B020E2B
:101410001923E5EC2FF0DF6E78DBDF5004E09C2B26
:101420001F0E9C65F0D71F0E38DBFC0E396F090EBE
:10143000386F010E3B6F770E3A6F30EC3DF034DBC6
:1014400064DB210E9C25186F196B020E1923E5EC45
:101450002FF0DF6E5ADBDF5004E09C2B1F0E9C65E3
:10146000EFD71F0E1ADBFF0E396F1F0E386F010EFC
:101470003B6F770E3A6F30EC3DF0F4D2C4518F0AD7
:1014800001E069D20501D46B01019E6B050E376F37
:101490001F0E366FFF0E396F890E386F30EC3DF03E
:1014A00036519D6F9D519E27500E196FBF0E186FBC
:1014B000E5EC2FF0616F500E196FBE0E186FE5EC62
:1014C0002FF09B6F61519A6F1F0EE7DA5FDB30ECF4
:1014D0003DF036519D6F9D519E27500E196FC10EE4
:1014E000186FE5EC2FF0616F500E196FC00E186F7A
:1014F000E5EC2FF09B6F61519A6F1F0ECEDA4FDB38
:1015000030EC3DF036519D6F9D519E271F0EC5DA80
:10151000FF0E396FA90E386F30EC3DF036519D6FDC
:101520009D519E27500E196FC50E186FE5EC2FF0D8
:10153000616F500E196FC40E186FE5EC2FF09B6FA2
:1015400061519A6F1F0EA9DA21DB30EC3DF0365164
:101550009D6F9D519E27500E196FC30E186FE5ECBD
:101560002FF0616F500E196FC20E186FE5EC2FF05F
:101570009B6F61519A6F1F0E90DA28DB30EC3DF0C3
:1015800036519D6F9D519E27500E196FCB0E186FCF
:10159000E5EC2FF0616F500E196FCA0E186FE5EC75
:1015A0002FF09B6F61519A6F1F0E77DAF8DA30ECEB
:1015B0003DF036519D6F9D519E271F0E6EDAFF0E36
:1015C000396FB10E386F30EC3DF036519D6F9D5143
:1015D0009E27500E196FC90E186FE5EC2FF0616F42
:1015E000500E196FC80E186FE5EC2FF09B6F61510C
:1015F0009A6F1F0E52DACADA30EC3DF036519D6F09
:101600009D519E27500E196FC70E186FE5EC2FF0F5
:10161000616F500E196FC60E186FE5EC2FF09B6FBF
:1016200061519A6F1F0E39DAD1DA30EC3DF0365144
:101630009D6F9D519E27500E196FCD0E186FE5ECD2
:101640002FF0616F500E196FCC0E186FE5EC2FF074
:101650009B6F61519A6F1F0E20DAA1DA30EC3DF0DA
:1016600036519D6F9D519E271F0E17DAFF0E396F61
:10167000130E386F30EC3DF036519D6F9D519E2713
:10168000500E196FCF0E186FE5EC2FF0616F500EF2
:10169000196FCE0E186FE5EC2FF09B6F61519A6FAA
:1016A0001F0EFBD973DA30EC3DF036519D6F9D5122
:1016B0009E27500E196FD10E186FE5EC2FF0616F59
:1016C000500E196FD00E186FE5EC2FF09B6F615123
:1016D0009A6F1F0EE2D963DA30EC3DF036519D6F00
:1016E0009D519E271F0ED9D9FF0E396F190E386FE5
:1016F00030EC3DF036519D6F9D519E27500E196F75
:10170000E30E186FE5EC2FF0616F500E196FE20ECB
:10171000186FE5EC2FF09B6F61519A6F1F0EBDD9CA
:101720005EDA30EC3DF036519D6F9D519E271F0EC5
:10173000B4D9FF0E396FC90E386F30EC3DF0365119
:101740009D6F9D519E27500E196FE10E186FE5ECAD
:101750002FF0616F500E196FE00E186FE5EC2FF04F
:101760009B6F61519A6F1F0E98D939DA30EC3DF0BA
:1017700036519D6F9D519E271F0E8FD9FF0E396FD9
:101780008E0E386F30EC3DF036519D6F9D519E2787
:10179000500E196FDB0E186FE5EC2FF0616F500ED5
:1017A000196FDA0E186FE5EC2FF09B6F61519A6F8D
:1017B0001F0E73D9FC0E396F630E386F9AC13AF160
:1017C0009BC13BF130EC3DF036519D6F9D519E2702
:1017D000500E196FDD0E186FE5EC2FF0616F500E93
:1017E000196FDC0E186FE5EC2FF09B6F61519A6F4B
:1017F0001F0E53D9FC0E396F6C0E386F9AC13AF137
:101800009BC13BF130EC3DF036519D6F9D519E27C1
:10181000500E196FD70E186FE5EC2FF0616F500E58
:10182000196FD60E186FE5EC2FF09B6F61519A6F10
:101830001F0E33D9FE0E396F220E386F9AC13AF15E
:101840009BC13BF130EC3DF036519D6F9D519E2781
:10185000500E196FD90E186FE5EC2FF0616F500E16
:10186000196FD80E186FE5EC2FF09B6F61519A6FCE
:101870001F0E13D9FE0E396F290E386F9AC13AF137
:101880009BC13BF130EC3DF036519D6F9D519E2741
:10189000500E196FDF0E186FE5EC2FF0616F500ED0
:1018A000196FDE0E186FE5EC2FF09B6F61519A6F88
:1018B0001F0EF3D8FD0E396F1B0E386F9AC13AF127
:1018C0009BC13BF130EC3DF036519D6F9D519E2701
:1018D0001F0EE3D8FF0E396F930E386F30EC3DF0DA
:1018E00036519D6F9D519E27500E196FD30E186F64
:1018F000E5EC2FF0616F500E196FD20E186FE5EC0A
:101900002FF09B6F61519A6F1F0EC7D83FD930ECF3
:101910003DF036519D6F9D519E27500E196FD50E8B
:10192000186FE5EC2FF0616F500E196FD40E186F21
:10193000E5EC2FF09B6F61519A6F1F0EAED8FF0E32
:10194000396F700E386F9AC13AF19BC13BF130ECA0
:101950003DF0FBEF83F00201F55129E0360EAE6E4B
:101960000101C451260A09E0C451270A06E0C45106
:10197000280A03E0C451290A75E10201F50506E1D0
:10198000050E010135D930EC3DF00ED0F551020ABB
:101990000BE1050E0101376F1F0E366FFA0E396F1E
:1019A0009E0E386F30EC3DF00201F56B5BD001010B
:1019B000C451300AD8B460BF05D0050E19D930EC37
:1019C0003DF050D060AF37D00501D46B00011EA6AA
:1019D0002ED001019E6B660E05011F6F0101A8D874
:1019E000660EDF6E9E2B1F0E7ED864D8616F613944
:1019F0000F0BFDEC44F0DF6E9E2B5CD80F0BFDEC63
:101A000044F0E0D89D65F1D71F0E63D81F0E9E25C8
:101A100075D8FDEC44F080D8FDEC44F0DF6E9E2BD1
:101A20009E51CAECF1F0C4D836EC22F01BD0000E67
:101A30004CECB8F017D00501D48117A408D0010EE2
:101A400001011E6F000E8FEC0CF0F0D802D00101E6
:101A50009E6B9E514CECB8F09E5190ECE3F002E28C
:101A60000101996B97C11EF501019E6B10D0650EA7
:101A70009E25D96EDA6A010EDA220E0E01019E252C
:101A8000E16EE26A050EE222DFCFE7FF9E2B97515F
:101A90009E5D02E396EF80F0EAD701019E25366F46
:101AA000376B050E3723120036519D6F9D519E27CF
:101AB0009C6B12001F0E01019E25D96EDA6A050E7D
:101AC000DA22C10E9D25E16EE26A010EE222E750A4
:101AD000120001019E25D96EDA6A050EDA222C0E5B
:101AE000DF6E9E2B2C0C9E25D96EDA6A050EDA224B
:101AF0002C0EDF6E9E2B010E9D6F010CD96EDA6AE3
:101B0000050EDA22C4390F0B1200770E9C25D96E10
:101B1000DA6A010EDA221200DF6E9E2B1F0E01011F
:101B20009E25D96EDA6A050EDA22C4510F0B120017
:101B30009E2B1F0E9E25D96EDA6A050EDA22120040
:101B4000376F1F0E366FFE0E396F1B0E386F130E78
:101B50003B6FFC0E3A6FFC0CD46B01019E6B300E98
:101B600005011F6F0101300CD46B050E0101376FA9
:101B70001F0E366F1200386F98C161F10F0E61179A
:101B800061293A6F3B6B000E3B23000CFF0E396F4F
:101B9000D90E386F9AC13AF19BC13BF11200FE0E8B
:101BA000396FD70E386F9AC13AF19BC13BF11200E1
:101BB0002D0E01019E25D96EDA6A0501050EDA2285
:101BC000DF6A000CDF6E9E2B9D2B020CFF0E396F1F
:101BD000DD0E386F9AC13AF19BC13BF11200FE0E47
:101BE000396FD10E386F9AC13AF19BC13BF11200A7
:101BF000376F1F0E366FFD0E396F700E386F120083
:101C00000E0E01019E25D96EDA6A050EDA22120047
:101C1000BA0E9C25186F196B010E1923010C9A0E30
:101C20009C25186F196B010E1923010C090E010177
:101C30009E6F090C330E0501FF6F4686FD694682D3
:101C400046804684060EFE6F20EC11F0E96B1AD038
:101C500083500F0BE06F270ED26F100ED16F01D0A3
:101C600004000101D107D8A0D207D129D8B4D229C4
:101C7000F7E183500F0BE01904E0E95103E0E907B5
:101C800001D0E92BE9510A0AE3E10F0EE01BE067FE
:101C900005D01780949C829C948450D0E051040A13
:101CA00010E10B82949C9484AD947E86090E7F6E25
:101CB000C20EB06EAC8EAC88AD8A9E9A9F9A9D8AF9
:101CC0003DD0E051060A02E111882DD0E0510E0A04
:101CD00008E1098A949C9484AD947E867F6A340ED0
:101CE000E8D7E00508E11382F188F092F08EF088E1
:101CF000060E766E23D0E0510A0A03E0E0510C0A8A
:101D00000AE10F8E0101E0510A0A01E11084F19C01
:101D1000F292F28813D0E051080A0DE10001058A21
:101D20007AEC41F09896949C9484AD947E86010E52
:101D30007F6E370EBED7E051020AABE0080E0101FC
:101D4000E96F8D968D948A988A968D9C8D9A8D8C4C
:101D50008D8A8D868D848A888A868F808F808C8AF2
:101D6000EA0ED26F600ED16F01D004000101D107DD
:101D7000D8A0D207D129D8B4D229F7E18D9C8D9A69
:101D80008D968D948A988A968F908F908C9AEA0E71
:101D9000D26F600ED16F01D004000101D107D8A02D
:101DA000D207D129D8B4D229F7E1E92FD0D7D08EE4
:101DB000F28EF28C196BFF0E1869E5EC2FF005011D
:101DC000FF1916E00101196BFF0E1869E5EC2FF001
:101DD0000501FF190DE063ECDFF00101186BFF0E48
:101DE0001769FFC519F1D6EC36F0010E0101E96F54
:101DF00046ECB0F0420E0101196F3B0E186FE5EC96
:101E00002FF00501FA6FFA29D8B48F80130E010163
:101E1000196F890E186FE5EC2FF00501FA6FFA299A
:101E2000D8B48F80D55113E0050E01011C6FD50E7B
:101E30001B6FFC0E1E6FDB0E1D6F206B070E1F6FDE
:101E40000AEC28F01C511B1102E01EA60E8C0701A3
:101E5000AB5102E01EA60E8CB8C3D1F1B9C3D2F1CA
:101E60000301B96B020EB86F00014694B3EC46F063
:101E70007BEC46F03D0E0101295D000E2A59F8E386
:101E8000D1C1B8F3D2C1B9F378EC2EF0DA6B148E6D
:101E90001580048E058000011990E2EC3BF086CF9E
:101EA000E8F1E8A916D0270ED26F100ED16FD10736
:101EB000D8A0D2070101D129D8B4D229F8E186CF20
:101EC000E8F1E8A906D000010F82000EBBEC3DF05E
:101ED0003FD0D9ECC1F013B03BD01A8C169E1584BC
:101EE000500E0101186FC00E176F000E196BD6EC63
:101EF00036F0500E0101186FC10E176F000E196BEE
:101F0000D6EC36F045ECE7F018A622D08D8C8D8A01
:101F1000EA0E0101D26F600ED16F01D000F0010115
:101F2000D107D8A0D207D129D8B4D229F7E18D9C06
:101F30008D9AEA0ED26F600ED16F01D000F00101D0
:101F4000D107D8A0D207D129D8B4D229DFE0F6D75B
:101F500012B014AA01D00E8612A005D000010EA660
:101F600002D0FF00FFD7000112A005D08D8C8D9A02
:101F7000010E63ECB4F012B00FA215D086CFE8F1D9
:101F80000101E8B910D0270ED26F100ED16FD10722
:101F9000D8A0D2070101D129D8B4D229F8E186CF3F
:101FA000E8F1E8A9FF0012B01BD086CFE8F10101EB
:101FB000E8A916D0270ED26F100ED16FD107D8A086
:101FC000D2070101D129D8B4D229F8E186CFE8F1AE
:101FD000E8A906D000010F82010EBBEC3DF0B8D796
:101FE00004B015A40BD015948D9C158A17A006D0AB
:101FF000040EBB6E9E949F949D84948C000112B03D
:1020000009D04DEC07F00301EB6FEB5103E0EB510E
:1020100056ECC9F013AE06D00301DD6703D07FECA8
:102020002CF0139E040E0301D3650AD0D36B500E1F
:102030000101206FDE0E1F6FACEC38F0D9ECC1F05F
:1020400003A403D003940301CB2B040E0301CB653F
:102050000AD0CB6B500E0101206FDE0E1F6FACEC6F
:1020600038F0D9ECC1F002AA09D0500E0101206F5E
:10207000D60E1F6FACEC38F0D9ECC1F002A809D035
:10208000500E0101206FD60E1F6FACEC38F0D9EC6A
:10209000C1F002AC10D0029C0301C92B010EC9652E
:1020A0000AD0C96B500E0101206FD80E1F6FACEC27
:1020B00038F0D9ECC1F002AE10D0029E0301CA2B59
:1020C000010ECA650AD0CA6B500E0101206FD80EEE
:1020D0001F6FACEC38F0D9ECC1F003AC04D00001B8
:1020E000039C83ECE0F009A80FD00998500E010181
:1020F000206FBE0E1F6FACEC38F0500E0101206F48
:10210000C00E1F6FACEC38F012A00EA471D016BE3A
:102110006FD00BA217D0030E0101176FF90E166FC7
:10212000E3EC40F0030E0101276FF90E266F32EC4D
:10213000D7F05EE2030E0101166FF90E156FA9ECE0
:102140002FF054D011A80FD0030E0101176FF90E14
:10215000166F17EC41F0030E0101206FF90E1F6F8F
:10216000A5ECD3F0E7D709AA0FD0030E0101176F32
:10217000F90E166F17EC41F0030E01012A6FF90EEC
:10218000296FE0ECD8F0D5D70FAE0FD0030E0101C8
:10219000176FF90E166F2FEC39F0030E0101276F40
:1021A000F90E266F79ECC4F0C4D713A20FD0030E3A
:1021B0000101176FF90E166FC9EC40F0030E010113
:1021C0001F6FF90E1E6FEAEC07F010D005BA05B6C6
:1021D0000FD0030E0101176FF90E166F0CEC40F0D3
:1021E0000301F951080A02E1058602D0168E168C09
:1021F00012A00FAE3ED04150080A25E110B406D01F
:102200000301EF51EB0A1FE10C841DD00101D5B58C
:102210001AD0D5A30FD00301EF51A50A14E0020E86
:102220000101D5170301EF51EB0A0DE1040E010185
:10223000D56F09D00301EF51A50A05E10101D5B120
:10224000E3D7D581D5831AB60BD01AA403D01A943C
:102250000301E76B0301E7A70CD01A86148609D0A7
:102260000C841AA406D01A940301E76B1A9610AADC
:10227000148812A005AA90D016BA29D00101D867F7
:102280008BD005A611D00588FCC316F1FAC317F14F
:10229000010E186F0301FB5145EC14F0168A059CE2
:1022A000F00E0101D86F78D00301BE2B450E01015D
:1022B000166FBEC317F1186B540E45EC14F00301F2
:1022C000BE510F0AEBE1BE6B8F801388E7D7010187
:1022D000D8670AD0169A000105B803D0C3EC1DF0E8
:1022E0005BD00598059658D005AC56D005A802D00D
:1022F00005980596059C169A0301EF51240A06E0FD
:10230000EF515E0A03E0EF51260A2FE1EF51240A54
:1023100002E1189E04D0EF515E0A03E1188E059E7B
:1023200002D0189E058E0301BF5123EEF0F0DF624C
:102330001CD04050120A03E04050060A16E14050FB
:10234000FEEC2CF012E30301F05194EC44F0D66F54
:102350004050120A1EE109A20BD0150E0101166FA2
:10236000BEC317F1186B45EC14F0C3EC1DF098D701
:10237000060E0101166FBEC317F1186B45EC14F081
:1023800022EC15F0030E0101176FEF0E166F91ECA2
:1023900042F054EC3CF084D712A013A213D013A641
:1023A00008D013960301E76B1AA60CD01A9614886E
:1023B00009D00301E7A306D0E76B1AB603D01A864B
:1023C00014860C8412B004D0000114B2ABECEAF015
:1023D00012A01BBC00D118AAFED0189A18A417ACE2
:1023E00078D012BE76D0000113AC08D090EC46F045
:1023F0007FEC2CF01682010E0101E96F310EA0EC8A
:102400000DF0E86FE85165EC13F00DE2000118B033
:1024100023D01880178E500E0101206FD00E1F6F31
:10242000ACEC38F019D000010490B3EC46F009D0C0
:10243000000104A006D018A00CD0189018820E92AB
:1024400008D07BEC46F0410E0101295D9C0E2A5913
:10245000EFE3000104A0DAD7300EA0EC0DF0E86F36
:10246000EA6BE85165EC13F00EE2010E0101EA6F30
:1024700017B821D017881786500E206FCE0E1F6F09
:10248000ACEC38F018D000010490B3EC46F009D061
:10249000000104A006D017A80CD01798178A0E9236
:1024A00008D07BEC46F0410E0101295D9C0E2A59B3
:1024B000EFE304A0DAD70101EA5103E0D9ECC1F05F
:1024C00002D046EC31F00101E95101E184D01B82D8
:1024D00082D018B412BC7FD0000113AC08D090ECAD
:1024E00046F07FEC2CF01682010E0101E96F300EF0
:1024F000A0EC0DF0E86FEA6BE85165EC13F00EE22A
:10250000010E0101EA6F17B828D017881786500E00
:10251000206FCE0E1F6FACEC38F01FD0000104907E
:10252000B3EC46F009D0000104A006D017A80CD0E7
:102530001798178A0E9208D07BEC46F0410E0101E5
:10254000295D9C0E2A59EFE304B007D0010E01016A
:10255000EA6F17B802D0178817860101EA5137E0F1
:10256000310EA0EC0DF0E86FEA6BE85165EC13F06A
:102570000EE2010E0101EA6F18B021D01880178E0B
:10258000500E206FD00E1F6FACEC38F018D0000149
:102590000490B3EC46F009D0000104A006D018A0C6
:1025A0000CD0189018820E9208D07BEC46F0410EA9
:1025B0000101295D9C0E2A59EFE304A0DAD701013D
:1025C000EA5103E0D9ECC1F002D046EC31F0010150
:1025D000E95101E07CD712A01AACD4D11A9CF10EBB
:1025E0000101176F320E166F010EA3EC33F0130EBC
:1025F00001012A6F880E296FD8EC38F00101E96BD0
:1026000018A402D0010EE96F0101E9511FEC09F095
:10261000020A07E10301E62BE651020A04E1FF008A
:1026200002D00301E66BFA0E0101176F2C0E166F34
:10263000010EA3EC33F0880E0101296F130E2A6FEF
:10264000000E2B6B2C6B2D6BFCEC9FF00101E86FE7
:10265000F80E176FE30E166F010EA3EC33F0880E21
:102660000101296F130E2A6F000E2B6B2C6B2D6B43
:10267000FCEC9FF00101E86F030EE96F0301CF2B23
:1026800018D0FE0E176F530E166F010EA3EC33F029
:10269000880E0101296F130E2A6F000E2B6B2C6B15
:1026A0002D6BFCEC9FF00101E86FE851230A04E078
:1026B000E9070101E967E5D7E9512BE00301CF6B99
:1026C0000101EA6B8F0E0101EA25D96EDA6A060E66
:1026D000DA229B0EEA25E16EE26A070EE222DFCFE4
:1026E000E7FF8F0EEA25D96EDA6A060EDA22DF508E
:1026F00004E0EA2B0F0EEA65E5D7880E0101296F89
:10270000130E2A6F2B6B2C6B010E2D6FFCEC9FF0C0
:1027100007D0020E0301CF6503D0CF6BD9ECC1F017
:10272000030E0101E96F0301CC2B6FD0FC0E176F74
:10273000BB0E166F010EA3EC33F0880E0101296F5A
:10274000130E2A6F000E2B6B2C6B2D6BFCEC9FF085
:102750000101E86F0601FE6B0101EA6B8F0E0101BA
:10276000EA25D96EDA6A060EDA22D20EEA25E16E81
:10277000E26A080EE222DFCFE7FF0601FE51030AFC
:102780000DE18F0E0101EA25D96EDA6A0601060E07
:10279000DA22370EDF6202D08C8A0ED0FE51030A95
:1027A0000BE18F0E0101EA25D96EDA6A060EDA22F4
:1027B000300EDF6201D08C9A8F0E0101EA25D96EAE
:1027C000DA6A0601060EDA222C0EDF6201D0FE2B39
:1027D0008F0E0101EA25D96EDA6A060EDA22DF5081
:1027E00004E0EA2B1F0EEA65B9D7880E0101296FB4
:1027F000130E2A6F2B6B2C6B010E2D6FFCEC9FF0D0
:102800000101E851130A04E0E9070101E9678ED7E5
:10281000E95103E00301CC6B07D0020E0301CC6544
:1028200003D0CC6BD9ECC1F0A8EC10F017E2500E3D
:102830000101206FDA0E1F6FACEC38F0D9ECC1F05B
:1028400017B812AE01D00E8218B012AC01D00E82B1
:1028500017B818A001D00E8216B01B82030E01011A
:10286000E96F0301C82B4FD0FB0E176F700E166F68
:10287000010EA3EC33F0880E0101296F130E2A6FAD
:10288000000E2B6B2C6B2D6BFCEC9FF00101E86FA5
:10289000EA6B8F0E0101EA25D96EDA6A060EDA229A
:1028A0008B0EEA25E16EE26A070EE222DFCFE7FF38
:1028B0008F0EEA25D96EDA6A060EDA22DF5004E0BE
:1028C000EA2B0F0EEA65E5D7880E0101296F130E7A
:1028D0002A6F2B6B2C6B010E2D6FFCEC9FF001010E
:1028E000E8511C0A13E0E8511D0A10E0E8511E0AE5
:1028F0000DE0E8511F0A0AE0E851200A07E0E8511C
:10290000210A04E0E9070101E967AED7E9510CE0CB
:10291000E851200A09E0E8511E0A06E0E8511F0AC2
:1029200003E00301C86B0ED0040E0301C8650AD092
:10293000C86B500E0101206FDC0E1F6FACEC38F03D
:10294000D9ECC1F0A00E0501FA6F070EFB6FFAC5B6
:102950001BF1FBC51CF149EC19F01B51E86FE85164
:10296000630A03E10301D66B0DD00B0EE86102D0C0
:10297000010E06D0100EE86102D0020E01D0030E47
:102980000301D66F12B0A1D21AB214AC01D01582D5
:1029900014BC1AA215921AB007AC01D0088A07BC61
:1029A0001AA0089A13BC07A609D0050E01015D6F95
:1029B0001F0E5C6F000E5E6B3FECA6F012A405D0FC
:1029C0000301BD51BC11D8B4FF0012A604D0000110
:1029D0001296D9ECC1F013BC03AE1DD0039EF80EC5
:1029E0000101176FB40E166F010EA3EC33F090ECDB
:1029F00046F0168209B608D0500E0101206FC20EB3
:102A00001F6FACEC38F007D0500E0101206FC60EDE
:102A10001F6FACEC38F01BA00ED01B9013AC0BD08A
:102A2000000109A608D090EC46F07FEC2CF0069847
:102A300009961B820B881BA2F3D013AC16A0EBD017
:102A400004B008BAE8D015B2E6D016B28AD006B8FB
:102A500043D00101E96BD50E0101E925D96EDA6A8F
:102A6000050EDA22CD0EE925186F196B000E192319
:102A7000E5EC2FF0DF6ED50E0101E925D96EDA6A9B
:102A8000050EDA22DF5004E0E92B0F0EE965E3D7EB
:102A90000101E96BF50E0101E925D96EDA6A050E2F
:102AA000DA22C80EE925186F196B000E1923E5EC20
:102AB0002FF0DF6EF50E0101E925D96EDA6A050EF9
:102AC000DA22DF5004E0E92B040EE965E3D70FB802
:102AD00006880001099647D000010FA844D00101E3
:102AE000E96BD50E0101E925D96EDA6A050EDA2205
:102AF0008A0EE925186F196B010E1923E5EC2FF0EA
:102B0000DF6ED50E0101E925D96EDA6A050EDA22EB
:102B1000DF5004E0E92B0F0EE965E3D70101E96B13
:102B2000F50E0101E925D96EDA6A050EDA22850E65
:102B3000E925186F196B010E1923E5EC2FF0DF6EF4
:102B4000F50E0101E925D96EDA6A050EDA22DF50A9
:102B500004E0E92B040EE965E3D706980001098635
:102B600002D000011692A8EC10F015AE0AD0020EA9
:102B700002019E6F000EF0EC31F00101E96F159E2D
:102B800008D0010E02019E6F000EF0EC31F0010141
:102B9000E96F0101E90506E0E951020A03E0E951A4
:102BA000040A20E109B608D0500E0101206FCA0EB8
:102BB0001F6FACEC38F007D0500E0101206FCC0E27
:102BC0001F6FACEC38F00FA80BD009B603D003018F
:102BD000D88102D00301D883D851030A19E1D86BF8
:102BE0000D8A16D0E96714D00301D86B0D9A09B687
:102BF00008D0500E0101206FC40E1F6FACEC38F0EE
:102C000007D0500E0101206FC80E1F6FACEC38F0DA
:102C10000301D96B1B900BA802D00B9801D01B921B
:102C200013BC15A654D000011596BFEC43F001016A
:102C3000E96F0301EB5104E0EB6BEB5156ECC9F08B
:102C40000101E96701D0168203AE17D009B608D09A
:102C5000500E0101206FC20E1F6FACEC38F007D090
:102C6000500E0101206FC60E1F6FACEC38F0000152
:102C7000039E90EC46F016822AD00101E95103E050
:102C8000E951050A16E109B608D0500E0101206F7E
:102C9000C20E1F6FACEC38F007D0500E0101206F50
:102CA000C60E1F6FACEC38F090EC46F07FEC2CF0C9
:102CB0000ED0E951030A04E1010E56ECC9F007D029
:102CC000E951040A04E1010E56ECC9F015860EAA7A
:102CD0000BD0139C0E9A0E9C16900301CD6B000135
:102CE0001A9C7FEC2CF0F1D00EACEFD00E9C13BCF4
:102CF000ECD016800101E96BD50E0101E925D96EF2
:102D0000DA6A050EDA22CD0EE925186F196B000E6E
:102D10001923E5EC2FF0DF6ED50E0101E925D96E00
:102D2000DA6A050EDA22DF5004E0E92B0F0EE965BE
:102D3000E3D70101E96BF50E0101E925D96EDA6AE5
:102D4000050EDA22C80EE925186F196B000E19233B
:102D5000E5EC2FF0DF6EF50E0101E925D96EDA6A98
:102D6000050EDA22DF5004E0E92B040EE965E3D713
:102D70000996069800010FA802D000010688A8EC69
:102D800010F0D5C39EF2000EF0EC31F00101E96FB6
:102D9000159EE90505E118B402D00D8801D00D8219
:102DA0000101E951020A03E0E951040A55E10F80EB
:102DB0000FA852D00101E96BD50E0101E925D96EAA
:102DC000DA6A050EDA228A0EE925186F196B010EF0
:102DD0001923E5EC2FF0DF6ED50E0101E925D96E40
:102DE000DA6A050EDA22DF5004E0E92B0F0EE965FE
:102DF000E3D70101E96BF50E0101E925D96EDA6A25
:102E0000050EDA22850EE925186F196B010E1923BC
:102E1000E5EC2FF0DF6EF50E0101E925D96EDA6AD7
:102E2000050EDA22DF5004E0E92B040EE965E3D752
:102E3000098600010698A8EC10F0D5C39EF2000E9A
:102E4000F0EC31F00101E96F159EE951020A03E04F
:102E5000E951040A01E10E8E0101E951050A01E17F
:102E6000088C0101E90506E0E951020A03E0E95195
:102E7000040A13E109B608D0500E0101206FCA0EF2
:102E80001F6FACEC38F007D0500E0101206FCC0E54
:102E90001F6FACEC38F00D8A14D0E96712D00D9A90
:102EA00009B608D0500E0101206FC40E1F6FACECA4
:102EB00038F007D0500E0101206FC80E1F6FACEC28
:102EC00038F01B920301D96B1B9012B023D00FA4D2
:102ED00002D00F941B8E46840101DA511AE0B1EC46
:102EE0000FF00101E96B11D0E951020D000EF3243E
:102EF000D96EDA6A060EDA220101DECF58F1DDCF93
:102F000059F141ECF0F004E3E92BDA51E95DECE32F
:102F1000DA6B469412B0F7D004A0F4D00401EF515C
:102F2000EE1101E0EFD0010EB0EC39F015C1D9FF80
:102F300016C1DAFFDF50E86F020EB0EC39F015C1B0
:102F4000D9FF16C1DAFFDF50E827000119BC09D00C
:102F5000030EB0EC39F015C1D9FF16C1DAFFDF500E
:102F6000E827040EB0EC39F015C1D9FF16C1DAFF1D
:102F7000DF50E827050EB0EC39F015C1D9FF16C1B6
:102F8000DAFFDF50E827E86711D00301EE6B0EA8E7
:102F900005D000010E987FEC2CF0FF0000011BAE65
:102FA000B1D0010EBBEC3DF01B9EACD00301EE2B6B
:102FB000050EEE6502D0010EEE6FEE51B0EC39F069
:102FC00015C1D9FF16C1DAFFDF50E86FE86701D0FD
:102FD00099D0EEC318F1000E4FEC42F018C1D1F1B8
:102FE00019C1D2F1EEC3ECF3D1C1FAF5D2C1FBF5B0
:102FF0000D0E0501FC6FD890FB33FA33FC2FFBD785
:10300000FA51030B0301C06FEC050DE1000113AC95
:103010000AD0000E0101D1115F6F800ED211606FD6
:1030200000EC80F006D0D1C15FF1D2C160F100ECBC
:1030300080F0E96F030E0401EF6FE80EEE6F0101FF
:10304000E96706D0ECC318F1000EE5EC28F05AD081
:1030500013AC04D0010E0301EC6506D00301EC5162
:10306000030AD8A4A8EC10F013AC04D0010E03019D
:10307000EC6536D00301D76745D000010C80BCEC6D
:10308000CFF019E2500E0101206FE20E1F6FACEC81
:1030900038F00301EC51030A0AE11EAA08D0D22B32
:1030A000038CD251050A03E1198CD26B049E0301F3
:1030B000EC29D16F13D00301C96BCA6BECC318F1B3
:1030C000000EE5EC28F00301EC51030A04E11EAA0E
:1030D00002D0D26B048E060E0301D76F0C9012D073
:1030E00000010C80F3EC12F005E2020E0301D16F37
:1030F000D32BF4D70301D36BECC318F1000EE5EC2E
:1031000028F0ECD700F012B0A8EF8FF0000103A078
:1031100003D0000E42EC17F0000103A2A8EF8FF0DD
:10312000010E42EC17F0A8EF8FF0E8CF6AF16DC600
:1031300015F101016A5192EC41F002E2D8901200BF
:1031400005012251740A03E02251540A4FE1235130
:10315000720A03E02351520A16E1D351050AEEE147
:1031600001016D6BC20E6D25176F186B500E182381
:10317000000E196BD6EC36F001016D2B250E6D6536
:10318000F1D794EF9FF0050ED36101D0D7D725EE8C
:10319000D3F0070EDF6401D0D1D71F0ED325D96E2F
:1031A000DA6A050EDA22DF6A230E0101686F050E66
:1031B000696F68C11BF169C11CF149EC19F01BC1B1
:1031C0006BF11CC16CF1000E6B5D010E6C59B6E227
:1031D0006C516B11B3E06BC1F2F2186B550E176FA7
:1031E000F2C219F1D6EC36F094EF9FF022516E0A3C
:1031F00003E022514E0A31E1050ED36101D09ED782
:1032000025EED3F0060EDF6401D098D71F0ED3252C
:10321000D96EDA6A050EDA22DF6A230E0101686FC1
:10322000050E696F68C11BF169C11CF149EC19F009
:103230001BC16BF11CC16CF1110E6B5D000E6C5962
:1032400001E37CD76BC1DCF1186B760E176FDCC124
:1032500019F1D6EC36F094EF9FF02251690A04E0A0
:103260002251490A01E0AED02351690A03E02351FB
:10327000490A5CE10C0ED36101D060D725EED3F092
:10328000140EDF6401D05AD7050E01016D6F21D0F5
:103290001F0E01016D25D96EDA6A050EDA22D00EF5
:1032A0006D25E16EE26A050EE222DFCFE7FF850EB3
:1032B0006D25176F186B010E18231F0E6D25D96E23
:1032C000DA6A050EDA22DF50196FD6EC36F001010A
:1032D0006D2B0501D35101016D5DDAE3D10E6D2532
:1032E000D96EDA6A050EDA22DF6A850E6D25176F50
:1032F000186B010E1823000E196BD6EC36F00F98E0
:103300000501D55157E0050E01011C6FD50E1B6F4D
:10331000FC0E1E6FDB0E1D6F206B070E1F6F0AEC7D
:1033200028F01C511B1146E00F8844D00B0ED361CE
:1033300001D004D725EED3F0130EDF6401D0FED602
:10334000040E01016D6F21D01F0E01016D25D96E94
:10335000DA6A050EDA22D10E6D25E16EE26A050EFB
:10336000E222DFCFE7FFC90E6D25176F186B000E45
:1033700018231F0E6D25D96EDA6A050EDA22DF508A
:10338000196FD6EC36F001016D2B0501D351010107
:103390006D5DDAE3D10E6D25D96EDA6A050EDA229B
:1033A000DF6AC90E6D25176F186B000E1823196B95
:1033B000D6EC36F006980996000113BC6EEC45F089
:1033C00094EF9FF02251610A04E02251410A01E08A
:1033D000BED02351610A03E02351410A4CE1060E9D
:1033E000D36101D0ABD625EED3F01F0EDF6401D040
:1033F000A5D6050E01016D6F24D018A40FD01F0EA5
:1034000001016D25D96EDA6A050EDA226B0E6D2583
:10341000E16EE26A070EE222DFCFE7FF1B0E010139
:103420006D25176F186B030E18231F0E6D25D96EAF
:10343000DA6A050EDA22DF50196FD6EC36F0010198
:103440006D2B0501D35101016D5DD7E318A407D0A1
:103450006B0E6D25D96EDA6A070EDA22DF6A1B0E53
:1034600001016D25176F186B030E1823000E196BE1
:10347000D6EC36F04AD0050ED36101D05FD625EEEA
:10348000D3F01E0EDF6401D059D6040E01016D6F1A
:1034900024D018B40FD01F0E01016D25D96EDA6A41
:1034A000050EDA226C0E6D25E16EE26A070EE2224D
:1034B000DFCFE7FF940E01016D25176F186B000E2B
:1034C00018231F0E6D25D96EDA6A050EDA22DF5039
:1034D000196FD6EC36F001016D2B0501D3510101B6
:1034E0006D5DD7E318B407D06C0E6D25D96EDA6A1E
:1034F000070EDA22DF6A940E01016D25176F186B33
:10350000000E1823196BD6EC36F013BC55D7EF0E0E
:103510000101176F9D0E166F010EA3EC33F0070E1D
:103520000101176F700E166F000EA3EC33F0220E20
:103530005CEC44F00D0E5CEC44F0130E01012A6FBC
:10354000880E296FD8EC38F009EC1DF035D72251E0
:10355000700A03E02251500A7CE12351700A03E013
:103560002351500A31E1060ED36101D0E7D525EE93
:10357000D3F0090EDF6401D0E1D5050E01016D6FB6
:1035800013D0800E6D25176F186B010E18231F0EB8
:1035900001016D25D96EDA6A050EDA22DF50196F46
:1035A000D6EC36F001016D2B0501D35101016D5DA3
:1035B000E8E3800E6D25176F186B010E1823000EBF
:1035C000196BD6EC36F0F6D6050ED36101D0B6D520
:1035D00025EED3F0080EDF6401D0B0D5040E010152
:1035E0006D6F21D01F0E01016D25D96EDA6A050EAF
:1035F000DA22F10E6D25E16EE26A050EE222DFCFDE
:10360000E7FFC40E6D25176F186B000E18231F0EF1
:103610006D25D96EDA6A050EDA22DF50196FD6EC05
:1036200036F001016D2B0501D35101016D5DDAE327
:10363000F10E6D25D96EDA6A050EDA22DF6AC40E44
:103640006D25176F186B000E1823196BD6EC36F02A
:10365000B1D62251640A03E02251440A57E12351B2
:10366000690A03E02351490A51E125EED3F0140E13
:10367000DF6401D063D5D351050A0CE1010E0101CD
:10368000186F750E176F000E196BD6EC36F0070128
:10369000AB6B92D6050E01016D6F21D01F0E01019B
:1036A0006D25D96EDA6A050EDA22A60E6D25E16E59
:1036B000E26A070EE222DFCFE7FF700E6D25176F7B
:1036C000186B010E18231F0E6D25D96EDA6A050ED0
:1036D000DA22DF50196FD6EC36F001016D2B0501AF
:1036E000D35101016D5DDAE3A60E6D25D96EDA6A5C
:1036F000070EDA22DF6A700E6D25176F186B010E48
:103700001823000E196BD6EC36F056D62251640AF7
:1037100003E02251440A4CE12351640A03E023519F
:10372000440A46E125EED3F0250EDF6401D006D52C
:10373000060ED36101D002D5050E01016D6F21D0B7
:103740001F0E01016D25D96EDA6A050EDA224B0EC5
:103750006D25E16EE26A070EE222DFCFE7FF500E31
:103760006D25176F186B010E18231F0E6D25D96E6E
:10377000DA6A050EDA22DF50196FD6EC36F0010155
:103780006D2B0501D35101016D5DDAE34B0E6D2503
:10379000D96EDA6A070EDA22DF6A500E6D25176FCE
:1037A000186B010E1823000E196BD6EC36F004D6F8
:1037B0002251770A03E02251570A69E125EED3F03E
:1037C000130EDF6401D0BAD4050ED36101D0B6D494
:1037D000040E01016D6F1CD01F0E01016D25D96E05
:1037E000DA6A0501050EDA22DF50800A500F01E285
:1037F000A5D41F0E01016D25D96EDA6A0501050EEB
:10380000DA22DF50800A460F01E398D401016D2BC4
:103810000501D35101016D5DDFE3040E6D6F21D011
:103820001F0E01016D25D96EDA6A050EDA22B70E78
:103830006D25E16EE26A070EE222DFCFE7FFAF0EF1
:103840006D25176F186B000E18231F0E6D25D96E8E
:10385000DA6A050EDA22DF50196FD6EC36F0010174
:103860006D2B0501D35101016D5DDAE3B70E6D25B6
:10387000D96EDA6A070EDA22DF6AAF0E6D25176F8E
:10388000186B000E1823196BD6EC36F095D5225123
:10389000720A03E02251520A34E1050ED36101D0CD
:1038A0004DD425EED3F0070EDF6401D047D41F0EB0
:1038B000D325D96EDA6A050EDA22DF6A230E0101FA
:1038C000686F050E696F68C11BF169C11CF149EC95
:1038D00019F01BC16BF11CC16CF1000E6B5D010E88
:1038E0006C5901E32BD46C516B1101E127D46BC1EE
:1038F000DEF2186B730E176FDEC219F1D6EC36F0DC
:1039000013D322516F0A03E022514F0A36E1050E0C
:10391000D36101D013D425EED3F0070EDF6401D0BC
:103920000DD41F0ED325D96EDA6A050EDA22DF6AAE
:10393000230E0101686F050E696F68C11BF169C133
:103940001CF149EC19F01BC16BF11CC16CF1000EAC
:103950006B5D010E6C5902E39EEF98F06C516B1198
:1039600002E19EEF98F06BC1E1F2186B700E176FD9
:10397000E1C219F1D6EC36F0D7D222516D0A03E03C
:1039800022514D0A38E1050ED36102D09EEF98F026
:1039900025EED3F0070EDF6402D09EEF98F01F0EE5
:1039A000D325D96EDA6A050EDA22DF6A230E010109
:1039B000686F050E696F68C11BF169C11CF149ECA4
:1039C00019F01BC16BF11CC16CF1000E6B5D010E97
:1039D0006C5902E39EEF98F06C516B1102E19EEF7F
:1039E00098F06BC1DDF1186B720E176FDDC119F124
:1039F000D6EC36F099D22251660A03E02251460AEB
:103A000039E1D351050A02E09EEF98F00101196BEC
:103A1000750E186FE5EC2FF06D6F05012351300A1C
:103A200006E11A901A92F90E01016D171AD023516E
:103A3000310A06E11A801A9201016D836D9511D049
:103A40002351320A06E11A901A8201016D856D93A5
:103A500008D02351330A05E11A801A82060E0101AB
:103A60006D130101186B750E176F6DC119F1D6EC4E
:103A700036F05AD22251650A03E02251450A25E167
:103A8000D351050A02E09EEF98F00101196B4F0E29
:103A9000186FE5EC2FF06D6F05012351300A04E13A
:103AA0001E9A01016D9908D02351310A05E11E8A41
:103AB00001016D8983ECE0F00101186B4F0E176F67
:103AC0006DC119F1D6EC36F02FD22251730A03E002
:103AD0002251530A0FE1D351050A02E09EEF98F0FC
:103AE0002351300A01E120D22351310A01E11CD2D5
:103AF0009EEF98F02251630A04E02251430A01E04C
:103B0000D3D0D351050A20E12351310A03E100014A
:103B10000A820AD22351320A03E100010A8404D244
:103B20002351330A03E10001098EFED12351340AE7
:103B300003E10001098CF8D12351360A02E09EEF1F
:103B400098F000010A86F0D1D3510A0A44E1EF0E41
:103B50000101176FC00E166F010EA3EC33F00501C3
:103B600023515CEC44F0050124515CEC44F03A0E26
:103B70005CEC44F0050125515CEC44F00501265154
:103B80005CEC44F03A0E5CEC44F0050127515CEC2F
:103B900044F0050128515CEC44F0FE0E0101176F62
:103BA000590E166F000EA3EC33F0130E01012A6FAD
:103BB000880E296FD8EC38F002E300011784B3ECCB
:103BC00046F07BEC46F0E90E0101295D030E2A590F
:103BD00001E3AAD1F6D7D351100A01E0A5D1FC0E1A
:103BE0000101176FD30E166F010EA3EC33F0050120
:103BF00027515CEC44F0050128515CEC44F02F0E99
:103C00005CEC44F0050125515CEC44F005012651C3
:103C10005CEC44F02F0E5CEC44F0050123515CECAD
:103C200044F0050124515CEC44F02C0E5CEC44F0B3
:103C3000050129515CEC44F005012A515CEC44F08B
:103C40003A0E5CEC44F005012B515CEC44F00501AC
:103C50002C515CEC44F03A0E5CEC44F005012D5123
:103C60005CEC44F005012E515CEC44F0FE0E0101C9
:103C7000176F590E166F000EA3EC33F0130E0101EF
:103C80002A6F880E296FD8EC38F002E30001178400
:103C9000B3EC46F07BEC46F0E90E0101295D030E22
:103CA0002A5901E341D1F6D72251790A05E0225180
:103CB000590A02E09EEF98F02351790A04E023515B
:103CC000590A01E098D0060ED36102D09EEF98F019
:103CD00025EED3F00E0EDF6402D09EEF98F0245153
:103CE000310A42E1060E01016D6F24D018A40FD0F5
:103CF0001F0E01016D25D96EDA6A050EDA22D90E82
:103D00006D25E16EE26A060EE222DFCFE7FF350E97
:103D100001016D25176F186B030E18231F0E6D25FB
:103D2000D96EDA6A050EDA22DF50196FD6EC36F05A
:103D300001016D2B0501D35101016D5DD7E318A47D
:103D400007D0D90E6D25D96EDA6A060EDA22DF6A3F
:103D5000350E01016D25176F186B030E1823000E29
:103D6000196BD6EC36F0DCD02451320A02E09EEF1B
:103D700098F0060E01016D6F24D018A40FD01F0E0D
:103D800001016D25D96EDA6A050EDA22E20E6D2583
:103D9000E16EE26A060EE222DFCFE7FF3E0E01018E
:103DA0006D25176F186B030E18231F0E6D25D96E26
:103DB000DA6A050EDA22DF50196FD6EC36F001010F
:103DC0006D2B0501D35101016D5DD7E318A407D018
:103DD000E20E6D25D96EDA6A060EDA22DF6A3E0E31
:103DE00001016D25176F186B030E1823000E196B58
:103DF000D6EC36F095D0050ED36102D09EEF98F048
:103E000025EED3F00D0EDF6402D09EEF98F0235123
:103E1000310A41E1050E01016D6F24D018B40FD0B5
:103E20001F0E01016D25D96EDA6A050EDA22DA0E4F
:103E30006D25E16EE26A060EE222DFCFE7FFE80EB3
:103E400001016D25176F186B000E18231F0E6D25CD
:103E5000D96EDA6A050EDA22DF50196FD6EC36F029
:103E600001016D2B0501D35101016D5DD7E318B43C
:103E700007D0DA0E6D25D96EDA6A060EDA22DF6A0D
:103E8000E80E01016D25176F186B000E1823196BD2
:103E9000D6EC36F045D02351320A02E09EEF98F07E
:103EA000050E01016D6F24D018B40FD01F0E010153
:103EB0006D25D96EDA6A050EDA22E30E6D25E16E04
:103EC000E26A060EE222DFCFE7FFF10E01016D2567
:103ED000176F186B000E18231F0E6D25D96EDA6A46
:103EE000050EDA22DF50196FD6EC36F001016D2B8A
:103EF0000501D35101016D5DD7E318B407D0E30E7E
:103F00006D25D96EDA6A060EDA22DF6AF10E01013A
:103F10006D25176F186B000E1823196BD6EC36F051
:103F2000000113AC09EC1DF0B1EC0FF001016A398E
:103F3000F00B6D6F0AA207D00A928A0E4A6F6D517C
:103F40008CECF2F038D00AA408D00A948B0E010150
:103F50004A6F6D518CECF2F02ED009AE08D0099E5C
:103F60008C0E01014A6F6D518CECF2F024D009AC3B
:103F700008D0099C8D0E01014A6F6D518CECF2F056
:103F80001AD00AA008D00A908E0E01014A6F6D5116
:103F90008CECF2F010D00AA608D00A968F0E010120
:103FA0004A6F6D518CECF2F006D0830E01014A6F1E
:103FB0006D518CECF2F04AC16BF14BC16CF119A45C
:103FC00004D000011994D880120006016D5129EC2B
:103FD00046F0F9E36A51C3EC3EF001016D6F6BC12D
:103FE00039F16CC13AF16AC13BF16DC13CF1030E8C
:103FF0003D6FABEC35F0E7D72D671BD005010A6BA1
:104000000B6B0C6B0D6B0294029604D0ABECEAF0D8
:1040100002B40FD005010D51800A800F08E1000E97
:104020000C5D05E1EA0E0B5D02E1610E0A5DEEE357
:104030000C0C05010A6B0B6B0C6B0D6B02A602944A
:1040400008D0ABECEAF002A404D002940201CE67DF
:1040500017D001012C51800A2E6F05010A51010170
:10406000295D05010B5101012A5905010C5101017E
:104070002B5905010D51800A01012E59D9E3E1D7D1
:10408000029601012F6BA00E01012F25D96EDA6A6D
:10409000080EDA228F0E2F25E16EE26A060EE2226A
:1040A000DFCFE7FF8F0E2F25D96EDA6A060EDA22F0
:1040B000DF5004E02F2B310E2F65E5D7060E0101EE
:1040C0001C6F8F0E1B6FF90E1E6F670E1D6F206B1E
:1040D0000A0E1F6F0AEC28F01C511B1106E10001AB
:1040E00002A4020C00010286020C060E01011C6FE4
:1040F0008F0E1B6FF40E1E6F6C0E1D6F206B0C0E5F
:104100001F6F0AEC28F01C511B1106E1000102A4EC
:104110002F0C000102862F0C060E01011C6F8F0E62
:104120001B6FFD0E1E6F130E1D6F206B070E1F6F92
:104130000AEC28F01C511B11D2E0060E01011C6F85
:104140008F0E1B6FEF0E1E6FD10E1D6F206B100EAA
:104150001F6F0AEC28F01C511B1106E1000102A49C
:10416000060C00010286060C060E01011C6F8F0E64
:104170001B6FFB0E1E6FB80E1D6F206B080E1F6F9E
:104180000AEC28F01C511B1106E1000102A4240CCA
:1041900000010286240C060E01011C6F8F0E1B6F9E
:1041A000FD0E1E6F700E1D6F206B020E1F6F0AEC4E
:1041B00028F01C511B1106E1000102A4080C0001AB
:1041C0000286080C060E0101236F8F0E226F070E68
:1041D000256FDB0E246F76EC27F02351221106E0C9
:1041E000000102A4030C00010286030C060E01016B
:1041F0001C6F8F0E1B6FF90E1E6F180E1D6F206B3C
:10420000010E1F6F0AEC28F01C511B1106E1000182
:1042100002A40D0C000102860D0C060E01011C6F9C
:104220008F0E1B6FFB0E1E6FAD0E1D6F206B010EF0
:104230001F6F0AEC28F01C511B1106E1000102A4BB
:10424000100C00010286100C060E01011C6F8F0E6F
:104250001B6FF60E1E6F1E0E1D6F206B010E1F6F63
:104260000AEC28F01C511B1106E1000102A4110CFC
:1042700000010286110C060E01011C6F8F0E1B6FD0
:10428000EF0E1E6FE00E1D6F206B010E1F6F0AEC0C
:1042900028F01C511B1106E1000102A40F0C0001C3
:1042A00002860F0C060E01011C6F8F0E1B6FFE0E97
:1042B0001E6F8F0E1D6F206B050E1F6F0AEC28F00E
:1042C0001C511B1106E1000102A43A0C00010286F8
:1042D0003A0C060E01011C6F8F0E1B6FFF0E1E6F36
:1042E0002F0E1D6F206B040E1F6F0AEC28F01C515F
:1042F0001B1106E1000102A43B0C000102863B0CED
:10430000060E01011C6F8F0E1B6FF50E1E6FFC0E4B
:104310001D6F206B0B0E1F6F0AEC28F01C511B1138
:1043200001E1DDD6060E01011C6F8F0E1B6FF60E2C
:104330001E6F200E1D6F206B0B0E1F6F0AEC28F0F6
:104340001C511B1101E1E2D6060E01011C6F8F0EFC
:104350001B6FF60E1E6F080E1D6F206B0B0E1F6F6E
:104360000AEC28F01C511B1106E1000102A4430CC9
:1043700000010286430C060E01011C6F8F0E1B6F9D
:10438000F00E1E6F470E1D6F206B0F0E1F6F0AEC95
:1043900028F01C511B1106E1000102A4440C00018D
:1043A0000286440C060E01011C6F8F0E1B6FEE0E71
:1043B0001E6FFB0E1D6F206B110E1F6F0AEC28F095
:1043C0001C511B1106E1000102A4450C00010286EC
:1043D000450C060E01011C6F8F0E1B6FF00E1E6F39
:1043E000370E1D6F206B0F0E1F6F0AEC28F01C514B
:1043F0001B1106E1000102A4390C00010286390CF0
:10440000060E01011C6F8F0E1B6FFA0E1E6F900EB1
:104410001D6F206B090E1F6F0AEC28F01C511B1139
:1044200006E1000102A43E0C000102863E0C060ECD
:1044300001011C6F8F0E1B6FF30E1E6FD60E1D6FCA
:10444000206B0D0E1F6F0AEC28F01C511B1106E1AA
:10445000000102A4400C00010286400C060E01017E
:104460001C6F8F0E1B6FF90E1E6F0F0E1D6F206BD2
:104470000A0E1F6F0AEC28F01C511B1106E1000107
:1044800002A4420C00010286420C060E01011C6FC0
:104490008F0E1B6FF90E1E6F1A0E1D6F206B0A0E0A
:1044A0001F6F0AEC28F01C511B1106E1000102A449
:1044B0003F0C000102863F0C060E01011C6F8F0E9F
:1044C0001B6FF40E1E6F520E1D6F206B0C0E1F6FB4
:1044D0000AEC28F01C511B1106E1000102A4410C5A
:1044E00000010286410C060E01011C6F8F0E1B6F2E
:1044F000F10E1E6F070E1D6F206B0E0E1F6F0AEC64
:1045000028F01C511B1106E1000102A4090C000156
:104510000286090C060E01011C6F8F0E1B6FF30E35
:104520001E6FF20E1D6F206B0D0E1F6F0AEC28F030
:104530001C511B1106E1000102A42C0C0001028693
:104540002C0C060E01011C6F8F0E1B6FFA0E1E6FD6
:104550009A0E1D6F206B090E1F6F0AEC28F01C517C
:104560001B11D2E0060E01011C6F8F0E1B6FFA0E9D
:104570001E6F9E0E1D6F206B050E1F6F0AEC28F03C
:104580001C511B11C1E0060E01011C6F8F0E1B6F29
:10459000FA0E1E6FA40E1D6F206B090E1F6F0AEC22
:1045A00028F01C511B1106E1000102A4320C00018D
:1045B0000286320C060E01011C6F8F0E1B6FF90E66
:1045C0001E6F250E1D6F206B0A0E1F6F0AEC28F060
:1045D0001C511B1106E1000102A41C0C0001028603
:1045E0001C0C060E01011C6F8F0E1B6FF90E1E6F47
:1045F000300E1D6F206B0A0E1F6F0AEC28F01C5145
:104600001B1106E1000102A41D0C000102861D0C15
:10461000060E01011C6F8F0E1B6FF90E1E6F3B0EF5
:104620001D6F206B0A0E1F6F0AEC28F01C511B1126
:1046300006E1000102A41E0C000102861E0C060EFB
:1046400001011C6F8F0E1B6FF90E1E6F460E1D6F42
:10465000206B0A0E1F6F0AEC28F01C511B1106E19B
:10466000000102A41F0C000102861F0C060E0101AE
:104670001C6F8F0E1B6FF90E1E6F510E1D6F206B7E
:104680000A0E1F6F0AEC28F01C511B1106E10001F5
:1046900002A4200C00010286200C060E01011C6FF2
:1046A0008F0E1B6FF90E1E6F5C0E1D6F206B0A0EB6
:1046B0001F6F0AEC28F01C511B1106E1000102A437
:1046C000210C00010286210C060E01011C6F8F0EC9
:1046D0001B6FFF0E1E6FFD0E1D6F206B010E1F6FF7
:1046E0000AEC28F01C511B1106E1000102A4250C64
:1046F00000010286250C060E01011C6F8F0E1B6F38
:10470000FD0E1E6F6B0E1D6F206B070E1F6F0AECE8
:1047100028F01C511B1106E1000102A4260C000127
:104720000286260C060E01011C6F8F0E1B6FFE0EFB
:104730001E6F890E1D6F206B050E1F6F0AEC28F08F
:104740001C511B1106E1000102A42B0C0001028682
:104750002B0C060E01011C6F8F0E1B6FFB0E1E6FC4
:10476000A60E1D6F206B080E1F6F0AEC28F01C515F
:104770001B1106E1000102A4040C00010286040CD6
:10478000060E01011C6F8F0E1B6FFB0E1E6F9D0E20
:104790001D6F206B080E1F6F0AEC28F01C511B11B7
:1047A00006E1000102A40B0C000102860B0C060EB0
:1047B00001011C6F8F0E1B6FFB0E1E6FAF0E1D6F66
:1047C000206B080E1F6F0AEC28F01C511B1106E12C
:1047D000000102A40A0C000102860A0C060E010167
:1047E0001C6F8F0E1B6FFD0E1E6FB90E1D6F206BA1
:1047F000060E1F6F0AEC28F01C511B1106E1000188
:1048000002A4150C00010286150C060E01011C6F96
:104810008F0E1B6FFE0E1E6F7D0E1D6F206B050E23
:104820001F6F0AEC28F01C511B1106E1000102A4C5
:10483000230C00010286230C060E01011C6F8F0E53
:104840001B6FFD0E1E6FC00E1D6F206B060E1F6FBF
:104850000AEC28F01C511B1106E1000102A4130C04
:1048600000010286130C060E01011C6F8F0E1B6FD8
:10487000FD0E1E6F030E1D6F206B070E1F6F0AECDF
:1048800028F01C511B1106E1000102A4140C0001C8
:104890000286140C060E01011C6F8F0E1B6FFD0E9D
:1048A0001E6FB90E1D6F206B060E1F6F0AEC28F0ED
:1048B0001C511B11A4E0060E01011C6F8F0E1B6F13
:1048C000FA0E1E6F540E1D6F206B090E1F6F0AEC3F
:1048D00028F01C511B1106E1000102A4180C000174
:1048E0000286180C060E01011C6F8F0E1B6FFA0E4C
:1048F0001E6F5E0E1D6F206B090E1F6F0AEC28F0F5
:104900001C511B1106E1000102A4160C00010286D5
:10491000160C060E01011C6F8F0E1B6FFA0E1E6F18
:10492000680E1D6F206B090E1F6F0AEC28F01C51DA
:104930001B1106E1000102A4190C00010286190CEA
:10494000060E01011C6F8F0E1B6FFA0E1E6F720E8A
:104950001D6F206B090E1F6F0AEC28F01C511B11F4
:1049600006E1000102A41A0C000102861A0C060ED0
:1049700001011C6F8F0E1B6FFA0E1E6F7C0E1D6FD8
:10498000206B090E1F6F0AEC28F01C511B1106E169
:10499000000102A41B0C000102861B0C060E010183
:1049A0001C6F8F0E1B6FFA0E1E6F860E1D6F206B15
:1049B000090E1F6F0AEC28F01C511B1106E10001C3
:1049C00002A4170C00010286170C060E01011C6FD1
:1049D0008F0E1B6FFE0E1E6F830E1D6F206B050E5C
:1049E0001F6F0AEC28F01C511B1106E1000102A404
:1049F000270C00010286270C060E01011C6F8F0E8A
:104A00001B6FF60E1E6F380E1D6F206B0B0E1F6F87
:104A10000AEC28F01C511B1106E1000102A4280C2D
:104A200000010286280C060E01011C6F8F0E1B6F01
:104A3000F00E1E6F670E1D6F206B0F0E1F6F0AECBE
:104A400028F01C511B1106E1000102A4350C0001E5
:104A50000286350C060E01011C6F8F0E1B6FF40EC3
:104A60001E6F000E1D6F206B0D0E1F6F0AEC28F0DD
:104A70001C511B1106E1000102A4290C0001028651
:104A8000290C060E01011C6F8F0E1B6FF00E1E6F9E
:104A9000570E1D6F206B0F0E1F6F0AEC28F01C5174
:104AA0001B1106E1000102A4360C00010286360C3F
:104AB000060E01011C6F8F0E1B6FF60E1E6F2C0E63
:104AC0001D6F206B0B0E1F6F0AEC28F01C511B1181
:104AD00006E1000102A42D0C000102862D0C060E39
:104AE00001011C6F8F0E1B6FF60E1E6F140E1D6FD3
:104AF000206B0B0E1F6F0AEC28F01C511B1106E1F6
:104B0000000102A42E0C000102862E0C060E0101EB
:104B10001C6F8F0E1B6FF40E1E6F450E1D6F206BEA
:104B20000C0E1F6F0AEC28F01C511B1106E100014E
:104B300002A4300C00010286300C060E01011C6F2D
:104B40008F0E1B6FF40E1E6F5F0E1D6F206B0C0E11
:104B50001F6F0AEC28F01C511B1106E1000102A492
:104B60003C0C000102863C0C060E01011C6F8F0EEE
:104B70001B6FF30E1E6FE40E1D6F206B0D0E1F6F6B
:104B80000AEC28F01C511B1106E1000102A4310CB3
:104B900000010286310C060E01011C6F8F0E1B6F87
:104BA000F90E1E6F040E1D6F206B0A0E1F6F0AECAC
:104BB00028F01C511B1106E1000102A43D0C00016C
:104BC00002863D0C060E01011C6F8F0E1B6FFA0E44
:104BD0001E6F400E1D6F206B090E1F6F0AEC28F030
:104BE0001C511B1106E1000102A4330C00010286D6
:104BF000330C060E01011C6F8F0E1B6FFA0E1E6F19
:104C00004A0E1D6F206B090E1F6F0AEC28F01C5115
:104C10001B1106E1000102A4340C00010286340CD1
:104C2000060E01011C6F8F0E1B6FFD0E1E6FB20E64
:104C30001D6F206B060E1F6F0AEC28F01C511B1114
:104C400006E1000102A4370C00010286370C060EB3
:104C500001011C6F8F0E1B6FFD0E1E6F0B0E1D6F63
:104C6000206B070E1F6F0AEC28F01C511B1106E188
:104C7000000102A4380C00010286380C000C0496D6
:104C800004980101D96B0201D46BF76B0101A66B8B
:104C9000A76B5E0501E0BFD000010B8A9C9EA88433
:104CA0007C867D6A670EAB6E9C8E9C88A88AA49ACF
:104CB000A59AA38A8E9C8D98B3EC46F07BEC46F0C7
:104CC000590E0101295D020E2A59F8E38D88B3ECD3
:104CD00046F07BEC46F0650E0101295D000E2A5975
:104CE000F8E38E8C270E0201B36F100EB26F000135
:104CF000FC6B10D00201B351B2110CE1EF0E0101B7
:104D0000166F1F0E156F100E176F60EC45F08E9C1E
:104D10008D9812000001FC51030AECE1030E020120
:104D2000B36FE80EB26F0001FC6BFF0E0101176F4D
:104D3000A10E166F010EA3EC33F00ED00201B35199
:104D4000B2110AE1EF0E0101166F310E156F100E50
:104D5000176F60EC45F0DBD70001FC05EFE1170EA3
:104D60000201B36F700EB26F0001FC6BFB0E01010C
:104D7000176FD30E166F010EA3EC33F00ED00201A5
:104D8000B351B2110AE1EF0E0101166F430E156F18
:104D9000100E176F60EC45F0BAD70001FC05EFE18B
:104DA000EE0E0101176F1E0E166F010EA3EC33F00D
:104DB000010E01012A6FF40E296FD8EC38F0170E9E
:104DC0000201B36F700EB26F0001FC6BEC0E0101BB
:104DD000176F510E166F010EA3EC33F00ED00201C7
:104DE000B351B2110AE1EF0E0101166F550E156FA6
:104DF000100E176F60EC45F08AD70001FC51020AD3
:104E0000EEE1EF0E0101166FE20E156F100E176F37
:104E100060EC45F09DD20796198EFA0E0101176FCE
:104E2000CC0E166F010EA3EC33F04C0E01012A6F6D
:104E3000080E296FD8EC38F0ED0E0101176F230E24
:104E4000166F010EA3EC33F0130E01012A6F880ECA
:104E5000296FD8EC38F0EB0E0101176FDF0E166FDB
:104E6000010EA3EC33F0130E01012A6F880E296F97
:104E7000D8EC38F0EC0E0101176F300E166F010EF2
:104E8000A3EC33F0070E01012A6FD00E296FD8EC86
:104E900038F0880E0101296F130E2A6F000E2B6B5C
:104EA0002C6B2D6BFCEC9FF00101B46FB451400AE8
:104EB00019E0F60E176F500E166F010EA3EC33F0CB
:104EC000030E01012A6FE80E296FD8EC38F0EE0EC0
:104ED00001012C6F860E2B6F2E6B130E2D6F05ECC0
:104EE00006F0C2D0F00E176F040E166F010EA3EC81
:104EF00033F0070E01012A6FD00E296FD8EC38F07D
:104F0000880E0101296F130E2A6F000E2B6B2C6B7C
:104F10002D6BFCEC9FF00101B46FB451420A0DE01F
:104F2000F9EC3AF0EE0E01012C6FD60E2B6F2E6BC2
:104F3000120E2D6F05EC06F097D0EE0E176F1E0EB9
:104F4000166F010EA3EC33F0010E01012A6FF40E6F
:104F5000296FD8EC38F011AE33D00101B06BB051ED
:104F60005C255F6F000E5D21606F0E0E5F25D96EB0
:104F7000000E6021DA6EEB0E0101B025E16EE26AEF
:104F8000070EE222DFCFE7FFB02B060EB065E7D7B2
:104F9000F90E176FB40E166F010EA3EC33F0070E67
:104FA0000101176FEB0E166F000EA3EC33F0EC0E41
:104FB0000101176FA60E166F000EA3EC33F042D15D
:104FC000F10E0101176F250E166F010EA3EC33F0E1
:104FD000E80E0101296F030E2A6F000E2B6B2C6B5C
:104FE0002D6BFCEC9FF00101B46FB451020A0DE08F
:104FF000F9EC3AF0ED0E01012C6F830E2B6F2E6B46
:10500000130E2D6F05EC06F02FD00C8E0201DD6B18
:10501000130E01012A6F880E296FD8EC38F0FC0EB0
:105020000201DD25D96EDA6A080EDA22DF6A0C9EEB
:10503000E80E0101296F030E2A6F000E2B6B2C6BFB
:105040002D6BFCEC9FF00101B46FB4513E0A0EE0F1
:10505000F9EC3AF0ED0E01012C6F830E2B6F2E6BE5
:10506000130E2D6F05EC06F0199E5ED0B16BB26B7E
:10507000B36B37D0000E0101B125D96EDA6A090E83
:10508000DA222E0EDF622BD0FE0E5F6F080E606FED
:10509000B1515F27000E60235FC11BF160C11CF19D
:1050A00049EC19F01BC1A8F11CC1A9F1FB0E0101CB
:1050B000B125D96EDA6A080EDA22460EDF6205D013
:1050C0000C88A8C1A3F1A9C1A4F10101A851B25D46
:1050D000A951B35904E2A8C1B2F1A9C1B3F10101C8
:1050E000B12B000E0101B125D96EDA6A090EDA2260
:1050F000DF50C0E10CA853D0110EB25D000EB359C1
:1051000019E2F9EC3AF0199EA80E0301BB6FC00E2C
:10511000BA6FEF0E01012C6FF30E2B6F2E6B100E7A
:105120002D6F05EC06F057D0000119A21200000EF9
:1051300068EF37F0090E0101376F000E366FFF0E72
:10514000396F430E386FB2C13AF1B3C13BF130EC65
:105150003DF0B351A41902E1B251A31908E1F00ED8
:10516000176F150E166F010EA3EC33F007D0F00E7B
:10517000176F870E166F010EA3EC33F0090E0101B5
:10518000176F000E166F000EA3EC33F0EC0E01014A
:10519000176FA60E166F000EA3EC33F053D007B4B2
:1051A00002D011AA41D0110E0101B25D000EB35917
:1051B00014E2F9EC3AF0199EA80E0301BB6FC00E81
:1051C000BA6FEF0E01012C6FF30E2B6F2E6B100ECA
:1051D0002D6F05EC06F0119AA7D7090E0101376F64
:1051E000000E366FFF0E396F430E386FB2C13AF1C1
:1051F000B3C13BF130EC3DF0F00E176F870E166F28
:10520000010EA3EC33F0090E0101176F000E166FAB
:10521000000EA3EC33F0EC0E0101176FA60E166F13
:10522000000EA3EC33F00ED007B40CD0000111BA7D
:1052300009D0F9EC3AF0199EA80E0301BB6FC00E1D
:10524000BA6FC00C119A030E01012A6FE80E296F84
:10525000D8EC38F0880E0101296F130E2A6F000E6A
:105260002B6B2C6B2D6BFCEC9FF00101B46FB451D8
:105270003F0A15E0F9EC3AF0EE0E01012C6F090E31
:105280002B6F2E6B140E2D6F05EC06F0000119A28A
:1052900003D0000E68EC37F00001199E1200F9EC03
:1052A0003AF0030E01012A6FE80E296FD8EC38F0AE
:1052B000500E0101186FE70E176F460E196FD6ECEE
:1052C00036F0500E0101186FE80E176F4C0E196F73
:1052D000D6EC36F0500E0101186FE90E176F530E21
:1052E000196FD6EC36F0500E0101186FEA0E176FE9
:1052F000310E196FD6EC36F0EC0E01012C6F8B0ECF
:105300002B6F2E6B1A0E2D6F05EC06F0030E0101AC
:105310002A6FE80E296FD8EC38F0F80E0101176FEC
:10532000B40E166F010EA3EC33F0030E01012A6FC9
:10533000E80E296FD8EC38F01284070E0301BD6F18
:10534000D00EBC6F000119A2D00C010E68EF37F02F
:105350000D9C10D001015E0506E1FA0E166FC20E1B
:10536000156F090E0CD1FA0E2C6FC20E2B6F2E6B1F
:10537000090E0CD15CC11DF15DC11EF13C0E010195
:105380001F6F5EC120F138EC37F00101B56FB5C178
:10539000A9FFA8A2FED71BBADDD70101B5513A0A71
:1053A000E9E1A64BA72B5CC127F15DC128F10A0EEC
:1053B000296F5EC12AF185EC3EF0B56F1BBACAD7E2
:1053C000B5C1ABF1ABC1D0F25CC127F15DC128F131
:1053D0000A0E0101296F5EC12AF185EC3EF0B56F1E
:1053E0001BBAB8D70101B551606F5F6B616B60513B
:1053F000626F61C1ACF162C1ADF1AE6BAF6B5CC10C
:1054000027F15DC128F10A0E296F5EC12AF185ECF2
:105410003EF0B56F1BBA9ED70101B551AC135CC10C
:1054200027F15DC128F10A0E296F5EC12AF185ECD2
:105430003EF0A56F1BBA8ED704A892D10101D89077
:10544000AE2B000EAF238CD15CC127F15DC128F1DA
:105450000A0E296F5EC12AF185EC3EF0AA6F1BBAD5
:1054600079D70101AF51AC11AD11AE1117E10B0E9F
:105470005C255F6F000E5D21606F5FC11BF160C135
:105480001CF1FB0E1E6FE50E1D6F206B080E1F6FCB
:105490000AEC28F01C511B1101E00D800101AD51F7
:1054A000040A600ED8B4AC19AE11AF1117E1090EA1
:1054B0005C255F6F000E5D21606F5FC11BF160C1F5
:1054C0001CF1FF0E1E6F340E1D6F206B040E1F6F3C
:1054D0000AEC28F01C511B1101E007820101AF51B9
:1054E000800A800F08E1010EAE5D05E1EC0EAD5DB6
:1054F00002E1010EAC5D01E3188C0101AC2B000E42
:10550000AD23AE23AF23AB070101AB299DE15CC105
:105510002DF15DC12EF10A0E2F6F5EC130F1A5ECA9
:1055200036F001E304861BBA15D724D75CC12DF1F0
:105530005DC12EF10A0E2F6F5EC130F1A5EC36F081
:1055400001E304861BBA06D704A610D001015E054C
:1055500006E1FB0E166FCA0E156F080E10D0FB0E7B
:105560002C6FCA0E2B6F2E6B080E10D00DA011D011
:1055700001015E0507E1F90E166F720E12D0176F6A
:1055800060EF45F0F90E2C6F720E11D02D6F05EF04
:1055900006F007A210D001015E0506E1F90E166FB4
:1055A0007D0E156F0A0EEBD7F90E2C6F7D0E2B6F4B
:1055B0002E6B0A0EEBD718AC10D001015E0506E188
:1055C000F10E166F160E156F0E0ED9D7F10E2C6F49
:1055D000160E2B6F2E6B0E0ED9D70101010E376FF1
:1055E000630E366FEC0E396F0E0E386FA6C13AF1AE
:1055F000A7C13BF130EC3DF03651B56F5E0515E1CA
:10560000010E166F630E156FB5C117F160EC45F012
:10561000270E0101A76F100EA66FA607D8A0A70737
:105620000101A751A6111CE0F8D7010E2C6F630EE3
:105630002B6FB5C12DF12E6B05EC06F0EC0E0101C0
:105640002C6F130E2B6F2E6B1C0E2D6F05EC06F0BE
:10565000F80E0101176FB40E166F010EA3EC33F0B4
:105660000B0E01012A6FB80E296FD8EC38F0500EDE
:105670000101186FE70E176F460E196FD6EC36F062
:10568000500E0101186FE80E176F4C0E196FD6EC13
:1056900036F0500E0101186FE90E176F530E196F97
:1056A000D6EC36F0500E0101186FEA0E176F300E6F
:1056B000196FD6EC36F0130E01012A6F880E296F90
:1056C000D8EC38F0FF001200AA6B0DD05CC127F1B6
:1056D0005DC128F10A0E296F5EC12AF185EC3EF00A
:1056E000AA131BBA37D60101AB07AB29EFE1AA51C8
:1056F000F00B100A02E1048801D004985CC12DF17E
:105700005DC12EF10A0E01012F6F5EC130F1A5ECD3
:1057100036F007D75CC127F15DC128F10A0E296F69
:105720005EC12AF185EC3EF0AA6F1BBA13D60101C7
:10573000AB07AB29EFE1AAC15FF10F0E5F175F0561
:1057400002E1048801D004985CC12DF15DC12EF105
:105750000A0E01012F6F5EC130F1A5EC36F0E1D6E3
:105760000101A55101E1CFD6010A01E1DFD6030A0B
:10577000ABE0060ADCE0FED50301BD51BC1103E03D
:10578000BC07D8A0BD070201B351B21103E0B207B4
:10579000D8A0B30704009E90D10ECF6E200ECE2667
:1057A0000301AE4BAF2BB64BB72B05010A2B000EF6
:1057B0000B230C230D230301B24BB32B13A409D0ED
:1057C0001394030E216EEF0E206E14EC25F08F80E3
:1057D000138A0401F551F41108E0F407D8A0F50785
:1057E000F551F41102E10201E86B0401EF51EE11F1
:1057F00003E0EE07D8A0EF070301A84BA92BA9519E
:10580000800A286EA651A85DA751800A285801E396
:105810001D8C0401D607D8A0D707D751D61102E1B5
:1058200010AE119214A20AD00301DE2B040EDE6525
:1058300005D0DE6B00011484FFEC3DF00301D1675D
:105840000AD00CA007BC07D015BA12B004D012B809
:1058500002D08D8A8D9C0301D15119E00201EC51D7
:1058600002E0EC073ED00BBE06D08D9A8D9C020163
:10587000EC690B8E36D08D9A8D8C0201EC690B9EF3
:105880000301D107D1672DD08D8A8D9C2AD012A813
:1058900012D00201ED2B270EED6523D0ED6B8D8C20
:1058A0008D8A0301D42BD451050A1BE18D9C8D9A5E
:1058B000D46B129816D00CA007D00201ED2B310E3C
:1058C000ED6502D0ED6B0CD007AC0BD00401F64BAC
:1058D000F72BE80EF65D030EF75903E3F66BF76B53
:1058E0008D7A13A808D00301DB2B310EDB6503D0C2
:1058F000DB6B13988F900CA20ED00301E02B310EBE
:10590000E06509D0E06B8F70DF2B3B0EDF6503D0C5
:10591000DF6B0C928F900CA410D00301E32B310E9F
:10592000E3650BD0E36B8F70E22B3B0EE26505D095
:10593000E26B8F900C941AB60C8413AA08D0030162
:10594000DC2B310EDC6503D0DC6B139A8F900201E7
:10595000EB2B1D0EEB6505D0EB6B0301E56B020134
:10596000EA6B46B409D20301E12B180EE16504D2BB
:10597000E16B0101E56BB8C323F0B9C324F053EC2C
:1059800028F00101E76F14B20AAE06D00201F95106
:10599000E00B0101E71905D00101E7510201F919F6
:1059A0000101E56FEDC31FF0E55196EC30F0296E73
:1059B000295001E18DD014AE8AD029A015D014A2AF
:1059C00005D00101E5513BEC2BF00ED00101E5A122
:1059D00006D0206A220E1F6E91EC1BF005D0206AC3
:1059E000240E1F6E91EC1BF029A215D014A205D035
:1059F0000101E551FCEC25F00ED00101E5A306D034
:105A0000206A260E1F6E91EC1BF005D0206A280E2E
:105A10001F6E91EC1BF029A415D014A205D0010132
:105A2000E551FAEC2AF00ED00101E5A506D0206A76
:105A30002A0E1F6E91EC1BF005D0206A2C0E1F6EF3
:105A400091EC1BF029A615D014A205D00101E55157
:105A50007CEC2BF00ED00101E5A706D0206A2E0EBB
:105A60001F6E91EC1BF005D0206A300E1F6E91EC7A
:105A70001BF029A815D014A205D00101E551FEECB8
:105A80002BF00ED00101E5A906D0206A360E1F6E5C
:105A900091EC1BF005D0206A380E1F6E91EC1BF0C4
:105AA00029AA15D014A205D00101E551CAEC45F090
:105AB0000ED00101E5AB06D0206A900E1F6E91EC6E
:105AC0001BF005D0206A920E1F6E91EC1BF0148E15
:105AD000E5C1EDF3E5C1E6F115A007D00001159091
:105AE000206A400E1F6E91EC1BF007AE07D000013C
:105AF000079E206A320E1F6E91EC1BF008A007D0A3
:105B000000010890206A340E1F6E91EC1BF01BA858
:105B10000CD000011B98206A440E1F6E91EC1BF004
:105B200013BC03D00FA60FB8128611AC07D000012A
:105B3000119C206A3E0E1F6E91EC1BF016AC07D034
:105B40000001169C206A460E1F6E91EC1BF00DA8FA
:105B500007D000010D98206A880E1F6E91EC1BF093
:105B60000DA208D000010D92020E206EB40E1F6E21
:105B700091EC1BF00FA007D000010F90206A8E0E51
:105B80001F6E91EC1BF00EAE08D000010E9E020EAF
:105B9000206EB60E1F6E91EC1BF008AC07D0000112
:105BA000089C206A960E1F6E91EC1BF014A607D07D
:105BB00000011496206A3A0E1F6E91EC1BF014A897
:105BC00007D000011498206A3C0E1F6E91EC1BF068
:105BD00017B6179617AE07D00001179E206A8C0ED5
:105BE0001F6E91EC1BF017AA0AD0179A000118B883
:105BF00006D0020E206EB80E1F6E91EC1BF018A29C
:105C000008D000011892020E206EBA0E1F6E91ECA1
:105C10001BF00201CC510AE0DE0ECC251F6E206A7B
:105C2000020E202291EC1BF00201CC6B0AA807D0D7
:105C300000010A98206A200E1F6E91EC1BF00BA643
:105C400007D000010B96206A860E1F6E91EC1BF0A8
:105C50000BA007D000010B90206A940E1F6E91ECF0
:105C60001BF0010E05A0000E286E010E04AE000E02
:105C7000281A15E0060E04BE070E0301F96F990EEF
:105C8000FA6FFB6F850EFC6F490EFD6F900EFE6F75
:105C9000050EFF6F168E168C059004BE058002015E
:105CA000C76722D014BE0CBA1FD006A003D006B41A
:105CB00051D052D006AC03D007B04CD04DD00DAE71
:105CC00003D00EB247D048D00DA403D00DBA42D0B5
:105CD00043D008A403D008B83DD03ED01AA804D0C1
:105CE0000201F35137E138D000F00201C86741D01A
:105CF000000114AE3ED000010CBC3BD006A204D083
:105D0000000106B42FD030D006AE04D0000107B099
:105D100029D02AD00EA004D000010EB223D024D066
:105D20000DB614A204D0000106BA1CD01DD00DA6D9
:105D300004D000010DBA16D017D008A604D0000177
:105D400008B810D011D000011AAA13D00201F451E2
:105D500009E10AD08A8C02D08A9CC6D7030E0201C0
:105D6000C76FC2D78A8E02D08A9E03D0030E02016B
:105D7000C86F00F00CEC3DF012BC02D012AE03D0A4
:105D80000201DB6B03D0010E0201DB6F0401E24B69
:105D9000E32BE051E25DE151E35934E3E26BE36B65
:105DA0000201DB6708D018B403D08A988A962AD0FB
:105DB0008D968D9427D0DB0525E11EA016D01E9070
:105DC00018B408D018B003D08A988A860AD08A8876
:105DD0008A9607D017B803D08D968D8402D08D8611
:105DE0008D940401E16B640E0CD01E8018B403D0B6
:105DF0008A988A9602D08D968D941F0E0401E16FC9
:105E0000400EE06F0401E64BE72BE451E65DE551FF
:105E1000E75960E3E66BE76B04B002D00301D66B91
:105E20000301D66723D01EA20CD01E9218B403D053
:105E30008D868D9402D08A888A960401E56B640E63
:105E400013D01E8218B403D08D968D9402D08A98F8
:105E50008A9604B005D0010E0401E56F900E04D0BF
:105E6000090E0401E56FC40EE46F34D0D60512E1CB
:105E70001EA22AD01E9218B403D08D868D9402D013
:105E80008A888A9613BCECD7D8D78A988A9613BC8E
:105E9000D4D7E6D7D651020A0AE11EA215D01E9227
:105EA00018B402D08D860CD08A888A86EBD7D6515A
:105EB000030A10E11EA208D01E9218B403D08D96DA
:105EC0008D84E0D78A98F1D71E8218B4DED78D96DC
:105ED0008D94DDD712A004D08D968D948A988A96E1
:105EE0000401F04BF12BE80EF05D030EF15969E36C
:105EF0000201F351D8A4F307F451D8A4F407040124
:105F0000F06BF16BE84BE92B000112A096EC11F05D
:105F10000301DD0714A206D00201CD5103E0CD2F0D
:105F200001D01B840501FE51D8A4FE070201F851DF
:105F3000D8A4F80719BE0DD0E151E22BE25D02E3CF
:105F4000E26B15860301CD2B1D0ECD6502D0CD6B06
:105F50001A8C1AAE08D0580E0401DA5D020EDB5915
:105F600002E2DA4BDB2B06A60AD00401D951D81184
:105F700003E18A9C069603D0D807D8A0D9071BACAA
:105F800009D00401F951F81102E11B9C03D0F80774
:105F9000D8A0F90714A00AD00401F351F21103E1CB
:105FA0008A9E149003D0F207D8A0F3070201C751CC
:105FB000D8A4C707C851D8A4C8070301D751D8A48B
:105FC000D7070401EC4BED2B600EEC5DEA0EED59AA
:105FD000D8A01200EC6BED6B0301BB51BA1103E0CA
:105FE000BA07D8A0BB07BA05BB1104E107860301B5
:105FF000BA6BBB6BE72B14A208D00201CA5105E0B3
:10600000CA2F03D0099008BE8A9C0101DD5102010C
:10601000E62BE65D02E3E66B1B820201DE51030123
:10602000D92BD95D02E3D96B1B800201CF2B020E65
:10603000CF6501D0CF6B0401EA4BEB2B0A0EEA5D72
:10604000000EEB591AE3EA6BEB6B0301D02B8F0EBA
:10605000D06502D0D06B09880201F251F12BF15DBD
:106060000CE3F16B1B88188A1AA802D0140EF36F88
:106070001AAA03D0140E0201F46F0201E52B020EDE
:10608000E565020CE56B0001148A12000101266B24
:10609000500E01012625D96EDA6A060EDA22265143
:1060A000186F196B18BF1907E5EC2FF0DF6E262B60
:1060B0002651800A610FECE3266B000E01012625B4
:1060C000D96EDA6A050EDA22800E90DBE5EC2FF04D
:1060D000DF6E262B2651800A7A0FEFE3196B550EDF
:1060E000186FE5EC2FF00201F26F0101196B4B0EF6
:1060F000186FE5EC2FF0236F226B196B4A0E186FA7
:10610000E5EC2FF022110301B86F010123510301C7
:10611000B96F0101196B520E186FE5EC2FF00201F7
:10612000F96F0101196B560E186FE5EC2FF00201A3
:10613000D16F0101196B570E186FE5EC2FF00301B9
:10614000C46F0101196B760E186FE5EC2FF0DC6F50
:10615000196B590E186FE5EC2FF0236F226B196B3A
:106160005A0E186FE5EC2FF02211CF6F2351D06F2C
:10617000196B4F0E186FE5EC2FF0266F1E9601017C
:1061800026B51E861E9826B71E88266B85DB9A0EBE
:1061900021DBE5EC2FF0DF6E7FDBDF5005E0262B07
:1061A0002651800A700FF2E30101266B5DDBBA0E07
:1061B00011DBE5EC2FF0DF6E57DBDF5005E0262B1F
:1061C0002651800A7B0FF2E31E9A0701CB5104E0AF
:1061D0000601F15101E01E8A0101196B750E186F5D
:1061E000E5EC2FF0266F179C010126B1178C1A9051
:1061F00026B31A80119426B71184079426BF07840A
:10620000129226BD12821A9226B51A820C9A069014
:10621000069C0D9E0D9408941A980C9C0692069E5E
:106220000E900D9608961A9A196B4C0E186FE5ECA5
:106230002FF0266F266702D00C8A18D026B1FCD723
:1062400026A302D0068012D026A502D0068C0ED03E
:1062500026A702D00D8E0AD026A902D00D8406D022
:1062600026AB02D0088402D026BD1A880101196B22
:106270004D0E186FE5EC2FF0266F266702D00C8CC0
:1062800018D026B1FCD726A302D0068212D026A5AC
:1062900002D0068E0ED026A702D00E800AD026A9E4
:1062A00002D00D8606D026AB02D0088602D026BDCD
:1062B0001A8A030E0101196F500E186FE5EC2FF0CA
:1062C000236F226B030E196F510E186FE5EC2FF040
:1062D00022110201B86F010123510201B96F030EAF
:1062E0000101196F520E186FE5EC2FF0236F226B2E
:1062F000030E196F530E186FE5EC2FF022110201F7
:10630000BA6F010123510201BB6F030E0101196F26
:10631000540E186FE5EC2FF0236F226B030E196FEC
:10632000550E186FE5EC2FF022110201BC6F010130
:1063300023510201BD6F030E0101196F560E186F34
:10634000E5EC2FF0236F226B030E196F570E186FB9
:10635000E5EC2FF022110201BE6F01012351020171
:10636000BF6F030E0101196F580E186FE5EC2FF087
:10637000236F226B030E196F590E186FE5EC2FF087
:1063800022110201C06F010123510201C16FE80E09
:10639000B85D030EB95917E3030E0101186F500ED3
:1063A000176F030E196FD6EC36F0030E0101186F4C
:1063B000510E176F3E0E196FD6EC36F0030E020128
:1063C000B96F3E0EB86FE80EBA5D030EBB5917E306
:1063D000030E0101186F520E176F030E196FD6ECE2
:1063E00036F0030E0101186F530E176F3E0E196F32
:1063F000D6EC36F0030E0201BB6F3E0EBA6FE80E0C
:10640000BC5D030EBD5917E3030E0101186F540E56
:10641000176F030E196FD6EC36F0030E0101186FDB
:10642000550E176F3E0E196FD6EC36F0030E0201B3
:10643000BD6F3E0EBC6FE80EBE5D030EBF5917E385
:10644000030E0101186F560E176F030E196FD6EC6D
:1064500036F0030E0101186F570E176F3E0E196FBD
:10646000D6EC36F0030E0201BF6F3E0EBE6FE80E93
:10647000C05D030EC15917E3030E0101186F580EDA
:10648000176F030E196FD6EC36F0030E0101186F6B
:10649000590E176F3E0E196FD6EC36F0030E02013F
:1064A000C16F3E0EC06F0101196B6C0E186FE5ECE9
:1064B0002FF0E16F1C940101E1B71C84070EE11776
:1064C000196B680E186FE5EC2FF0E26F1C9E01014E
:1064D000E2B71C8E070EE217196B690E186FE5EC18
:1064E0002FF0E36F1D940101E3B71D84070EE3173E
:1064F000196B6A0E186FE5EC2FF0E46F1D9A01011D
:10650000E4B71D8A070EE417196B540E186FE5ECFB
:106510002FF0266F2651F00B09E1069A199626C135
:1065200022F10F0E01012217222924D02651F00B4F
:10653000100A0EE1068A199626C122F10F0E0101FA
:1065400022172229D46F0301AD6B010EAC6F14D05A
:106550002651F00B200A03E1069A1986E0D726514E
:10656000F00B300A03E1068A1986E6D7069A0798E7
:106570001996010E0201CB6F1CA41CBE04D01DB4E1
:1065800002D01DAA02D0198801D019980101196BF7
:10659000640E186FE5EC2FF00201D56F0101196B45
:1065A000650E186FE5EC2FF00201D66F0101196B33
:1065B000660E186FE5EC2FF00201D96F0101196B1F
:1065C000670E186FE5EC2FF00201D26F0101196B15
:1065D0006B0E186FE5EC2FF0266F109E010126B1AF
:1065E000108E0A9E26B50A8E089E14A207D0088E29
:1065F0000C9A0690069C0D9E0D9408940101196B4F
:10660000700E186FE5EC2FF00201E16F0101196BBC
:10661000720E186FE5EC2FF0DD6F196B710E186FAD
:10662000E5EC2FF00301D56F0101196B730E186FA4
:10663000E5EC2FF00201DE6F0101266BE0D88A0E37
:10664000C9D8E5EC2FF0DF6EDAD8DF5005E0262B55
:106650002651800A700FF2E30F980501D55107E02B
:10666000E0D80AEC28F01C511B1101E00F88010151
:10667000266BC5D8CD0EBAD8E5EC2FF0DF6EBFD8AB
:10668000DF5005E0262B2651800A700FF2E30F96AB
:106690000501D55107E0C5D80AEC28F01C511B11A3
:1066A00001E00F860101266BD0D8B30E9FD8E5EC30
:1066B0002FF0DF6ECAD8DF5005E0262B2651800A66
:1066C000700FF2E30101266BEFD8DD0E8FD8E5ECF9
:1066D0002FF0DF6EE9D8DF5005E0262B2651800A27
:1066E000700FF2E30101256B980E246F18A404D0FB
:1066F000030E256F200E246F0101266B9FD887D8CB
:10670000E5EC2FF0DF6E9AD8DA22DF5005E0262B79
:106710002651800A650FF2E30101256BED0E246F0F
:1067200018A404D0030E256F3B0E246F0101266BC5
:1067300094D86DD8E5EC2FF0DF6E8FD8DA22DF50D9
:1067400005E0262B2651800A770FF2E30101256B25
:10675000F60E246F18A404D0030E256F440E246F88
:106760000101266BA9D853D8E5EC2FF0DF6EA4D831
:10677000DA22DF5005E0262B2651800A770FF2E35C
:106780000101266B79D8550E25D8E5EC2FF0DF6E88
:1067900073D8DF5005E0262B2651800A600FF2E304
:1067A0000101266B71D8750E15D8E5EC2FF0DF6E60
:1067B0006BD8DF5005E0262B2651800A700FF2E3DC
:1067C000420E0101196F3A0E186FE5EC2FF002012D
:1067D000F66F1200226F010E236F22512625186FCB
:1067E000000E26BFFF0E2321196F12002625186FF9
:1067F000E86AD8B0E82A26BFE806196F1200D50E5D
:1068000001012625D96EDA6A050EDA221200DA2293
:1068100024512625186F000E26BFFF0E2521196F63
:106820001200050E01011C6FD50E1B6FFC0E1E6FB2
:10683000DB0E1D6F206B070E1F6F070C700E010122
:106840002625D96EDA6A070E1200BB0E0101262535
:10685000D96EDA6A070EDA221200DF0E0101262550
:10686000D96EDA6A060E1200F10E01012625D96EE4
:10687000DA6A060EDA221200500E01012625D96EC0
:10688000DA6A070EDA221200AB0E01012625D96E54
:10689000DA6A070EDA221200CB0E01012625D96E24
:1068A000DA6A070EDA221200DB0E01012625D96E04
:1068B000DA6A070EDA221200E80E01012625D96EE7
:1068C000DA6A060E1200E8CF97F2020197050FE18F
:1068D000020E0101166F500E156FFDEC40F0020123
:1068E000966F966701D01200E56B149A28D0966BCC
:1068F00014D002019651800A400F21E21F0E962506
:10690000D96EDA6A050EDA22500E9625E16EE26A39
:10691000020EE222DFCFE7FF962BD3C5B6F10101CD
:10692000B76B96C2B8F1B96BB8BFB907B951800A55
:10693000BA6FB651B85DB751800ABA59DAE30201AD
:10694000E56B149A970567E1020E01011C6F500E6A
:106950001B6FFE0E1E6FC50E1D6F206B050E1F6F89
:106960000AEC28F01C511B1118E1130E696F6A0E16
:10697000686F6B6B1E0E6A6F020E01016D6F500E19
:106980006C6F97C26EF10BECC7F001016951681191
:1069900004E1020197512BEC43F0020E01011C6F40
:1069A000500E1B6FFB0E1E6FDC0E1D6F206B080E52
:1069B0001F6F0AEC28F01C511B112DE1130E186FEC
:1069C0006A0E176F000E196BD6EC36F0130E01012C
:1069D000186F790E176F000E196BD6EC36F00101A7
:1069E000196B750E186FE5EC2FF00201906F905146
:1069F000F70B916F0101186B750E176F91C219F1AA
:106A0000D6EC36F0F00E0101166F770E156F0F0EF3
:106A1000176F60EC45F00201970529E1020E0101B4
:106A20001C6F500E1B6FFE0E1E6FBF0E1D6F206B76
:106A3000050E1F6F0AEC28F01C511B1118E1186B92
:106A4000FF0E17691969D6EC36F04F0E0101186F69
:106A5000D60E176F000E196BD6EC36F0ED0E010155
:106A6000166F9A0E156F160E176F60EC45F0020E3A
:106A700001011C6F500E1B6FFE0E1E6FB30E1D6FBB
:106A8000206B050E1F6F0AEC28F01C511B1149E109
:106A900014A202D006BAB9D24F0E0101196FD30E5B
:106AA000186FE5EC2FF0B66FB6AD2BD0020E0101DA
:106AB000376F500E366FF40E396F860E386F130E27
:106AC0003B6FFC0E3A6F30EC3DF036510201966F91
:106AD000975109E0020E0101166F500E156F96C214
:106AE00017F160EF45F0020E01012C6F500E2B6F75
:106AF0000201965101012D6F2E6B2DBF2E0705EF60
:106B000006F0020E0101376F500E366FF40E396F2A
:106B1000790E386F130E3B6FFC0E3A6F30EC3DF080
:106B2000D4D7020E01011C6F500E1B6FABEC1CF092
:106B30001BC194F21CC195F24F0E196FD50E186F40
:106B4000E5EC2FF0B66F4F0E196FD40E186FE5EC11
:106B50002FF00201936F0101B6510201926F550EA1
:106B60000101B66F020EB76FB6C11BF1B7C11CF1C0
:106B7000FE0E1E6FA70E1D6F206B050E1F6F0AEC19
:106B800028F01C511B1121E102019351951902E1DA
:106B90009251941901E0C1D04F0E0101196FD30E2B
:106BA000186FE5EC2FF00201966F3F0E96174F0E0F
:106BB0000101186FD30E176F96C219F1D6EC36F09B
:106BC00002019751FFEC42F097D0550EB66F020EBE
:106BD000B76FB6C11BF1B7C11CF1FE0E1E6FAD0E33
:106BE0001D6F206B050E1F6F0AEC28F01C511B1146
:106BF00020E102019351951902E19251941901E0AB
:106C00008CD04F0E0101196FD30E186FE5EC2FF0E9
:106C10000201966F968D4F0E0101186FD30E176FFC
:106C200096C219F1D6EC36F002019751FFEC42F012
:106C300063D0550EB66F020EB76FB6C11BF1B7C168
:106C40001CF1FE0E1E6FB90E1D6F206B050E1F6F1F
:106C50000AEC28F01C511B114FE102019651800AE9
:106C6000720F06E39351951902E19251941901E0D4
:106C700054D00A0E966F500E9625D96EDA6A020E1F
:106C8000DA22DF50800A500F0AE3500E9625D96EA3
:106C9000DA6A020EDA22DF50800A460F01E33DD0A5
:106CA000962B9651800A720FE6E35E6B5A0E010135
:106CB000B66F020EB76FB6C11BF1B7C11CF1ABECDA
:106CC0001CF01BC194F21CC195F24F0E186FD40E2C
:106CD000176F020195510101196FD6EC36F04F0E76
:106CE0000101186FD50E176F94C219F1D6EC36F06A
:106CF00002019751FFEF42F04F0E0101196FD30EC1
:106D0000186FE5EC2FF0B66FB6AD0AD002019351C3
:106D1000951902E19251941903E09751D3EF42F093
:106D2000550E0101B66F020EB76FB6C11BF1B7C1A8
:106D30001CF1FF0E1E6F480E1D6F206B040E1F6F9F
:106D40000AEC28F01C511B1141E146B604D00001A9
:106D500013A085EC08F00101696B686B040E6B6F82
:106D60006A6B020E6D6F500E6C6F97C26EF10BEC7A
:106D7000C7F001016951681104E1020197512BEC40
:106D800043F0000146B61200010E0101186F000E1B
:106D9000176B196BD6EC36F0010E0101186F110E4E
:106DA000176F000E196BD6EC36F0010E0101186F4B
:106DB000220E176F000E196BD6EC36F0010E010192
:106DC000186F330E176F196BD6EF36F0550EB66F7E
:106DD000020EB76FB6C11BF1B7C11CF1FF0E1E6FDB
:106DE000520E1D6F206B040E1F6F0AEC28F01C5111
:106DF0001B1111E1040E696F686B0D0E6B6FE80ECD
:106E00006A6F020E01016D6F500E6C6F97C26EF1CA
:106E10000BECC7F06FD0550EB66F020EB76FB6C150
:106E20001BF1B7C11CF1FF0E1E6F5C0E1D6F206BB6
:106E3000040E1F6F0AEC28F01C511B1112E1130EF7
:106E4000696F880E686F2E0E6B6FB30E6A6F020E3D
:106E500001016D6F500E6C6F97C26EF10BECC7F0B5
:106E600049D0550EB66F020EB76FB6C11BF1B7C150
:106E70001CF1FF0E1E6F390E1D6F206B040E1F6F6D
:106E80000AEC28F01C511B1112E1420E696F3B0EF7
:106E9000686F0B0E6B6FB80E6A6F020E01016D6F9B
:106EA000500E6C6F97C26EF10BECC7F023D0550EED
:106EB000B66F020EB76FB6C11BF1B7C11CF1FF0E62
:106EC0001E6F570E1D6F206B040E1F6F0AEC28F00B
:106ED0001C511B1118E1510E696F686B2F0E6B6FFF
:106EE0006A6B020E01016D6F500E6C6F97C26EF1EE
:106EF0000BECC7F0010169516811D8A4120002011E
:106F000097512BEF43F0550EB66F020EB76FB6C117
:106F10001BF1B7C11CF1FE0E1E6FCB0E1D6F206B57
:106F2000050E1F6F0AEC28F01C511B111AE114A268
:106F300002D006BA6AD0020197050AE0EC0E010100
:106F40002C6FC00E2B6F2E6B180E2D6F05EF06F0F9
:106F5000020E01015D6F500E5C6F97C25EF13FEF54
:106F6000A6F0550EB66F020EB76FB6C11BF1B7C1D2
:106F70001CF1FB0E1E6FEE0E1D6F206B080E1F6FB7
:106F80000AEC28F01C511B1106E114A202D006BA2B
:106F90003CD0118EDDD7550EB66F020EB76FB6C15D
:106FA0001BF1B7C11CF1FC0E1E6FE40E1D6F206BB0
:106FB000060E1F6F0AEC28F01C511B1106E114A2EB
:106FC00002D006BA22D0118AC3D7550EB66F020E70
:106FD000B76FB6C11BF1B7C11CF1FF0E1E6F4D0E8E
:106FE0001D6F206B040E1F6F0AEC28F01C511B1143
:106FF00010E114A202D006BA08D001017D6B7C6BAF
:10700000040E7F6F7E6B020E20D00201975157EF66
:1070100043F0550EB66F020EB76FB6C11BF1B7C184
:107020001CF1FF0E1E6F610E1D6F206B040E1F6F93
:107030000AEC28F01C511B110FE1130E7D6F880E16
:107040007C6F2E0E7F6FB30E23D0816F500E806F3A
:1070500097C282F1BBEFD1F0550EB66F020EB76F3B
:10706000B6C11BF1B7C11CF1FF0E1E6F3E0E1D6FA6
:10707000206B040E1F6F0AEC28F01C511B11D8A4C2
:107080001200420E7D6F3B0E7C6F0B0E7F6FB80EB1
:107090007E6F020E0101D9D7E8CF46F101014E6B98
:1070A000010E4D6F96DB446F44390F0BFDEC44F03D
:1070B000DF6E4E2B8EDB0F0BFDEC44F0DF6E4E2BA4
:1070C0004D2B020E4D65EED7470E4E25D96EDA6A6E
:1070D000010EDA22DF6A46C14EF1C451310A0CE1D9
:1070E00070DBF20E396F150E386F010E3B6F470ED5
:1070F0003A6F30EC3DF049D3C451910A0CE161DBA9
:10710000F20E396F240E386F010E3B6F470E3A6F47
:1071100030EC3DF03AD3C451320A0CE152DBF20EAE
:10712000396F7E0E386F010E3B6F470E3A6F30ECB1
:107130003DF02BD3C451920A0CE143DBF20E396FC0
:107140008D0E386F010E3B6F470E3A6F30EC3DF0FD
:107150001CD3C451330A0CE134DBF20E396FE70E55
:10716000386F010E3B6F470E3A6F30EC3DF00DD398
:10717000C451930A0CE125DBF20E396FF60E386F1D
:10718000010E3B6F470E3A6F30EC3DF0FED2C4511A
:10719000340A0CE116DBF30E396F140E386F010E52
:1071A0003B6F470E3A6F30EC3DF0EFD2C451940A7A
:1071B0000CE107DBF30E396F230E386F010E3B6FC6
:1071C000470E3A6F30EC3DF0E0D2C451990A0CE121
:1071D000F8DAF30E396F410E386F010E3B6F470E30
:1071E0003A6F30EC3DF0D1D2C451390A0CE1E9DA02
:1071F000F30E396F500E386F010E3B6F470E3A6F2A
:1072000030EC3DF0C2D2C451890A0CE1DADAF30E57
:10721000396F5F0E386F010E3B6F470E3A6F30ECDF
:107220003DF0B3D2C451900A0CE1CBDAF30E396FC2
:107230006E0E386F010E3B6F470E3A6F30EC3DF02B
:10724000A4D2C451980A0CE1BCDAF10E396FCA0E0F
:10725000386F010E3B6F470E3A6F30EC3DF095D220
:10726000C451350A0CE1ADDAF10E396F7F0E386F7B
:10727000010E3B6F470E3A6F30EC3DF086D2C451A1
:10728000950A0CE19EDAF10E396F8E0E386F010E01
:107290003B6F470E3A6F30EC3DF077D2C451960AFF
:1072A0000CE18FDAF10E396F9D0E386F010E3B6FD6
:1072B000470E3A6F30EC3DF068D2C451380A0CE109
:1072C00080DAF10E396FBB0E386F010E3B6F470E3F
:1072D0003A6F30EC3DF059D2C451710A0CE171DAC9
:1072E000F10E396FAC0E386F010E3B6F470E3A6FDF
:1072F00030EC3DF04AD2C451850A0CE162DAF20E5C
:10730000396F510E386F010E3B6F470E3A6F30ECFC
:107310003DF03BD2C451880A0CE153DAF20E396FCA
:10732000BA0E386F010E3B6F470E3A6F30EC3DF0EE
:107330002CD2C451460A0CE144DAF30E396F050E23
:10734000386F010E3B6F470E3A6F30EC3DF01DD2A7
:10735000C451450A0CE135DAF30E396F320E386F3D
:10736000010E3B6F470E3A6F30EC3DF00ED2C45128
:10737000030A05E126DA44DA30EC3DF006D2C451C6
:10738000050A05E11EDA3CDA30EC3DF0FED1C451CD
:10739000040A0CE116DAF20E396F420E386F010E54
:1073A0003B6F470E3A6F30EC3DF0EFD1C451060A07
:1073B00005E107DA1CDA30EC3DF0E7D1C451080AE8
:1073C00005E1FFD914DA30EC3DF0DFD1C451070AF2
:1073D0000CE1F7D9F20E396FAB0E386F010E3B6F2F
:1073E000470E3A6F30EC3DF0D0D1C451360A0CE173
:1073F000E8D9F10E396FF70E386F010E3B6F470E6B
:107400003A6F30EC3DF0C1D1C451370A0CE1D9D903
:10741000F20E396F060E386F010E3B6F470E3A6F52
:1074200030EC3DF0B2D1C451990A0CE1CAD9F10E49
:10743000396F430E386F010E3B6F470E3A6F30ECD9
:107440003DF0A3D1C451390A0CE1BBD9F10E396F1B
:10745000520E386F010E3B6F470E3A6F30EC3DF025
:1074600094D1C46712D01F0E01014E25366F376BC1
:10747000050E3723F10E396FD90E386F010E3B6FB1
:10748000470E3A6F30EC3DF080D1C451780A0CE1E0
:1074900098D9F10E396FE80E386F010E3B6F470E29
:1074A0003A6F30EC3DF071D1C451700A0CE189D9CA
:1074B000F10E396F700E386F010E3B6F470E3A6F49
:1074C00030EC3DF062D1C451400A0CE17AD9F20EA1
:1074D000396F600E386F010E3B6F470E3A6F30EC1C
:1074E0003DF053D1C451410A0CE16BD9F20E396F12
:1074F000C90E386F010E3B6F470E3A6F30EC3DF00E
:1075000044D1C451420A0CE15CD9F20E396F6F0EBE
:10751000386F010E3B6F470E3A6F30EC3DF035D1BE
:10752000C451430A0CE14DD9F20E396FD80E386FB1
:10753000010E3B6F470E3A6F30EC3DF026D121EE45
:10754000C4F09F0EDF642DD0B00EC4612AD0C451A8
:10755000610F4C6F0A0E4C6115D01F0E01014E25B4
:10756000366F376B050E3723F00E396FB70E386F55
:10757000010E3B6F470E3A6F4CC13CF13D6B30EC56
:107580003DF003D11ED9F30E396F8C0E386F010E0A
:107590003B6F470E3A6F4CC13CF13D6B30EC3DF018
:1075A000F4D021EEC4F0AF0EDF642DD0C00EC46164
:1075B0002AD0C451510F4C6F0A0E4C6115D01F0ECA
:1075C00001014E25366F376B050E3723F00E396FEC
:1075D000A70E386F010E3B6F470E3A6F4CC13CF15E
:1075E0003D6B30EC3DF0D1D0ECD8F30E396F7D0E11
:1075F000386F010E3B6F470E3A6F4CC13CF13D6B4B
:1076000030EC3DF0C2D021EEC4F0CF0EDF642DD0BF
:10761000E00EC4612AD0C451310F4C6F0A0E4C6188
:1076200015D01F0E01014E25366F376B050E37231F
:10763000F00E396FD70E386F010E3B6F470E3A6F61
:107640004CC13CF13D6B30EC3DF09FD0BAD8F30E0D
:10765000396FAA0E386F010E3B6F470E3A6F4CC15F
:107660003CF13D6B30EC3DF090D021EEC4F0DF0EEC
:10767000DF642DD0F00EC4612AD0C451210F4C6FAD
:107680000A0E4C6115D01F0E01014E25366F376B67
:10769000050E3723F00E396FC70E386F010E3B6FA2
:1076A000470E3A6F4CC13CF13D6B30EC3DF06DD074
:1076B00088D8F30E396F9B0E386F010E3B6F470E63
:1076C0003A6F4CC13CF13D6B30EC3DF05ED021EEA9
:1076D000C4F0BF0EDF642DD0D00EC4612AD0C451D7
:1076E000410F4C6F0A0E4C6115D01F0E01014E2543
:1076F000366F376B050E3723F00E396FE70E386F94
:10770000010E3B6F470E3A6F4CC13CF13D6B30ECC4
:107710003DF03BD056D8F30E396FB90E386F010EDD
:107720003B6F470E3A6F4CC13CF13D6B30EC3DF086
:107730002CD0C451230A1EE0C451240A1BE0C451BA
:10774000250A18E0C451260A15E0C451270A12E0A0
:10775000C451280A0FE0C451300A0CE0C451150A84
:1077600009E0C451790A06E0C451840A03E0C45117
:10777000830A0DE126D8F10E396F610E386F010EC4
:107780003B6F470E3A6F30EC3DF036514D6F4D5127
:107790004625CAECF1F01F0E0101446F050E456F3E
:1077A00046514427000E45234D514427000E4523E2
:1077B0000E0E4425D96E000E4521DA6EDF6A36EFD3
:1077C00022F01F0E01014E25366F376B050E372351
:1077D0001200470E4E25D96EDA6A010EDA22C10E6A
:1077E0004D25E16EE26A010EE222E7501200F20E30
:1077F000396F9C0E386F010E3B6F470E3A6F1200C7
:10780000F20E396F330E386F010E3B6F470E3A6F31
:107810001200E8CF45F1460E0601C16F0101455146
:10782000310A0FE1FCDAD8B4B81902E0E3DA12D079
:10783000060E0101376FC10E366FF70E396F400E1D
:1078400059D14551910A16E1EADAD8B4B81909E0DC
:10785000060ED9DA386FB8C23AF1B9C23BF130EF4F
:107860003DF0060E0101376FC10E366FF70E396F0E
:107870004C0E40D14551320A0FE1D5DAD8B4BA19CD
:1078800002E0B8DA12D0060E0101376FC10E366F72
:10789000F70E396F940E2ED14551920A16E1C3DAD4
:1078A000D8B4BA1909E0060EAEDA386FBAC23AF1A6
:1078B000BBC23BF130EF3DF0060E0101376FC10E48
:1078C000366FF70E396FA00E15D14551330A0FE10F
:1078D000B2DAD8B4BC1902E08DDA12D0060E01017A
:1078E000376FC10E366FF70E396FE80E03D1455171
:1078F000930A16E1A0DAD8B4BC1909E0060E83DABF
:10790000386FBCC23AF1BDC23BF130EF3DF0060E1C
:107910000101376FC10E366FF70E396FF40EEAD0E2
:107920004551340A0FE183DAD8B4BE1902E062DAB5
:1079300012D0060E0101376FC10E366FF80E396F87
:107940000C0ED8D04551940A16E171DAD8B4BE199C
:1079500009E0060E58DA386FBEC23AF1BFC23BF1F9
:1079600030EF3DF0060E0101376FC10E366FF80E95
:10797000396F180EBFD04551990A0FE14CDAD8B4CF
:10798000C01902E037DA12D0060E0101376FC10EBE
:10799000366FF80E396F300EADD04551390A16E109
:1079A0003ADAD8B4C01909E0060E2DDA386FC0C231
:1079B0003AF1C1C23BF130EF3DF0060E0101376FE5
:1079C000C10E366FF80E396F3C0E94D04551890ABE
:1079D00009E1060E0101376FC10E366FF80E396FDF
:1079E000480E88D04551900A09E1060E0101376F13
:1079F000C10E366FF80E396F540E7CD04551980A7F
:107A000009E1060E0101376FC10E366FF70E396FAF
:107A1000040E70D04551350A09E1060E0101376F99
:107A2000C10E366FF60E396FC80E64D04551950AF7
:107A300009E1060E0101376FC10E366FF60E396F80
:107A4000D40E58D04551960A09E1060E0101376F50
:107A5000C10E366FF60E396FE00E4CD04551380A24
:107A600009E1060E0101376FC10E366FF60E396F50
:107A7000F80E40D04551710A09E1060E0101376F39
:107A8000C10E366FF60E396FEC0E34D04551850AB3
:107A900009E1060E0101376FC10E366FF70E396F1F
:107AA000700E28D04551880A09E1060E0101376F92
:107AB000C10E366FF70E396FC40E1CD04551460A01
:107AC00009E1060E0101376FC10E366FF80E396FEE
:107AD000000E10D04551450A09E1060E0101376F2D
:107AE000C10E366FF80E396F240E04D04551030ACB
:107AF00004E106D0386F30EF3DF04551050A09E149
:107B0000060E0101376FC10E366FF70E396F580E32
:107B1000F1D74551040A09E1060E0101376FC10E84
:107B2000366FF70E396F640EE5D74551060A01E14D
:107B300003D04551080A09E1060E0101376FC10E55
:107B4000366FF70E396FAC0ED5D74551070A09E1EC
:107B5000060E0101376FC10E366FF70E396FB80E82
:107B6000C9D74551360A09E1060E0101376FC10E2A
:107B7000366FF70E396F280EBDD74551370A09E128
:107B8000060E0101376FC10E366FF70E396F340ED6
